S01C00005354345F537065637472756D5F576F726B696E672E737265633B
S3150800800000000220A1940508F1940508F1940508DA
S31508008010F1940508F1940508F1940508000000009C
S31508008020000000000000000000000000F1940508B0
S31508008030F194050800000000F1940508018A050876
S31508008040F1940508F1940508F1940508F1940508DA
S31508008050F1940508F1940508F1940508F1940508CA
S31508008060F1940508F1940508F1940508F1940508BA
S31508008070F1940508F1940508F1940508F1940508AA
S315080080800D8A0508218A0508F1940508F194050862
S31508008090F1940508F1940508F1940508258B05085F
S315080080A0F1940508F1940508F1940508F19405087A
S315080080B0358A0508498A0508F1940508F1940508E2
S315080080C0F1940508F1940508F1940508F19405085A
S315080080D0F19405085D8A0508718A0508F194050872
S315080080E0598B0508F1940508F1940508F1940508DB
S315080080F0F1940508F1940508F1940508858A0508A0
S31508008100F1940508998A0508F1940508AD8A0508C9
S31508008110F1940508F1940508F1940508F194050809
S31508008120F1940508F1940508C18A0508D58A050859
S31508008130F19405080000000000000000F19405080D
S31508008140F1940508F1940508F1940508E98A0508EB
S31508008150F1940508FD8A0508118B0508F1940508B0
S31508008160F1940508F1940508F1940508F1940508B9
S31508008170F1940508F1940508F1940508000000003B
S3150800818000000000F194050800000000000000004F
S31508008190F19405080000000000000000F1940508AD
S315080081A0000000000000000000000000F19405082F
S315080081B0F1940508F1940508F1940508F194050869
S30D080081C0F1940508443322116D
S315080081D010B5054C237833B9044B13B10448AFF3F3
S315080081E000800123237010BDB41100200000000098
S315080081F0540C070808B5034B1BB103490348AFF3F2
S31508008200008008BD00000000B8110020540C0708C3
S3150800821010F8012B11F8013B012A28BF9A42F7D022
S31508008220D01A7047034613F8012B002AFBD1181AF7
S315080082300138704700000000000000000000000040
S3150800824001F0FF01102A2BDB10F0070F08D010F8F9
S31508008250013B013A8B422DD010F0070F42B3F6D1FD
S31508008260F0B441EA012141EA014122F007047FF016
S3150800827000070023F0E80256083C85EA010586EA6D
S31508008280010685FA47F5A3FA87F586FA47F6A5FAA9
S3150800829087F68EB9EED1F0BC01F0FF0102F00702B5
S315080082A032B110F8013B013A83EA010313B1F8D160
S315080082B00020704701387047002D06BF3546033841
S315080082C0073815F0010F07D1013015F4807F02BF7A
S315080082D0013015F4C03F0130F0BC0138704700BFCB
S315080082E081F0004102E000BF83F0004330B54FEA59
S315080082F041044FEA430594EA050F08BF90EA020FC6
S315080083001FBF54EA000C55EA020C7FEA645C7FEA58
S31508008310655C00F0E2804FEA5454D4EB5555B8BF7B
S315080083206D420CDD2C4480EA020281EA030382EAEC
S31508008330000083EA010180EA020281EA0303362D7E
S3150800834088BF30BD11F0004F4FEA01314FF4801C51
S315080083504CEA113102D0404261EB410113F0004F63
S315080083604FEA03334CEA133302D0524263EB43031A
S3150800837094EA050F00F0A780A4F10104D5F1200EB8
S315080083800DDB02FA0EFC22FA05F2801841F1000113
S3150800839003FA0EF2801843FA05F359410EE0A5F1E7
S315080083A020050EF1200E012A03FA0EFC28BF4CF018
S315080083B0020C43FA05F3C01851EBE37101F00045CE
S315080083C007D54FF0000EDCF1000C7EEB00006EEBDB
S315080083D00101B1F5801F1BD3B1F5001F0CD3490865
S315080083E05FEA30004FEA3C0C04F101044FEA4452BC
S315080083F012F5800F80F09A80BCF1004F08BF5FEA43
S31508008400500C50F1000041EB045141EA050130BD22
S315080084105FEA4C0C404141EB0101013C28BFB1F534
S31508008420801FE9D291F0000F04BF01460020B1FA7F
S3150800843081F308BF2033A3F10B03B3F120020CDA52
S315080084400C3208DD02F1140CC2F10C0201FA0CF030
S3150800845021FA02F10CE002F11402D8BFC2F1200C95
S3150800846001FA02F120FA0CFCDCBF41EA0C0190404B
S31508008470E41AA2BF01EB0451294330BD6FEA040494
S315080084801F3C1CDA0C340EDC04F11404C4F120027F
S3150800849020FA04F001FA02F340EA030021FA04F391
S315080084A045EA030130BDC4F10C04C4F1200220FAE8
S315080084B002F001FA04F340EA0300294630BD21FA26
S315080084C004F0294630BD94F0000F83F4801306BFEC
S315080084D081F480110134013D4EE77FEA645C18BFE0
S315080084E07FEA655C29D094EA050F08BF90EA020F77
S315080084F005D054EA000C04BF1946104630BD91EA6F
S31508008500030F1EBF0021002030BD5FEA545C05D171
S315080085104000494128BF41F0004130BD14F58004B0
S315080085203CBF01F5801130BD01F0004545F0FE4124
S3150800853041F470014FF0000030BD7FEA645C1ABF59
S31508008540194610467FEA655C1CBF0B46024650EA90
S31508008550013406BF52EA033591EA030F41F40021BC
S3150800856030BD00BF90F0000F04BF0021704730B542
S315080085704FF4806404F132044FF000054FF0000117
S3150800858050E700BF90F0000F04BF0021704730B5D8
S315080085904FF4806404F1320410F0004548BF4042AD
S315080085A04FF000013EE700BF42004FEAE2014FEA02
S315080085B031014FEA02701FBF12F07F4393F07F4FDD
S315080085C081F06051704732F07F4208BF704793F0E0
S315080085D07F4F04BF41F40021704730B54FF46074F3
S315080085E001F0004521F000411CE700BF50EA0102F6
S315080085F008BF704730B54FF000050AE050EA01029F
S3150800860008BF704730B511F0004502D5404261EB0E
S3150800861041014FF4806404F132045FEA915C3FF44F
S31508008620D8AE4FF003025FEADC0C18BF03325FEAEC
S31508008630DC0C18BF033202EBDC02C2F1200300FA9D
S3150800864003FC20FA02F001FA03FE40EA0E0021FAC2
S3150800865002F11444BDE600BF70B54FF0FF0C4CF4B0
S31508008660E06C1CEA11541DBF1CEA135594EA0C0F62
S3150800867095EA0C0F00F0DEF82C4481EA030621EA9D
S315080086804C5123EA4C5350EA013518BF52EA0335D8
S3150800869041F4801143F4801338D0A0FB02CE4FF08A
S315080086A00005E1FB02E506F00042E0FB03E54FF0BA
S315080086B00006E1FB03569CF0000F18BF4EF0010EB2
S315080086C0A4F1FF04B6F5007F64F5407404D25FEAAE
S315080086D04E0E6D4146EB060642EAC62141EA555161
S315080086E04FEAC52040EA5E504FEACE2EB4F1FD0CA3
S315080086F088BFBCF5E06F1ED8BEF1004F08BF5FEA21
S31508008700500E50F1000041EB045170BD06F00046D2
S3150800871046EA010140EA020081EA0301B4EB5C047F
S31508008720C2BFD4EB0C0541EA045170BD41F4801177
S315080087304FF0000E013C00F3AB8014F1360FDEBF9C
S31508008740002001F0004170BDC4F10004203C35DA78
S315080087500C341BDC04F11404C4F1200500FA05F3FB
S3150800876020FA04F001FA05F240EA020001F000429C
S3150800877021F0004110EBD37021FA04F642EB060112
S315080087805EEA430E08BF20EAD37070BDC4F10C043C
S31508008790C4F1200500FA04F320FA05F001FA04F200
S315080087A040EA020001F0004110EBD37041F10001EC
S315080087B05EEA430E08BF20EAD37070BDC4F12005F7
S315080087C000FA05F24EEA020E20FA04F301FA05F25F
S315080087D043EA020321FA04F001F0004121FA04F207
S315080087E020EA020000EBD3705EEA430E08BF20EAD7
S315080087F0D37070BD94F0000F0FD101F00046400011
S3150800880041EB010111F4801F08BF013CF7D041EA92
S31508008810060195F0000F18BF704703F00046520096
S3150800882043EB030313F4801F08BF013DF7D043EA67
S315080088300603704794EA0C0F0CEA135518BF95EA1D
S315080088400C0F0CD050EA410618BF52EA4306D1D1A4
S3150800885081EA030101F000414FF0000070BD50EAC3
S31508008860410606BF1046194652EA430619D094EA4D
S315080088700C0F02D150EA013613D195EA0C0F05D137
S3150800888052EA03361CBF104619460AD181EA03018B
S3150800889001F0004141F0FE4141F470014FF0000043
S315080088A070BD41F0FE4141F4780170BD70B54FF0DE
S315080088B0FF0C4CF4E06C1CEA11541DBF1CEA13555E
S315080088C094EA0C0F95EA0C0F00F0A7F8A4EB050440
S315080088D081EA030E52EA03354FEA013100F0888037
S315080088E04FEA03334FF0805545EA131343EA126300
S315080088F04FEA022245EA111545EA10654FEA0026B5
S315080089000EF000419D4208BF964244F1FD0404F56D
S31508008910407402D25B084FEA3202B61A65EB0305C9
S315080089205B084FEA32024FF480104FF4002CB6EB86
S31508008930020E75EB030E22BFB61A754640EA0C0006
S315080089405B084FEA3202B6EB020E75EB030E22BF46
S31508008950B61A754640EA5C005B084FEA3202B6EB87
S31508008960020E75EB030E22BFB61A754640EA9C0046
S315080089705B084FEA3202B6EB020E75EB030E22BF16
S31508008980B61A754640EADC0055EA060E18D04FEAD4
S31508008990051545EA16754FEA06164FEAC30343EA74
S315080089A052734FEAC2025FEA1C1CC0D111F4801F41
S315080089B00BD141EA00014FF000004FF0004CB6E73A
S315080089C011F4801F04BF01430020B4F1FD0C88BFD9
S315080089D0BCF5E06F3FF6AFAEB5EB030C04BFB6EBE4
S315080089E0020C5FEA500C50F1000041EB045170BDD7
S315080089F00EF0004E4EEA113114EB5C04C2BFD4EB04
S31508008A000C0541EA045170BD41F480114FF0000E87
S31508008A10013C90E645EA060E8DE60CEA135594EA03
S31508008A200C0F08BF95EA0C0F3FF43BAF94EA0C0F06
S31508008A300AD150EA01347FF434AF95EA0C0F7FF47B
S31508008A4025AF104619462CE795EA0C0F06D152EACF
S31508008A5003353FF4FDAE1046194622E750EA4106B3
S31508008A6018BF52EA43067FF4C5AE50EA41047FF4C4
S31508008A700DAF52EA43057FF4EBAE12E74FF0FF3C29
S31508008A8006E000BF4FF0010C02E000BF4FF0010CFA
S31508008A904DF804CD4FEA410C7FEA6C5C4FEA430C73
S31508008AA018BF7FEA6C5C1BD001B050EA410C0CBFC2
S31508008AB052EA430C91EA030F02BF90EA020F002024
S31508008AC0704710F1000F91EA030F58BF994208BF8B
S31508008AD090422CBFD8176FEAE37040F00100704748
S31508008AE04FEA410C7FEA6C5C02D150EA013C07D19F
S31508008AF04FEA430C7FEA6C5CD6D152EA033CD3D0EA
S31508008B005DF8040B704700BF8446104662468C46E3
S31508008B101946634600E000BF01B5FFF7B7FF002816
S31508008B2048BF10F1000F01BD4DF808EDFFF7F4FF3F
S31508008B300CBF012000205DF808FB00BF4DF808EDCA
S31508008B40FFF7EAFF34BF012000205DF808FB00BFED
S31508008B504DF808EDFFF7E0FF94BF012000205DF80F
S31508008B6008FB00BF4DF808EDFFF7CEFF94BF0120C4
S31508008B7000205DF808FB00BF4DF808EDFFF7C4FFBD
S31508008B8034BF012000205DF808FB00BF4FEA410C06
S31508008B907FEA6C5C02D150EA013C0AD14FEA430CE9
S31508008BA07FEA6C5C02D152EA033C02D14FF0000026
S31508008BB070474FF0010070474FEA410212F5001264
S31508008BC015D211D56FF47873B3EB625212D94FEA06
S31508008BD0C12343F0004343EA505311F0004F23FAF0
S31508008BE002F018BF404270474FF00000704750EA45
S31508008BF0013005D111F0004008BF6FF00040704702
S31508008C004FF00000704700BF4A0011D212F500125B
S31508008C1011D20DD56FF47873B3EB62520ED44FEAC6
S31508008C20C12343F0004343EA505323FA02F0704746
S31508008C304FF00000704750EA013002D14FF0FF3084
S31508008C4070474FF0000070474FEA4102B2F1E04327
S31508008C5024BFB3F5001CDCF1FE5C0DD901F0004C15
S31508008C604FEAC0024CEA5070B2F1004F40EB830065
S31508008C7008BF20F00100704711F0804F21D113F191
S31508008C803872BCBF01F00040704741F480114FEACA
S31508008C905252C2F11802C2F1200C10FA0CF320FA53
S31508008CA002F018BF40F001004FEAC1234FEAD32370
S31508008CB003FA0CFC40EA0C0023FA02F34FEA4303DA
S31508008CC0CCE77FEA625307D150EA01331EBF4FF063
S31508008CD0FE4040F44000704701F0004040F0FE407E
S31508008CE040F40000704700BF53B94AB9002908BFCD
S31508008CF000281CBF4FF0FF314FF0FF3000F0A4B939
S31508008D00ADF1080C6DE904CE00F03CF8DDF804E09E
S31508008D10DDE9022304B0704738B500220023044673
S31508008D200D46FFF70BFF28B920462946BDE838400F
S31508008D3000F00AB8204605F1004100F005F8404267
S31508008D4061EB410138BD00BFD0B50C4B0022064689
S31508008D500F46FFF781FCFFF757FF0446FFF702FCB3
S31508008D60074B0022FFF778FC02460B463046394689
S31508008D70FFF7BAFAFFF748FF2146D0BD0000F03DDD
S31508008D800000F0412DE9F047089D04468C46002B6B
S31508008D9040F083808A42174647D9B2FA82F242B136
S31508008DA0C2F1200024FA00F09140974040EA010CF5
S31508008DB094404FEA1748230CBCFBF8F61FFA87FEC7
S31508008DC008FB16C143EA014306FB0EF1994209D98D
S31508008DD0FB1806F1FF3080F01981994240F216819E
S31508008DE0023E3B445B1AA4B2B3FBF8F008FB10330F
S31508008DF044EA034400FB0EFEA64509D93C1900F1D6
S31508008E00FF3380F00581A64540F2028102383C44D2
S31508008E1040EA0640A4EB0E0400261DB1D440002308
S31508008E20C5E900433146BDE8F08702B9FFDEB2FA6C
S31508008E3082F2002A50D1CB1B4FEA174E1FFA87F849
S31508008E400126B3FBFEFC210C0EFB1C3341EA034151
S31508008E5008FB0CF38B4207D979180CF1FF3002D2C4
S31508008E608B4200F2E9808446C91AA3B2B1FBFEF030
S31508008E700EFB101143EA014408FB00F8A04507D988
S31508008E803C1900F1FF3302D2A04500F2D9801846FA
S31508008E90A4EB080440EA0C40BFE78B4209D9002D31
S31508008EA000F0B1800026C5E9000130463146BDE82C
S31508008EB0F087B3FA83F6002E4AD18B4202D3824258
S31508008EC000F2B880841A61EB030101208C46002D5C
S31508008ED0A8D0C5E9004CA5E7C2F1200320FA03F69D
S31508008EE0974001FA02F04FEA174ED9403043030C77
S31508008EF0B1FBFEF61FFA87F80EFB161143EA01438B
S31508008F0006FB08F1994204FA02F409D9FB1806F19E
S31508008F10FF3C80F08D80994240F28A80023E3B44B5
S31508008F205B1A81B2B3FBFEF00EFB103341EA034134
S31508008F3000FB08F38B4207D9791800F1FF3C73D27E
S31508008F408B4271D902383944CB1A40EA064678E78B
S31508008F50C6F1200C03FA06F422FA0CF31C4320FA95
S31508008F600CF701FA06F34FEA144E21FA0CF11F43E7
S31508008F703B0CB1FBFEF91FFA84F80EFB191143EA04
S31508008F80014109FB08FA8A4502FA06F200FA06F3D5
S31508008F9008D9611809F1FF3048D28A4546D9A9F19E
S31508008FA002092144A1EB0A01BFB2B1FBFEF00EFB98
S31508008FB0101147EA014700FB08F8B84507D9E71931
S31508008FC000F1FF312ED2B8452CD90238274440EAA1
S31508008FD00940A7EB0807A0FB02894F45C646494644
S31508008FE01AD317D05DB1B3EB0E0267EB010707FA88
S31508008FF00CFCF2404CEA0202F740C5E900270026BD
S315080090003146BDE8F0872E4628460BE70646E9E6D0
S315080090101846FDE64345E5D2B8EB020E69EB0401B6
S315080090200138DFE70846D2E760468DE78146B9E7AB
S31508009030664675E730464AE7ACF1020C394413E751
S3150800904002383C4424E700BF704700BF80B483B0B1
S3150800905000AF78607B689B6818460C37BD465DF89C
S31508009060047B704780B483B000AF78607B681B6868
S3150800907018460C37BD465DF8047B704790B583B03B
S3150800908000AF786039603B68002B01D100230DE002
S315080090907B681B6804331C683868FFF7C3F8034607
S315080090A01A4639687868A047034600BF18460C3741
S315080090B0BD4690BD80B586B000AFF860B9607A60ED
S315080090C000237B617B685A1E7A60002B14BF01233C
S315080090D00023DBB2002B0ED0FB681B681A68BB683E
S315080090E0591CB9601B781946F868904702467B698F
S315080090F013447B61E6E77B6918461837BD4680BD91
S3150800910080B582B000AF7860396039687868FFF753
S31508009110B5FF034618460837BD4680BD80B582B000
S3150800912000AF786004497868FFF7A8FF0346184639
S315080091300837BD4680BD00BF700C070880B584B0EF
S3150800914000AF7860396039687868FFF7D9FFF8604A
S315080091507868FFF7E3FF0246FB681344FB60FB6889
S3150800916018461037BD4680BD80B582B000AF78601E
S315080091700B46FB707B681B6804331B68F91C0122CD
S3150800918078689847034618460837BD4680BD80B5B7
S3150800919086B000AFF860B9607A60BB687B61FB682F
S315080091A018697B689AB24FF0FF33796958F03CFB2F
S315080091B07B6818461837BD4680BD80B584B000AFB9
S315080091C078607B68186907F10F014FF0FF330122B9
S315080091D058F0BCFBFB7B18461037BD4680BD80B4F3
S315080091E083B000AF78604FF0FF3318460C37BD46A2
S315080091F05DF8047B704780B483B000AF78604FF0A9
S31508009200FF3318460C37BD465DF8047B704780B4BB
S3150800921083B000AF786000BF0C37BD465DF8047BAD
S31508009220704780B582B000AF78600B46FB70FB785C
S315080092301946786800F0A6F97B6818460837BD46CF
S3150800924080BD80B582B000AF78603960786800F07C
S3150800925041F83B68002B08D03868FEF7E3FF034661
S315080092601A463968786800F0ACF87B6818460837FB
S31508009270BD4680BD80B582B000AF78603960786839
S3150800928000F028F83968786800F0FCF87B6818461A
S315080092900837BD4680BD80B582B000AF78603960BA
S315080092A0786800F017F83968786800F0AFF87B68D6
S315080092B018460837BD4680BD80B582B000AF7860D5
S315080092C07B681B68184663F0F9F97B681846083707
S315080092D0BD4680BD80B483B000AF78607B6800224D
S315080092E01A607B6800225A607B6800229A6000BF79
S315080092F00C37BD465DF8047B704780B582B000AF79
S3150800930078607B681B68002B04D07B681B6818464E
S3150800931063F0D4F97B6800221A607B6800229A60A1
S315080093207B689A687B685A6000BF0837BD4680BD6F
S3150800933080B582B000AF786039607B681B68002B07
S3150800934006D07B685B683A689A4201D8012316E022
S315080093503968786800F017F80346002B14BF012314
S315080093600023DBB2002B09D07B689B68002B03D156
S315080093707B681B6800221A70012300E00023184648
S315080093800837BD4680BD80B584B000AF78603960C7
S315080093907B681A683B6801331946104663F0F2FE8B
S315080093A0F860FB68002B07D07B68FA681A607B6850
S315080093B03A685A60012300E0002318461037BD4674
S315080093C080BD80B584B000AFF860B9607A6079680E
S315080093D0F868FFF7ADFF0346002B0CBF01230023F7
S315080093E0DBB2002B04D0F868FFF787FFFB6809E0BB
S315080093F0FB687A689A60FB681B68B968184663F068
S315080094008DFFFB6818461037BD4680BD80B582B013
S3150800941000AF786039607B681B68002B1AD07B68C0
S315080094205A683B689B689A420FD37B681A683B6800
S315080094301B681946104663F071FF3B689A687B689B
S315080094409A603B6800229A6019E07B681B68184698
S3150800945063F034F93B681A687B681A603B685A6897
S315080094607B685A603B689A687B689A603B6800220A
S315080094701A603B6800225A603B6800229A600837E7
S31508009480BD4680BD80B582B000AF786039607A6825
S315080094903B689A4201D17B6810E03B681B68002B49
S315080094A008D03B6819683B689B681A467868FFF7D6
S315080094B088FF02E07868FFF720FF7B6818460837C0
S315080094C0BD4680BD80B582B000AF786039607A68E5
S315080094D03B689A4203D039687868FFF797FF7B683C
S315080094E018460837BD4680BD80B582B000AF7860A3
S315080094F039603B68002B09D03868FEF793FE0346AF
S315080095001A4639687868FFF75CFF02E07868FFF763
S31508009510F4FE7B6818460837BD4680BD80B586B020
S3150800952000AFF860B9607A60FB689B687A68134494
S315080095307B61BB68002B01D100231FE07B68002BF1
S3150800954001D101231AE07969F868FFF7F1FE0346AD
S31508009550002B0CBF01230023DBB2002B01D0002314
S315080095600CE0FB681A68FB689B681344B9681846E0
S3150800957063F0D4FEFB687A699A60012318461837A7
S31508009580BD4680BD80B584B000AF78600B46FB70E1
S31508009590FB783B7300237B7307F10C030122194602
S315080095A07868FFF7BBFF034618461037BD4680BDEF
S315080095B080B582B000AF786039607B689B68002B05
S315080095C00AD13B68002B03D03B681B78002B01D1DE
S315080095D0012300E0002317E03B68002B08D17B68D5
S315080095E01B681B78002B0CBF01230023DBB20BE0A2
S315080095F07B681B6839681846FEF70AFE0346002B87
S315080096000CBF01230023DBB218460837BD4680BDD0
S3150800961080B483B000AF786039607B689B683A682D
S315080096209A4203D27B681B68002B04D1074B0022A1
S315080096301A70064B03E07B681A683B6813441846A1
S315080096400C37BD465DF8047B704700BFD01100207B
S3150800965080B586B000AFF8600B467A60FB72FB688F
S315080096609B687A689A4202D34FF0FF3313E0FB688F
S315080096701A687B681344FA7A1146184663F041FE65
S3150800968078617B69002B02D14FF0FF3303E0FB685A
S315080096901B687A69D31A18461837BD4680BD00007C
S315080096A080B586B000AFF860B9607A603B607A68CA
S315080096B03B689A4205D93B687B617B683B607B695E
S315080096C07B601849F868FFF7BCFDBB689B687A6839
S315080096D09A4222D2BB689B683A689A4202D9BB680A
S315080096E09B683B60BB681A683B6813441B78FB742D
S315080096F0BB681A683B68134400221A70BB681A686C
S315080097007B6813441946F868FFF7EEFEBB681A68CB
S315080097103B681344FA7C1A7000E000BFF8681837F3
S31508009720BD4680BD840C070880B582B000AF78605E
S315080097307B681B68002B06D07B681B68184662F09E
S3150800974086FF034600E0002318460837BD4680BD5D
S3150800975080B588B004AF03463960FB801346BB80EA
S31508009760FA88BB88134440F2FE32934201DD002397
S3150800977019E0FB88184600F048F90346FB73FB8896
S31508009780BB73FB7B99B2BB7B9AB20E230293BB8851
S3150800979001933B6800930123054851F087FE042096
S315080097A04FF01AFF012318461037BD4680BD00BF8B
S315080097B07C8D012080B588B004AF03463960FB80F4
S315080097C01346BB803B68FB60FA88BB88134440F2AB
S315080097D0FE32934201DD002319E0FB88184600F0AB
S315080097E014F90346FB72FB88BB72FB7A99B2BB7A03
S315080097F09AB20E230293BB880193FB680093012358
S31508009800054851F053FE04204FF0E6FE01231846A2
S315080098101037BD4680BD00BF7C8D012080B588B05D
S3150800982004AF03463960FB801346BB803B681B8840
S315080098301B12DBB23B733B681B88DBB27B73FA886F
S31508009840BB88134440F2FE32934201DD00231AE03E
S31508009850FB88184600F0D9F80346FB73FB88BB73F0
S31508009860FB7B99B2BB7B9AB20E230293BB8801930A
S3150800987007F10C0300930123054851F017FE042055
S315080098804FF0AAFE012318461037BD4680BD00BF1B
S315080098907C8D012080B588B004AF03463960FB8013
S315080098A01346BB80FA88BB88134440F2FE329342C3
S315080098B001DD002316E0FB88184600F083F803460E
S315080098C0FB73FB88BB73FB7B99B2BB7B9AB20E23F7
S315080098D00293BB8801933B6800930123034851F028
S315080098E0DFFE012318461037BD4680BD7C8D01205A
S315080098F080B588B004AF03463960FB801346BB8049
S31508009900FA88BB88134440F2FE32934201DD0023F5
S3150800991022E0FB88184600F055F80346FB73FB88DF
S31508009920BB73FB7B99B2BB7B9AB20E230293BB88AF
S31508009930019307F1080300930123094851F0B0FE8B
S315080099403B7A1B021AB27B7A1BB213431BB2BB814A
S315080099503B68BA891A80012318461037BD4680BD70
S315080099607C8D012080B588B004AF03463960FB8042
S315080099701346BB803B68FB60FA88BB88134440F2F9
S31508009980FE32934201DD002316E0FB88184600F0FC
S3150800999019F80346FB72FB88BB72FB7A99B2BB7A4D
S315080099A09AB20E230293BB880193FB6800930123A6
S315080099B0034851F075FE012318461037BD4680BD91
S315080099C07C8D012080B483B000AF0346FB80FB8802
S315080099D0FF2B01D8A12312E0FB88B3F5007F01D243
S315080099E0A3230CE0FB88B3F5407F01D2A52306E04C
S315080099F0FB88B3F5806F01D2A72300E0A72318469A
S31508009A000C37BD465DF8047B704780B483B000AF61
S31508009A100346FB80FB88FF2B01D8A02312E0FB88B6
S31508009A20B3F5007F01D2A2230CE0FB88B3F5407F93
S31508009A3001D2A42306E0FB88B3F5806F01D2A623E2
S31508009A4000E0A62318460C37BD465DF8047B704730
S31508009A5080B584B000AF78600B46FB70FB7819467A
S31508009A60786800F04DFA0346FB73FB7B002B03D1A5
S31508009A70786800F029F81BE0FB7B012B17D0FB7BED
S31508009A80052B04D10C490D48FFF758FB10E0FB7B6A
S31508009A90022B04D10A490948FFF750FB08E0FB7B73
S31508009AA0032B05D107490548FFF748FB00E000BF2F
S31508009AB01037BD4680BD00BF880C0708401E012030
S31508009AC0980C0708A40C070880B582B000AF786028
S31508009AD0786800F019F97B6803F5197319467868F0
S31508009AE000F0B4FA02467B68DA637B68DA6B7B6857
S31508009AF0D3F850321A447B681A607B6803F51A73E8
S31508009B001946786800F0A2FA02467B681A647B68F0
S31508009B101A6C7B68D3F854321A447B685A607B689F
S31508009B2003F51B731946786800F090FA02467B68BD
S31508009B305A647B685A6C7B68D3F858321A447B6837
S31508009B409A607B6803F51C731946786800F07EFAFC
S31508009B5002467B68DA607B6803F51D7319467868E8
S31508009B6000F074FA02467B681A617B6803F51E7377
S31508009B701946786800F054FA03461A467B681A8331
S31508009B807B6803F27A231946786800F049FA034697
S31508009B901A467B685A837B6803F51F7319467868EB
S31508009BA000F03EFA03461A467B689A837B6893F868
S31508009BB07E227B6883F824207B6893F87F227B6863
S31508009BC083F825207B6893F880227B6883F8262013
S31508009BD07B6893F881227B6883F827207B6893F853
S31508009BE082227B6883F82E207B6893F883227B6821
S31508009BF083F82F207B6893F884227B6883F83020CB
S31508009C007B6893F885227B6883F831207B6893F814
S31508009C1086227B6883F832207B6893F887227B68E4
S31508009C2083F833207B6893F888227B6883F834208E
S31508009C307B6893F889227B6883F835207B6893F8DC
S31508009C408A227B6883F836207B6893F88B227B68A8
S31508009C5083F837207B6893F88C227B6883F8382052
S31508009C607B6893F88D227B6883F839207B6893F8A4
S31508009C708E227B6883F83A207B6893F88F227B686C
S31508009C8083F83B207B6803F523731946786800F050
S31508009C90DDF902467B685A617B6803F52473194629
S31508009CA0786800F0BDF903461A467B689A857B6892
S31508009CB093F892227B6883F848207B6893F893226E
S31508009CC07B6883F849207B6893F89432A3F1800275
S31508009CD07B681A627B6893F89532803B07EE903A68
S31508009CE0B8EEE77AF2EE046AC7EE267A7B68C3ED29
S31508009CF00A7A786800F019F87B68012283F85C22F2
S31508009D0000BF0837BD4680BD80B582B000AF786019
S31508009D107B687A6803F5FC7311464C22184662F094
S31508009D20D5FC00BF0837BD4680BD80B582B000AF00
S31508009D3078607B689B8D002B3AD07B68B3F8242229
S31508009D407B689B8D9A4210D07B689A8D7B68A3F8B6
S31508009D50F4217B68D3F8F8117B68D3F8FC217B687B
S31508009D60D3F80032786800F027F87B6893F8482023
S31508009D707B6893F877309A4204D17B68012283F88E
S31508009D804A2003E07B68002283F84A207B6893F820
S31508009D9049207B6893F897309A4204D17B68012260
S31508009DA083F84B2005E07B68002283F84B2000E00F
S31508009DB000BF0837BD4680BD80B485B000AFF860E7
S31508009DC0B9607A603B60FB68DB6BBA68D21AFB68DD
S31508009DD0C3F85022FB681B6C7A68D21AFB68C3F872
S31508009DE05422FB685B6C3A68D21AFB68C3F858229F
S31508009DF000BF1437BD465DF8047B704780B485B054
S31508009E0000AFF860B9607A603B60FB68DB7B0133C2
S31508009E10DAB2FB68DA73FB68DB7B002B02D1FB68DE
S31508009E200122DA73FB68BA681A61FB687A685A61B4
S31508009E30FB683A689A61BB699AB2FB689A8300BF65
S31508009E401437BD465DF8047B7047000080B582B0C4
S31508009E5000AF78607B6893F85C32002B16D07B687D
S31508009E60002283F85C227B68012283F818210A4BBA
S31508009E701B7883F00103DBB2002B05D0786800F06D
S31508009E8027F8054B01221A70012300E00023184623
S31508009E900837BD4680BD00BFD111002080B483B00D
S31508009EA000AF78607B689A8D084B1B889A4205D06C
S31508009EB07B689A8D054B1A80012300E0002318461B
S31508009EC00C37BD465DF8047B704700BFD2110020F1
S31508009ED080B582B000AF78600121786800F000FB99
S31508009EE00221786800F0FCFA0321786800F0F8FA95
S31508009EF00421786800F0F4FA00BF0837BD4680BD33
S31508009F0080B592B000AF78600B46FB7001237B6486
S31508009F107B6C3C2B10DC7B6C013B79687A6C0A44C1
S31508009F2002F25D2211787A6813440A4683F85D22A4
S31508009F307B6C01337B64EBE77B68FA7883F89922BC
S31508009F407B6893F85D32492B01D0012364E07B6876
S31508009F5093F85E32572B01D001235DE07B6893F8B6
S31508009F605F32412B01D0012356E07B6893F86032BB
S31508009F70502B01D001234FE07B6893F86132492BBF
S31508009F8001D0012348E07B6893F86232022B01D0A6
S31508009F90052341E07B6893F897323B2B01D00223D7
S31508009FA03AE07B6893F89832212B01D0022333E0FC
S31508009FB07B6893F899323B2B01D002232CE00023CF
S31508009FC03B643B6C332B0FDC3B6C05337A681344DC
S31508009FD093F85D1207F108023B6C13440A461A709F
S31508009FE03B6C01333B64ECE77B6893F8963287F861
S31508009FF03F3007F1080334221946786800F0C4FA9E
S3150800A000034687F83E3097F83F2097F83E309A4245
S3150800A01001D0032300E0002318464837BD4680BD1B
S3150800A02080B483B000AF786039603B681B781B0248
S3150800A0301AB23B6801331B781BB253401BB29BB262
S3150800A04018460C37BD465DF8047B704780B483B06C
S3150800A05000AF786039603B681B781A063B680133A5
S3150800A0601B781B045A403B6802331B781B0253407B
S3150800A0703A6803321278534018460C37BD465DF8E5
S3150800A080047B704780B5BCB002AF78600023C7F880
S3150800A090E0307B6803F219117B6803F24522D7F892
S3150800A0A0E03000930523786800F004FAC7F8E0006A
S3150800A0B07B6803F219117B6803F51172D7F8E03053
S3150800A0C000930123786800F0F5F9C7F8E0007B688B
S3150800A0D003F219117B6803F5FA72D7F8E03000939A
S3150800A0E00223786800F0E6F9C7F8E0007B6803F217
S3150800A0F019117A68D7F8E03000930423786800F0DD
S3150800A100D9F9C7F8E0007B6803F219117B681A1DB4
S3150800A110D7F8E03000930423786800F0CBF9C7F845
S3150800A120E0007B6803F219117B6803F10802D7F88F
S3150800A130E03000930423786800F0BCF9C7F8E00023
S3150800A1407B6803F219117B6803F14C02D7F8E030FB
S3150800A15000930923786800F0ADF9C7F8E0007B683A
S3150800A16003F219117B6803F16402D7F8E030009313
S3150800A1700123786800F09EF9C7F8E0007B6803F2CF
S3150800A18019117B6803F15502D7F8E03000930F23C5
S3150800A190786800F08FF9C7F8E0007B6803F21911B8
S3150800A1A07B6803F16802D7F8E03000930F237868DC
S3150800A1B000F080F9C7F8E0007B6803F219117B68A4
S3150800A1C003F17802D7F8E03000930423786800F0AA
S3150800A1D071F9C7F8E0007B6803F219117B6803F18F
S3150800A1E07C02D7F8E03000930423786800F062F91F
S3150800A1F0C7F8E0007B6803F219117B6803F1800257
S3150800A200D7F8E03000930423786800F053F9C7F8CC
S3150800A210E0007B6803F219117B6803F18402D7F822
S3150800A220E03000930223786800F044F9C7F8E000AC
S3150800A2307B6803F219117B6803F17702D7F8E030DF
S3150800A24000930123786800F035F9C7F8E0007B68C9
S3150800A25003F219117B6803F18802D7F8E0300093FE
S3150800A2600F23786800F026F9C7F8E0007B6803F248
S3150800A27019117B6803F19802D7F8E030009304239C
S3150800A280786800F017F9C7F8E0007B6803F219113F
S3150800A2907B6803F19C02D7F8E030009304237868C2
S3150800A2A000F008F9C7F8E0007B6803F219117B682B
S3150800A2B003F1A002D7F8E03000930423786800F091
S3150800A2C0F9F8C7F8E0007B6803F219117B6803F117
S3150800A2D0A402D7F8E03000930223786800F0EAF881
S3150800A2E0C7F8E0007B6803F219117B6803F197024F
S3150800A2F0D7F8E03000930123786800F0DBF8C7F858
S3150800A300E0007B6803F219117B6803F1A802D7F80D
S3150800A310E03000930F23786800F0CCF8C7F8E00027
S3150800A3207B6803F219117B6803F1B702D7F8E030AE
S3150800A33000930F23786800F0BDF8C7F8E0007B6843
S3150800A34003F219117B6803F1C602D7F8E0300093CF
S3150800A3500F23786800F0AEF8C7F8E0007B6803F2D0
S3150800A36019117B6803F1D502D7F8E03000930F2363
S3150800A370786800F09FF8C7F8E0007B6803F21911C7
S3150800A3807B6803F1E402D7F8E03000930F2378687E
S3150800A39000F090F8C7F8E0007B6803F219117B68B3
S3150800A3A003F1F302D7F8E03000930F23786800F042
S3150800A3B081F8C7F8E0007B6803F219117B6803F59A
S3150800A3C08272D7F8E03000930423786800F072F8B8
S3150800A3D0C7F8E0007B6803F219117B6803F58472FD
S3150800A3E0D7F8E03000930423786800F063F8C7F8DC
S3150800A3F0E0007B6803F219117B6803F58672D7F8CB
S3150800A400E03000930423786800F054F8C7F8E000B9
S3150800A4107B6803F219117B6803F58872D7F8E03078
S3150800A42000930823786800F045F8C7F8E000002391
S3150800A430C7F8E430D7F8E430D12B13DCD7F8E4308A
S3150800A44005337A68134493F8191107F10C02D7F803
S3150800A450E43013440A461A70D7F8E4300133C7F8D3
S3150800A460E430E7E707F10C03D2221946786800F0D2
S3150800A4708BF80346FB727B6803F2191107F10B028E
S3150800A480D7F8E03000930123786800F013F8C7F88E
S3150800A490E0007B6803F219117B6803F24A22D7F8B9
S3150800A4A0E03000930323786800F004F800BFE8372B
S3150800A4B0BD4680BD80B584B000AFF860B9607A60EB
S3150800A4C03B60BB69BA6813443A687968184662F013
S3150800A4D0FDF8BA693B68134418461037BD4680BD77
S3150800A4E080B483B000AF78600B46FB70FB78012B15
S3150800A4F00DD17B6893F82E20224B5B789A4239D08F
S3150800A5007B6893F82E201F4B5A70012333E0FB78A3
S3150800A510022B0DD17B6893F82F201A4B9B789A4211
S3150800A52028D07B6893F82F20164B9A70012322E0D7
S3150800A530FB78032B0DD17B6893F83020114BDB7821
S3150800A5409A4217D07B6893F830200E4BDA700123B5
S3150800A55011E0FB78042B0DD17B6893F83120094B69
S3150800A5601B799A4206D07B6893F83120054B1A71FD
S3150800A570012300E0002318460C37BD465DF8047B2E
S3150800A580704700BFD411002080B487B000AFF860D0
S3150800A590B9607A600023FB7400237B617A697B6863
S3150800A5A09A420ADABB685A1CBA601A78FB7C1344CA
S3150800A5B0FB747B6901337B61F0E7FB7C18461C372B
S3150800A5C0BD465DF8047B704780B483B000AF786001
S3150800A5D000BF0C37BD465DF8047B704780B483B076
S3150800A5E000AF786039603B681B68002B06D17B6832
S3150800A5F000221A607B6800225A6005E07B68054ADB
S3150800A6001A607B6800225A6078680C37BD465DF888
S3150800A610047B7047C9A5000880B483B000AF786092
S3150800A620002318460C37BD465DF8047B704780B496
S3150800A63083B000AF7860002318460C37BD465DF836
S3150800A640047B704780B485B000AFF860B9601346E4
S3150800A650FB7100BF1437BD465DF8047B704780B4B4
S3150800A66083B000AF786000BF0C37BD465DF8047B49
S3150800A670704780B483B000AF7860002318460C3763
S3150800A680BD465DF8047B7047B0B588B002AFF86088
S3150800A6907A603B600B46FB72F868F97A02230093EE
S3150800A6A0FB6A7A6801F0C2FB224AFB681A60FB68FB
S3150800A6B02C3300221A605A601A81FB68403303243F
S3150800A6C01D46002C06DB1C492846FEF7BAFD0C354C
S3150800A6D0013CF6E73B68002B1ED000237B617B69B3
S3150800A6E0032B16DC7A6913465B0013449B00403340
S3150800A6F0FA68D0187A6913465B0013449B001A4619
S3150800A7003B6813441946FEF7BDFE7B6901337B613E
S3150800A710E5E7FB683A6B9A63BB6A002B02D0FB68D5
S3150800A720BA6ADA63FB680122DA71FB6818461837D9
S3150800A730BD46B0BD50400708B40C070890B585B0B3
S3150800A74000AF78600B46FB707B68184601F04EFC3C
S3150800A7507B6840331846FEF779FC0346002B0CBF8E
S3150800A76001230023DBB2002B33D07A687B6893F889
S3150800A77020301946104601F0BFFCFB78002B08D0A4
S3150800A780554B1988554B1B789AB2554B55480DF0C1
S3150800A79008F9554B1B881C467B68083319465148EF
S3150800A7A00DF008FA0346E31ADA0F13445B109AB25F
S3150800A7B0494B1B8813449AB2474B1A80464B198853
S3150800A7C0464B1B789AB27B68083346480DF0E9F881
S3150800A7D07DE07A687B6893F82030013BDBB2194646
S3150800A7E0104601F089FCFB78002B08D03A4B1988F3
S3150800A7F03A4B1B789AB23A4B3A480DF0D2F87B6836
S3150800A80008331A4639493A4862F018FD364B1B8810
S3150800A8101C46374933480DF0CDF90346E31A9AB278
S3150800A8202D4B1B8813449AB22B4B1A802A4B198836
S3150800A8302A4B1B789AB22E4B2A480DF0B2F87B6841
S3150800A8409B6B1B781A4613465B0013449B004033E8
S3150800A8507A681A4407F1080311461846FFF7BEFE40
S3150800A860BB68002B06D1FB6803F00103002B01D15E
S3150800A870012300E0002383F00103DBB2002B26D07E
S3150800A8807A687B6893F820300133DBB219461046A4
S3150800A89001F032FC7B689B6B1B781A4613465B00FB
S3150800A8A013449B0040337A6813441846FEF7DAFBD4
S3150800A8B003461A460F490E4862F0C0FC064B198833
S3150800A8C0064B1B789AB20A4B06480DF06AF800BF89
S3150800A8D01437BD4690BD00BFDC110020DE110020F4
S3150800A8E0B80C0708B48C0120DA110020BC0C070844
S3150800A8F0E0110020C40C070880B483B000AF78606C
S3150800A900396000BF0C37BD465DF8047B704780B5DB
S3150800A91082B000AF78600B46FB707B68FA78114608
S3150800A920184601F0DBFA7B68DB6B18460837BD462C
S3150800A93080BD80B483B000AF7860002318460C371A
S3150800A940BD465DF8047B704780B582B000AF78607D
S3150800A95039607B682C333968184662F0DFFC00BF23
S3150800A9600837BD4680BD000090B583B000AF78605B
S3150800A9700E4A7B681A607B684033002B0CD07B68D4
S3150800A980403303F130047B6840339C4204D00C3CCE
S3150800A9902046FEF791FCF6E77B68184601F088FA30
S3150800A9A07B6818460C37BD4690BD00BF5040070867
S3150800A9B080B582B000AF78607868FFF7D5FF702160
S3150800A9C0786860F093FC7B6818460837BD4680BDFA
S3150800A9D080B483B000AF7860396000BF0C37BD46DD
S3150800A9E05DF8047B704780B483B000AF7860396047
S3150800A9F03B6818460C37BD465DF8047B704780B542
S3150800AA0082B000AF7860786800F014FD7B6818465D
S3150800AA100837BD4680BD80B582B000AF78607B68D8
S3150800AA20184600F0F7FC7B6818460837BD4680BD17
S3150800AA3080B582B000AF78607B681846FFF7EBFFF9
S3150800AA407B6818460837BD4680BD000080B588B0CB
S3150800AA5002AFF8607A603B600B46FB72F868F97AD9
S3150800AA60022300933B6A7A6801F0E0F9444AFB68DE
S3150800AA701A60FB682C3343491846FEF7E2FBFB686D
S3150800AA803C3340491846FEF7DCFBFB683E4A4C332C
S3150800AA9011469822184661F019FEFB68E4331846F9
S3150800AAA0FFF7C6FFFB683A685A62FB68002283F81C
S3150800AAB03820FB683C33F96A1846FEF7E3FCFB6866
S3150800AAC00422DA7100237B61FB685B6A1846FEF78D
S3150800AAD0BDFA02467B699A428CBF01230023DBB28A
S3150800AAE0002B2AD0FB685B6A1846FEF7BBFA0246BB
S3150800AAF07B6913441B7897F824209A420CBF0123DC
S3150800AB000023DBB2002B0AD0FB68E4332522BA7493
S3150800AB1007F112021146184600F0CBFC09E0FB6863
S3150800AB20E4332422FA7407F113021146184600F09A
S3150800AB30C0FC7B6901337B61C6E7FB685B6A184624
S3150800AB40FEF784FA0346DAB2FB6883F82820FB6826
S3150800AB5003F12C02FB685B6A19461046FEF792FC65
S3150800AB60FB6897F8282083F8F020FB6897F82420DC
S3150800AB7083F84820FB6818461837BD4680BD00BFD5
S3150800AB8088400708600D0708640D070880B588B077
S3150800AB9002AFF8607A603B600B46FB72F868F97A98
S3150800ABA097F8203000937B6A7A6801F03FF9414AAA
S3150800ABB0FB681A60FB682C333F491846FEF741FBD1
S3150800ABC0FB683C333C491846FEF73BFBFB683B4AAF
S3150800ABD04C3311469822184661F078FDFB68E43339
S3150800ABE01846FFF725FFFB683A685A62FB68002299
S3150800ABF083F83820FB680422DA7100237B61FB683E
S3150800AC005B6A1846FEF722FA02467B699A428CBFAF
S3150800AC1001230023DBB2002B2AD0FB685B6A1846A7
S3150800AC20FEF720FA02467B6913441B7897F828201A
S3150800AC309A420CBF01230023DBB2002B0AD0FB6823
S3150800AC40E4332522BA7407F112021146184600F0B9
S3150800AC5030FC09E0FB68E4332422FA7407F1130296
S3150800AC601146184600F025FC7B6901337B61C6E76F
S3150800AC70FB685B6A1846FEF7E9F90346DAB2FB6831
S3150800AC8083F82820FB6803F12C02FB685B6A1946E7
S3150800AC901046FEF7F7FBFB6897F82C2083F8F020A0
S3150800ACA0FB6897F8282083F84820FB681846183769
S3150800ACB0BD4680BD88400708600D0708640D070873
S3150800ACC080B582B000AF78600D4A7B681A607B68F1
S3150800ACD0E433184600F0D2FB7B683C331846FEF78F
S3150800ACE0EBFA7B682C331846FEF7E6FA7B681846BB
S3150800ACF001F0DEF87B6818460837BD4680BD00BF00
S3150800AD008840070880B582B000AF78607868FFF79A
S3150800AD10D7FFF421786860F0E9FA7B6818460837A7
S3150800AD20BD4680BD80B582B000AF78600B46FB702B
S3150800AD307B68FA781146184601F0D0F87B6893F8D4
S3150800AD40F030002B04D07B6893F8F030012B04D147
S3150800AD507B68002283F8492008E07B6893F8F03086
S3150800AD60022B03D17B681A2283F849207B680022CC
S3150800AD7083F83820002318460837BD4680BD80B4BE
S3150800AD8083B000AF786000BF18460C37BD465DF843
S3150800AD90047B7047B0B588B002AF78600B46FB708D
S3150800ADA07B68184601F022F97A687B6893F82030A8
S3150800ADB01946104601F0A0F9FB78002B08D0844B01
S3150800ADC01988844B1B789AB2834B84480CF0E9FDAA
S3150800ADD07B6808331A468249824862F02FFA824B0A
S3150800ADE01B881C467F497D480CF0E4FE0346E31A9F
S3150800ADF09AB2774B1B8813449AB2754B1A80744BD8
S3150800AE001988744B1B789AB2764B74480CF0C9FDB6
S3150800AE107B681B79002B40F093807A687B6893F8EF
S3150800AE2020300233DBB21946104601F065F96F4946
S3150800AE306A480CF0BFFE03461A46654B1B88134446
S3150800AE409AB2634B1A8000237B617B685B6A18465B
S3150800AE50FEF7FCF802467B699A428CBF0123002361
S3150800AE60DBB2002B00F0B08003215C480DF03DF901
S3150800AE707B6893F838301A467B69934237D17B68EA
S3150800AE8093F949307A6812339B0013445B68FB6078
S3150800AE904F4B1C884F4B1B789DB2F9684F480CF0F6
S3150800AEA089FE03461A46524B1B789BB200931346FB
S3150800AEB02A46214649480DF040FD002147480DF035
S3150800AEC014F9434B1988434B1B789AB2FB684348DD
S3150800AED00CF067FDF96841480CF06CFE03461A460B
S3150800AEE03B4B1B8813449AB2394B1A8024E07B6883
S3150800AEF0E4337A691146184600F0ECFA034693F9EA
S3150800AF0000307A6812339B0013445B683B61304B10
S3150800AF101988304B1B789AB23B6930480CF041FDD2
S3150800AF2039692E480CF046FE03461A46284B1B88FC
S3150800AF3013449AB2264B1A807B6901337B6184E7F6
S3150800AF407A687B6893F820300233DBB219461046DC
S3150800AF5001F0D2F87B683C331846FEF783F80346BF
S3150800AF601A4624491F4862F069F9194B1988194B82
S3150800AF701B789AB21B4B19480CF013FD7B683C33BF
S3150800AF801846FEF76FF80346194614480CF012FEE9
S3150800AF9003461A460E4B1B8813449AB20C4B1A806A
S3150800AFA07B685B6A1846FEF75DF803461A46114940
S3150800AFB00C4862F043F9064B1988064B1B789AB27F
S3150800AFC0084B06480CF0EDFC00BF1837BD46B0BD6F
S3150800AFD0DC110020DE110020FC0D0708B48C0120CE
S3150800AFE0000E0708E0110020DA110020080E0708F5
S3150800AFF0F41100200C0E070890B585B000AF7860F4
S3150800B00039603B681B780B3B202B00F2F48101A2C8
S3150800B01052F823F099B0000833B20008F7B30008D5
S3150800B020A9B20008F7B30008F7B300081BB3000875
S3150800B030F7B3000889B30008F7B30008F7B30008A8
S3150800B040F7B30008F7B30008F7B30008F7B300082A
S3150800B050F7B30008F7B30008F7B30008F7B300081A
S3150800B060F7B30008F7B30008F7B30008F7B300080A
S3150800B070F7B30008F7B30008F7B30008F7B30008FA
S3150800B080F7B30008F7B30008F7B30008F7B30008EA
S3150800B090F7B300080DB200087B6803F1E4027B6889
S3150800B0A093F838301946104600F014FA02467B68C1
S3150800B0B093F9493013707B6893F838301C467B68DF
S3150800B0C05B6A1846FDF7C2FF0346013B9C4234BF44
S3150800B0D001230023DBB2002B38D07B6893F8383085
S3150800B0E00133DAB27B6883F838207B6893F84830F6
S3150800B0F0002B11D07B685B6A1846FDF7B3FF024642
S3150800B1007B6893F8383013441A787B6893F848308C
S3150800B1109A4201D1012300E00023002B00F06D8143
S3150800B1207B6803F1E4027B6893F8383019461046C9
S3150800B13000F0D0F9034625221A707B6893F8383058
S3150800B1400133DAB27B6883F8382056E10023FB60C6
S3150800B1507B6893F828301A46FB68934247DA7B687F
S3150800B160E433FA681146184600F0B4F9034693F931
S3150800B1700030252B0CBF01230023DBB2002B19D08E
S3150800B1807B68E433FA681146184600F0A3F90346CB
S3150800B19093F900307A6812339B0013445C687B6825
S3150800B1A02C33FA6811461846FEF732FA0346227817
S3150800B1B01A7018E07B68E433FA681146184600F0FE
S3150800B1C089F9034693F900307A6812339B001344D1
S3150800B1D05C687B682C33FA6811461846FEF718FA3D
S3150800B1E0034622781A70FB680133FB60B0E77B6878
S3150800B1F05A6A7B682C3319461046FEF743F97B6872
S3150800B20001225A717B6801221A71F6E07B6893F86D
S3150800B2103830002B08D07B6893F83830013BDAB217
S3150800B2207B6883F83820F1E07B685A797B681A7165
S3150800B230ECE07B6893F94930DBB20133DBB25AB2F2
S3150800B2407B6883F849207B6893F8F030002B0AD195
S3150800B2507B6893F94930232B40F3D1807B68002221
S3150800B26083F84920CBE07B6893F8F030012B0AD1AC
S3150800B2707B6893F94930192B40F3C1807B6800221B
S3150800B28083F84920BBE07B6893F8F030022B40F046
S3150800B290B6807B6893F94930232B40F3B0807B68EE
S3150800B2A01A2283F84920AAE07B6893F94930DBB271
S3150800B2B0013BDBB25AB27B6883F849207B6893F876
S3150800B2C0F030002B0AD17B6893F94930002B80F2C5
S3150800B2D098807B68232283F8492092E07B6893F85C
S3150800B2E0F030012B0AD17B6893F94930002B80F2A4
S3150800B2F088807B68192283F8492082E07B6893F866
S3150800B300F030022B7DD17B6893F94930192B78DC14
S3150800B3107B68232283F8492073E07B6893F94930D8
S3150800B320DBB20133DBB25AB27B6883F849207B680B
S3150800B33093F8F030002B09D17B6893F94930232B19
S3150800B34061DD7B68002283F849205CE07B6893F81E
S3150800B350F030012B09D17B6893F94930192B52DD5E
S3150800B3607B68002283F849204DE07B6893F8F0302B
S3150800B370022B48D17B6893F94930232B43DD7B6840
S3150800B3801A2283F849203EE07B6893F94930DBB2FC
S3150800B390013BDBB25AB27B6883F849207B6893F895
S3150800B3A0F030002B09D17B6893F94930002B2CDA51
S3150800B3B07B68232283F8492027E07B6893F8F030DE
S3150800B3C0012B09D17B6893F94930002B1DDA7B687C
S3150800B3D0192283F8492018E07B6893F8F030022B8D
S3150800B3E013D17B6893F94930192B0EDC7B6823222D
S3150800B3F083F8492009E000BF08E000BF06E000BF67
S3150800B40004E000BF02E000BF00E000BF00BF143741
S3150800B410BD4690BD80B582B000AF7860786800F010
S3150800B42068F87B68184600F070F87B681846083795
S3150800B430BD4680BD80B582B000AF7860786800F000
S3150800B44078F87B6818460837BD4680BD80B582B057
S3150800B45000AF78607B6819687B689A687B681B68A8
S3150800B460D31A1A46786800F06FF87B681846FFF713
S3150800B470C6FA7B6818460837BD4680BDB0B582B0A7
S3150800B48000AF78607B681C687B685D687B681846D7
S3150800B49000F06DF803461A462946204600F072F871
S3150800B4A07B681846FFF7D2FF7B6818460837BD4603
S3150800B4B0B0BD80B582B000AF78603960386800F0FA
S3150800B4C06FF803461946786800F075F800BF083724
S3150800B4D0BD4680BD80B483B000AF786039607B68B4
S3150800B4E01A683B68134418460C37BD465DF8047B5A
S3150800B4F0704780B582B000AF7860786800F089F848
S3150800B5007B6818460837BD4680BD80B483B000AF57
S3150800B51078607B6800221A607B6800225A607B6824
S3150800B52000229A607B6818460C37BD465DF8047B96
S3150800B530704780B483B000AF78607B6818460C37D4
S3150800B540BD465DF8047B704780B584B000AFF860EF
S3150800B550B9607A60BB68002B05D0FB687A68B96861
S3150800B560184600F061F800BF1037BD4680BD80B4AC
S3150800B57083B000AF78607B6818460C37BD465DF827
S3150800B580047B704780B584B000AFF860B9607A6014
S3150800B590B968F86800F057F800BF1037BD4680BD97
S3150800B5A080B483B000AF78607B6818460C37BD4618
S3150800B5B05DF8047B7047B0B582B000AF786039603B
S3150800B5C07B685A687B689B689A4211D07C687B685E
S3150800B5D05D68386800F044F803461A46294620464E
S3150800B5E000F049F87B685B685A1C7B685A600CE077
S3150800B5F0786800F053F80446386800F031F80346D6
S3150800B6001A462146786800F071F800BF0837BD462B
S3150800B610B0BD80B483B000AF78607B6818460C373D
S3150800B620BD465DF8047B704780B584B000AFF8600E
S3150800B630B9607A607A68B968F86800F00FF900BFEF
S3150800B6401037BD4680BD80B582B000AF78603960DE
S3150800B6503968786800F00FF900BF0837BD4680BD25
S3150800B66080B483B000AF78607B6818460C37BD4657
S3150800B6705DF8047B704780B584B000AFF860B960A8
S3150800B6807A607868FFF7ECFF03461A46B968F868E7
S3150800B69000F0FCF800BF1037BD4680BD80B584B009
S3150800B6A000AF78607B681A1D07F10C03114618462F
S3150800B6B000F004F9FB6818461037BD4680BD80B512
S3150800B6C082B000AF184600F005F80346184608375A
S3150800B6D0BD4680BD80B483B000AF387101231846DB
S3150800B6E00C37BD465DF8047B70470000B0B58CB0DA
S3150800B6F000AFF860B9607A60574A0121F86800F02F
S3150800B700EDF8B862FB681B687B62FB685B683B62A6
S3150800B710F86800F02AF903467B6107F1140207F17D
S3150800B72008031146184600F030F90346FB61FB682A
S3150800B730B96A184600F03DF9B861BB69FB62FC6856
S3150800B740BA69FB69D5187868FFF78AFF03461A466F
S3150800B75029462046FFF78FFF0023FB62FFF7AFFF5E
S3150800B7600346002B27D007F10803184600F049F9CD
S3150800B77003461C68FB681846FFF7F9FE0346BA69D4
S3150800B7802146786A00F029F9F862FB6A0133FB6200
S3150800B79007F10803184600F034F903461C68FB68ED
S3150800B7A01846FFF7E4FE0346FA6A396A204600F0AF
S3150800B7B014F9F86226E007F10803184600F021F9A3
S3150800B7C003461C68FB681846FFF7D1FE0346BA69AC
S3150800B7D02146786A00F020F9F862FB6A0133FB62B9
S3150800B7E007F10803184600F00CF903461C68FB68C5
S3150800B7F01846FFF7BCFE0346FA6A396A204600F087
S3150800B8000BF9F862FFF75BFF034683F00103DBB22F
S3150800B810002B09D0FB681846FFF7A9FE03461A460F
S3150800B820396A786AFFF7AEFEF868FB689A687B6A39
S3150800B830D31A1A46796AFFF787FEFB68BA691A604F
S3150800B840FB68FA6A5A60BA69BB6A1A44FB689A6066
S3150800B85000BF3037BD46B0BD100E070880B584B0AE
S3150800B86000AFF860B9607A60B8685FF03DFD00BF68
S3150800B8701037BD4680BD80B483B000AF78603960AC
S3150800B88000BF0C37BD465DF8047B704790B585B0A0
S3150800B89000AFF860B9607A607868FFF7E1FE0346A2
S3150800B8A093F90040BB6819460120FFF79CF8034648
S3150800B8B022461A7000BF1437BD4690BD80B483B0C7
S3150800B8C000AF786039603B681A687B681A607B68E5
S3150800B8D018460C37BD465DF8047B704790B587B0AF
S3150800B8E000AFF860B9607A60F86800F0AEF8044610
S3150800B8F0F86800F0BBF80346E21ABB689A4234BF00
S3150800B90001230023DBB2002B02D078685FF007FD25
S3150800B910F86800F0ABF80446F86800F0A7F80346A4
S3150800B9203B6107F1080207F110031146184600F0BB
S3150800B930ACF803461B6823447B61F86800F096F868
S3150800B94002467B69934206D3F86800F07EF8024601
S3150800B9507B69934204D9F86800F077F8034600E05B
S3150800B9607B6918461C37BD4690BD80B584B000AFCC
S3150800B97078607A6807F10C0311461846FFF79EFFB0
S3150800B980FB6818461037BD4680BD90B583B000AF3A
S3150800B99078603960786800F034F803461C683868BF
S3150800B9A000F02FF803461B68E31A18460C37BD4605
S3150800B9B090BD80B582B000AF786039603B68002BD7
S3150800B9C006D07B683968184600F073F8034600E02D
S3150800B9D0002318460837BD4680BD90B589B002AF2A
S3150800B9E0F860B9607A603B608DF800403B687A6819
S3150800B9F0B968F86800F06CF8034618461C37BD4667
S3150800BA0090BD80B483B000AF78607B6818460C3769
S3150800BA10BD465DF8047B704790B585B000AFF86009
S3150800BA20B9607A603B60F86800F064F80446B86864
S3150800BA3000F060F801463B687A68204600F069F82D
S3150800BA40034618461437BD4690BD80B582B000AF90
S3150800BA5078607B68184600F087F80346184600F0B9
S3150800BA6069F8034618460837BD4680BD80B483B0DA
S3150800BA7000AF78607B685A687B681B68D31A1846DB
S3150800BA800C37BD465DF8047B704780B483B000AFC1
S3150800BA90786039607B681A683B681B689A4201D2ED
S3150800BAA03B6800E07B6818460C37BD465DF8047BAA
S3150800BAB0704780B582B000AF786039600022396877
S3150800BAC0786800F05CF8034618460837BD4680BD1E
S3150800BAD080B584B000AFF860B9607A603B603B68B7
S3150800BAE07A68B968F86800F066F8034618461037A9
S3150800BAF0BD4680BD80B584B000AF786007F10C0301
S3150800BB007968184600F074F8FB6818461037BD4681
S3150800BB1080BD80B584B000AFF860B9607A603B60DC
S3150800BB207A68B968F86800F072F80346184610375C
S3150800BB30BD4680BD80B584B000AF78606FF0004325
S3150800BB40FB60786800F075F80346BB6007F10802E9
S3150800BB5007F10C031146184600F077F803461B68F0
S3150800BB6018461037BD4680BD80B483B000AF7860F4
S3150800BB707B6818460C37BD465DF8047B704780B570
S3150800BB8084B000AFF860B9607A60F86800F071F8C0
S3150800BB900246BB6893428CBF01230023DBB2002B0D
S3150800BBA001D05FF0B9FBB8685FF0A2FB0346184600
S3150800BBB01037BD4680BDB0B584B000AFF860B96037
S3150800BBC07A603B60F86800F060F80446B86800F0F0
S3150800BBD05CF80546786800F058F802463B6829463E
S3150800BBE0204600F05DF8034618461037BD46B0BD3E
S3150800BBF080B483B000AF786039607B683A681A60B1
S3150800BC007B6818460C37BD465DF8047B704780B5DF
S3150800BC1086B000AFF860B9607A600123FB757A6870
S3150800BC20B968F86800F057F8034618461837BD464D
S3150800BC3080BD80B582B000AF7860786800F019F8EA
S3150800BC40034618460837BD4680BD80B483B000AFAA
S3150800BC50786039603B681A687B681B689A4201D22B
S3150800BC603B6800E07B6818460C37BD465DF8047BE8
S3150800BC70704780B483B000AF78606FF00043184611
S3150800BC800C37BD465DF8047B704780B483B000AFBF
S3150800BC9078607B6818460C37BD465DF8047B7047AC
S3150800BCA080B586B000AFF860B9607A603B60BA6864
S3150800BCB0FB68D31A7B617B69002B05DD7B691A4615
S3150800BCC0F968786860F010FD7B697A68134418464D
S3150800BCD01837BD4680BD80B584B000AFF860B9603E
S3150800BCE07A607A68B968F86800F005F80346184675
S3150800BCF01037BD4680BD90B585B000AFF860B96015
S3150800BD007A60F86800F00FF80446B86800F00BF897
S3150800BD1003467A681946204600F016F80346184680
S3150800BD201437BD4690BD80B582B000AF78603B1D24
S3150800BD30184600F02CF80346184600F034F8034677
S3150800BD4018460837BD4680BDB0B584B000AFF86068
S3150800BD50B9607A60F868FFF798FF0446B868FFF795
S3150800BD6094FF05467B681846FFF78FFF03461A4679
S3150800BD702946204600F022F802463B1D1146184681
S3150800BD8000F02EF8034618461037BD46B0BD80B4FD
S3150800BD9083B000AF78607B681B6818460C37BD46D1
S3150800BDA05DF8047B704780B483B000AF78607B6829
S3150800BDB018460C37BD465DF8047B704780B586B0DB
S3150800BDC000AFF860B9607A600123FB757A68B968D4
S3150800BDD0F86800F011F8034618461837BD4680BDC6
S3150800BDE080B483B000AF786039603B6818460C377A
S3150800BDF0BD465DF8047B704780B586B000AFF86035
S3150800BE00B9607A60BA68FB68D31A7B617B69002BD4
S3150800BE1005D07B691A46F968786860F065FC7B6925
S3150800BE207A68134418461837BD4680BD80B584B075
S3150800BE3000AFF8607A603B600B46FB721B4AFB68F2
S3150800BE401A60FB6802221A71FB6802225A71FB68A3
S3150800BE5000229A71FB680522DA71FB68002283F8D2
S3150800BE602020FB68082283F82120FB68002283F83B
S3150800BE702220FB7A0F2B02D8FB7A002B01D1002354
S3150800BE80FB72FB68FA7A83F82020FB680833796826
S3150800BE90184661F043FAFB683A68DA61FB683A7E4D
S3150800BEA01A71FB6818461037BD4680BDC0400708A2
S3150800BEB080B582B000AF7860074A7B681A607B68F5
S3150800BEC00833002B03D0012118465FF00FFA7B6870
S3150800BED018460837BD4680BDC040070880B582B001
S3150800BEE000AF78600B46FB707B689B79012B11D0FD
S3150800BEF07B681B79032B0DD0FB781946786800F010
S3150800BF000EF87B68DB69002B04D07B68DB69FA785E
S3150800BF1010469847002318460837BD4680BD80B4AA
S3150800BF2083B000AF78600B46FB707B681B79FA78A4
S3150800BF309A4203D07B681A797B685A717B68FA78CB
S3150800BF401A7100BF0C37BD465DF8047B704780B494
S3150800BF5083B000AF78607B685A797B681A7100BF36
S3150800BF600C37BD465DF8047B704780B483B000AFDC
S3150800BF7078607B681B7918460C37BD465DF8047BEC
S3150800BF80704780B483B000AF78607B689B791846A9
S3150800BF900C37BD465DF8047B704780B483B000AFAC
S3150800BFA078607B6800229A7100BF0C37BD465DF841
S3150800BFB0047B704780B483B000AF78600B46FB7093
S3150800BFC07B68FA789A7100BF0C37BD465DF8047B2A
S3150800BFD0704780B483B000AF78607B68DB79184619
S3150800BFE00C37BD465DF8047B7047000080B582B00B
S3150800BFF000AF78607B6893F82130082B04D1234979
S3150800C00023480BF0FAFD08E07B6893F82130062BED
S3150800C01003D120491E480BF0F0FD1D480BF06FFDBB
S3150800C0201B480BF0B7FD1A4B93F92930DAB2184BB7
S3150800C03093F92A30DBB2D31ADAB2174B1A707B6837
S3150800C04093F82230002B04D1114B1A88134B1A800F
S3150800C05005E07B6893F822309AB2104B1A807B6809
S3150800C0609B79012B03D07B681B79032B04D1012113
S3150800C07007480CF03AF804E0032105480CF035F8B7
S3150800C08000BF00BF0837BD4680BD00BF1067070860
S3150800C090B48C012028490708F4110020F611002065
S3150800C0A080B483B000AF78600B46FB707B68FA7883
S3150800C0B083F8222000BF0C37BD465DF8047B704725
S3150800C0C080B483B000AF78607B68083318460C37B5
S3150800C0D0BD465DF8047B704780B582B000AF7860D6
S3150800C0E039607B6808333968184661F017F900BF6C
S3150800C0F00837BD4680BD000080B483B000AF7860C5
S3150800C1000B46FB70FB78013B0E2B00F2E58001A283
S3150800C11052F823F051C100086DC1000885C1000816
S3150800C120A7C10008C7C10008E3C1000809C2000882
S3150800C1302DC200084DC2000877C2000897C2000841
S3150800C140B3C20008D9C20008D9C20008D9C200087B
S3150800C150654B1A78654B1A70654B1B885B089AB253
S3150800C160644B1A80644B00221A80B6E05E4B1A783C
S3150800C1705E4B1A705E4B1A885E4B1A805E4B002225
S3150800C1801A80AAE0584B1A78584B1A70584B1B88D5
S3150800C1905B089AB2574B1A80554B1B885B089AB2B4
S3150800C1A0554B1A8099E0504B1B785B00DAB24F4B1F
S3150800C1B01A704F4B1B885B089AB24E4B1A804E4B2F
S3150800C1C000221A8089E0484B1B785B00DAB2474B9D
S3150800C1D01A70474B1A88474B1A80474B00221A8019
S3150800C1E07BE0414B1B785B00DAB2404B1A70404B40
S3150800C1F01B885B089AB23F4B1A803D4B1B885B082D
S3150800C2009AB23D4B1A8068E0374B1B781A465200A3
S3150800C2101344DAB2354B1A70354B1B885B089AB251
S3150800C220344B1A80344B00221A8056E02E4B1B786A
S3150800C2301A4652001344DAB22C4B1A702C4B1A8841
S3150800C2402C4B1A802C4B00221A8046E0264B1B7872
S3150800C2501A4652001344DAB2244B1A70244B1B8830
S3150800C2605B089AB2234B1A80214B1B885B089AB24B
S3150800C270214B1A8031E01C4B1B789B00DAB21B4B12
S3150800C2801A701B4B1B885B089AB21A4B1A801A4BFA
S3150800C29000221A8021E0144B1B789B00DAB2134B5C
S3150800C2A01A70134B1A88134B1A80134B00221A80E4
S3150800C2B013E00D4B1B789B00DAB20C4B1A700C4B33
S3150800C2C01B885B089AB20B4B1A80094B1B885B08C4
S3150800C2D09AB2094B1A8000E000BF00BF0C37BD4672
S3150800C2E05DF8047B704700BFF4110020DE110020C2
S3150800C2F0F6110020DA110020DC11002080B586B086
S3150800C30002AFF8607A603B600B46FB72F868F97A10
S3150800C310022300937B6A7A68FFF788FD154AFB6853
S3150800C3201A60FB68002283F82820FB680022DA627C
S3150800C330FB68002283F83020FB68002283F831204E
S3150800C340FB6897F8202083F83820FB680322DA7107
S3150800C3503B68002B06D0FB683A685A62FB683A7E4F
S3150800C36083F82820FB68FA695A63FB681846103771
S3150800C370BD4680BDF840070880B582B000AF78603A
S3150800C380134A7B681A60786800F0D2FB7B685B6B9F
S3150800C390002B03D0012118465EF0A8FF7B68DB6AF4
S3150800C3A0002B03D0012118465EF0A0FF7B680833F6
S3150800C3B0002B03D0012118465EF098FF7B681846CB
S3150800C3C0FFF776FD7B6818460837BD4680BD00BF77
S3150800C3D0F840070880B582B000AF78607868FFF744
S3150800C3E0CBFF3C2178685EF081FF7B6818460837EA
S3150800C3F0BD4680BD80B586B002AFF8607A601A4641
S3150800C4000B46FB721346BB72F868F97ABB7A00933F
S3150800C410BB697A68FFF70AFD164AFB681A60FB686B
S3150800C420002283F82820FB680022DA62FB680022D3
S3150800C43083F83020FB68002283F83120FB6897F8E0
S3150800C440282083F83820FB680322DA713B6A002B20
S3150800C45007D0FB683A6A5A62FB6897F8242083F883
S3150800C4602820FB68FA695A63FB6818461037BD46E8
S3150800C47080BD00BFF840070880B586B000AF786079
S3150800C48039603B681B782B2B19D02B2B00F3A38024
S3150800C4900E2B19D00E2B00F39E800B2B02D00C2BE3
S3150800C4A055D098E07B681B680C331B6878689847FA
S3150800C4B07B6801225A717B6801221A7190E07B68B9
S3150800C4C05A797B681A718BE07B6893F93130DBB255
S3150800C4D00133DBB25AB27B6883F831200123FB753E
S3150800C4E0FB7D002B25D00023FB7500233B617B6871
S3150800C4F093F830301A463B699342F1DA7B6893F930
S3150800C500313019467B68DA6A3B6913441B789942CD
S3150800C5100BD17B6893F93130DBB20133DBB25AB207
S3150800C5207B6883F831200123FB753B6901333B6146
S3150800C530DDE77B6893F828301A467B6893F9313033
S3150800C5409A424ADC7B68002283F8312045E07B6802
S3150800C55093F93130DBB2013BDBB25AB27B6883F820
S3150800C56031200123FB73FB7B002B25D00023FB73B3
S3150800C5700023BB607B6893F830301A46BB68934249
S3150800C580F1DA7B6893F9313019467B68DA6ABB6859
S3150800C59013441B7899420BD17B6893F93130DBB28F
S3150800C5A0013BDBB25AB27B6883F831200123FB7367
S3150800C5B0BB680133BB60DDE77B6893F93130002B3C
S3150800C5C00DDA7B6893F82830013BDBB25AB27B68F8
S3150800C5D083F8312003E000BF02E000BF00E000BF9F
S3150800C5E000BF1837BD4680BD80B582B000AF786001
S3150800C5F00B46FB707B68FA7811461846FFF76EFC07
S3150800C6007B6893F83830022B22D17B6893F9313056
S3150800C610DBB20133DBB25AB27B6883F831207B6820
S3150800C62093F828301A467B6893F931309A4203DC2E
S3150800C6307B68002283F831207B681B680C331B68F3
S3150800C640786898477B6801225A717B6801221A71BB
S3150800C650002318460837BD4680BD80B483B000AFB6
S3150800C66078607B685B6B002B06D07B6893F931207A
S3150800C6707B685B6BD2B21A70002318460C37BD462E
S3150800C6805DF8047B7047000090B585B000AF786010
S3150800C6900B46FB707B681846FFF7A8FC7B6893F887
S3150800C6A03830012B40F099807A687B6893F82030FF
S3150800C6B019461046FFF720FDFB78002B08D0A14B42
S3150800C6C01988A14B1B789AB2A04BA1480BF069F9BF
S3150800C6D07B681B79002B57D10023FB600023FB6086
S3150800C6E0FB68032B48DC7A68FB680133DBB2194622
S3150800C6F049000B44DBB219461046FFF7FDFC7B6880
S3150800C70093F93130002B00DA03339B105BB29B00A0
S3150800C710FA681344BB607B6893F931301A46BB68E4
S3150800C72093420FD18B4B1C888B4989480BF042FAF0
S3150800C7300346E31A99B2844B1B789AB2864B84480F
S3150800C7400BF02FF97B6893F828301A46BB6893429A
S3150800C7500EDA7C4B19887C4B1B7898B27B685A6A30
S3150800C760BB689B0013441B68024679480BF019F90D
S3150800C770FB680133FB60B3E77B6808331A467749E1
S3150800C780774860F05BFD06E07B6808331A46754912
S3150800C790734860F053FD7A687B6893F82030194631
S3150800C7A01046FFF7A9FC704B1B881C466C49684865
S3150800C7B00BF000FA0346E31A9AB2624B1B8813443D
S3150800C7C09AB2604B1A805F4B19885F4B1B789AB2F6
S3150800C7D0634B5F480BF0E5F880E17B6893F83830E7
S3150800C7E0002B40F0C7807A687B6893F8203019469A
S3150800C7F01046FFF781FCFB78002B08D0514B1988AF
S3150800C800514B1B789AB2514B51480BF0CAF87B68CA
S3150800C8101B79002B3AD17A687B6893F8203002336B
S3150800C820DBB219461046FFF767FC7B6893F8283099
S3150800C830002B0DD14D494A4860F000FD414B19883F
S3150800C840414B1B789AB2464B41480BF0AAF815E0C3
S3150800C8507B685A6A7B6893F931309B0013441B68DE
S3150800C8601A4643493E4860F0E9FC364B1988364B70
S3150800C8701B789AB23A4B36480BF093F87B68083324
S3150800C8801A463649364860F0D9FC39E07A687B683A
S3150800C89093F820300233DBB219461046FFF72CFC1A
S3150800C8A07B6893F82830002B0DD130492C4860F06E
S3150800C8B0C5FC244B1988244B1B789AB2284B24486C
S3150800C8C00BF06FF815E07B685A6A7B685B6B1B7820
S3150800C8D09B0013441B681A462549214860F0AEFCA4
S3150800C8E0184B1988184B1B789AB21D4B18480BF031
S3150800C8F058F87B6808331A461849194860F09EFCB0
S3150800C9007A687B6893F8203019461046FFF7F4FBDF
S3150800C910154B1B881C4612490D480BF04BF903466C
S3150800C920E31A9AB2074B1B8813449AB2054B1A802E
S3150800C930044B1988044B1B789AB2094B04480BF030
S3150800C94030F8CBE0DC110020DE1100202C0E0708A1
S3150800C950B48C0120F6110020300E0708340E0708A3
S3150800C960E0110020380E0708DA1100203C0E0708EF
S3150800C970480E07087B6893F83830022B40F0AE80E3
S3150800C9807A687B6893F8203019461046FFF7B4FB9F
S3150800C990FB78002B08D0534B1988534B1B789AB257
S3150800C9A0524B53480AF0FDFF7B681B79002B3AD19E
S3150800C9B07A687B6893F820300233DBB21946104652
S3150800C9C0FFF79AFB7B6893F82830002B0DD149496D
S3150800C9D0494860F033FC434B1988434B1B789AB29D
S3150800C9E0454B43480AF0DDFF15E07B685A6A7B68C9
S3150800C9F093F931309B0013441B681A463F493E4859
S3150800CA0060F01CFC374B1988374B1B789AB23A4BA7
S3150800CA1037480AF0C6FF7B6808331A46384936484D
S3150800CA2060F00CFC39E07A687B6893F820300233B2
S3150800CA30DBB219461046FFF75FFB7B6893F8283090
S3150800CA40002B0DD12B492C4860F0F8FB254B198893
S3150800CA50254B1B789AB2284B25480AF0A2FF15E009
S3150800CA607B685A6A7B685B6B1B789B0013441B6860
S3150800CA701A462249204860F0E1FB1A4B19881A4BDE
S3150800CA801B789AB21C4B1A480AF08BFF7B6808334E
S3150800CA901A461B49184860F0D1FB7A687B6893F8F8
S3150800CAA0203019461046FFF727FB164B1B881C46F5
S3150800CAB011490F480BF07EF80346E31A9AB2094B60
S3150800CAC01B8813449AB2074B1A80064B1988064BE3
S3150800CAD01B789AB2084B06480AF063FF00BF143762
S3150800CAE0BD4690BDDC110020DE1100202C0E070883
S3150800CAF0B48C01203C0E0708E0110020480E0708F8
S3150800CB00340E0708DA11002080B485B000AFF8604B
S3150800CB10B9601346FB71FB68BA685A62FB68FA7912
S3150800CB2083F8282000BF1437BD465DF8047B70479C
S3150800CB3080B584B000AF78607B685B6A002B1ED036
S3150800CB400023FB607B6893F828301A46FB689342FB
S3150800CB5015DA7B685A6AFB689B0013441B68002B2E
S3150800CB6009D07B685A6AFB689B0013441B6801213D
S3150800CB7018465EF0BBFBFB680133FB60E2E700BFCB
S3150800CB801037BD4680BD80B483B000AF78607B683F
S3150800CB905A6A7B6893F931309B0013441B68184620
S3150800CBA00C37BD465DF8047B704780B483B000AF90
S3150800CBB078607B6893F8383018460C37BD465DF8C0
S3150800CBC0047B704780B483B000AF7860064A7B6800
S3150800CBD01A607B680022DA607B6818460C37BD4607
S3150800CBE05DF8047B704700BFA041070880B586B092
S3150800CBF002AFF8607A603B600B46FB72F868F97A18
S3150800CC0002230093FB697A68FFF710F9114AFB685B
S3150800CC101A60FB682C3300221A605A601A81FB6876
S3150800CC20002283F836203B68002B07D03B685A68F9
S3150800CC30FB689A623B681A68FB685A62FB68BA69BD
S3150800CC409A63FB680222DA71FB6818461037BD46FC
S3150800CC5080BD00BF3041070880B582B000AF78605C
S3150800CC60054A7B681A607B681846FFF721F97B68D6
S3150800CC7018460837BD4680BD3041070880B582B0E2
S3150800CC8000AF78607868FFF7E7FF3C2178685EF0C8
S3150800CC902DFB7B6818460837BD4680BD80B483B037
S3150800CCA000AF7860396000BF0C37BD465DF8047B7D
S3150800CCB0704780B582B000AF78600B46FB707B6822
S3150800CCC0FA7811461846FFF709F97B689B6B1846F0
S3150800CCD00837BD4680BD80B483B000AF786000BF1A
S3150800CCE018460C37BD465DF8047B704790B583B08F
S3150800CCF000AF78600B46FB707B681846FFF776F93D
S3150800CD007A687B6893F82030013BDBB219461046F7
S3150800CD10FFF7F2F9FB78002B08D02C4B19882C4B1F
S3150800CD201B789AB22B4B2C480AF03BFE7B680833DB
S3150800CD301A462A492A4860F081FA2A4B1B881C465B
S3150800CD40274925480AF036FF0346E31A9AB21F4BCD
S3150800CD501B8813449AB21D4B1A801C4B19881C4B0E
S3150800CD601B789AB21E4B1C480AF01BFE7B681B797F
S3150800CD70022B07D17B685B6A1A461B49184860F084
S3150800CD805DFA0CE07B681B79012B08D17B6803F1FF
S3150800CD902C027B689B6A1549114860F04FFA7A683D
S3150800CDA07B6893F820300133DBB219461046FFF74B
S3150800CDB0A3F9064B1988064B1B789AB2084B064806
S3150800CDC00AF0EFFD00BF0C37BD4690BDDC11002010
S3150800CDD0DE1100204C0E0708B48C0120500E0708FF
S3150800CDE0E0110020DA110020580E07085C0E07082B
S3150800CDF080B483B000AF78607B6893F83630184605
S3150800CE000C37BD465DF8047B704780B582B000AF2D
S3150800CE10786039607B682C333968184660F07EFA8A
S3150800CE2000BF0837BD4680BD80B483B000AF7860C8
S3150800CE3039607B683A685A6200BF0C37BD465DF8B0
S3150800CE40047B704780B584B000AFF8607A601A46F4
S3150800CE500B46FB721346BB72FB6800221A70FB680E
S3150800CE6008225A70FB68043312491846FCF7E9F998
S3150800CE70FB6810330F491846FCF7E3F9FB680022F4
S3150800CE805A84FB68002283F82420FB6804337968F7
S3150800CE901846FCF729FBFB68FA7A1A77FB68BA7A10
S3150800CEA09A77FB683A7E5A77FB6818461037BD466C
S3150800CEB080BD00BF640E070880B582B000AF7860F9
S3150800CEC07B6810331846FCF7F7F97B680433184675
S3150800CED0FCF7F2F97B6818460837BD4680BD80B472
S3150800CEE083B000AF78607B689B7F18460C37BD46D9
S3150800CEF05DF8047B7047000090B591B000AF78608C
S3150800CF007B681B78012B4FD0786800F09BF878680F
S3150800CF1000F0E2F87B6804331846FCF7A3F80446E9
S3150800CF207B6810331846FCF79DF8034607F10C009A
S3150800CF3022461F4960F082F97B681B7F002B16D0BA
S3150800CF407B681B8C1C4607F10C03194619480AF026
S3150800CF5031FE0346E31ADA0F13445B1019467B6861
S3150800CF605A8C8BB213449AB27B685A8411E07B6858
S3150800CF701B8C1C4607F10C0319460E480AF01AFECC
S3150800CF800346E11A7B685A8C8BB213449AB27B68C3
S3150800CF905A847B68598C7B6893F824309AB207F1D7
S3150800CFA00C0304480AF0FDFC00BF4437BD4690BD9B
S3150800CFB0680E0708B48C012080B582B000AF78608F
S3150800CFC039607B68103339681846FCF75BFA00BF8E
S3150800CFD00837BD4680BD80B582B000AF786039603D
S3150800CFE07B68043339681846FCF74CFA00BF0837E3
S3150800CFF0BD4680BD80B483B000AF78600B46FB7039
S3150800D0007B68FA781A7000BF0C37BD465DF8047B5A
S3150800D010704780B483B000AF78607B681B78184689
S3150800D0200C37BD465DF8047B704780B483B000AF0B
S3150800D03078607B685B7F18460C37BD465DF8047BD5
S3150800D0407047000080B582B000AF78607B685B7877
S3150800D050082B04D1154916480AF0CFFD07E07B686E
S3150800D0605B78062B03D1134911480AF0C6FD104810
S3150800D0700AF045FD0E480AF08DFD0D4B93F929304F
S3150800D080DAB20B4B93F92A30DBB2D31ADAB27B68E1
S3150800D09083F82520064B1A887B68DA84032104481E
S3150800D0A00BF023F800BF0837BD4680BD1067070898
S3150800D0B0B48C01202849070880B483B000AF786093
S3150800D0C00B46FB707B68FA785A7000BF0C37BD4672
S3150800D0D05DF8047B7047000080B483B000AF7860C9
S3150800D0E07B681B7F0F2B00F2108101A252F823F0F8
S3150800D0F031D1000853D1000873D100088FD1000838
S3150800D100B5D10008D9D10008F9D1000823D2000802
S3150800D1104BD200086FD200089DD20008C1D2000881
S3150800D120E1D200080BD300080BD300080BD3000884
S3150800D1307B68002283F824207B68DB8C5B089AB224
S3150800D1407B681A847B68DB8C5B089AB27B685A8496
S3150800D150DCE07B6893F825207B6883F824207B68CD
S3150800D160DB8C5B089AB27B681A847B6800225A8437
S3150800D170CCE07B6893F825207B6883F824207B68BD
S3150800D180DA8C7B681A847B6800225A84BEE07B6846
S3150800D19093F825207B6883F824207B68DB8C5B0862
S3150800D1A09AB27B681A847B68DB8C5B089AB27B68C8
S3150800D1B05A84ABE07B6893F825305B00DAB27B686B
S3150800D1C083F824207B68DB8C5B089AB27B681A8418
S3150800D1D07B6800225A8499E07B6893F825305B00C7
S3150800D1E0DAB27B6883F824207B68DA8C7B681A8439
S3150800D1F07B6800225A8489E07B6893F825305B00B7
S3150800D200DAB27B6883F824207B68DB8C5B089AB2E9
S3150800D2107B681A847B68DB8C5B089AB27B685A84C5
S3150800D22074E07B6893F825301A4652001344DAB244
S3150800D2307B6883F824207B68DB8C5B089AB27B6862
S3150800D2401A847B6800225A8460E07B6893F825304C
S3150800D2501A4652001344DAB27B6883F824207B68A6
S3150800D260DA8C7B681A847B6800225A844EE07B68D5
S3150800D27093F825301A4652001344DAB27B6883F8CD
S3150800D28024207B68DB8C5B089AB27B681A847B68EF
S3150800D290DB8C5B089AB27B685A8437E07B6893F824
S3150800D2A025309B00DAB27B6883F824207B68DB8C08
S3150800D2B05B089AB27B681A847B6800225A8425E048
S3150800D2C07B6893F825309B00DAB27B6883F82420C4
S3150800D2D07B68DA8C7B681A847B6800225A8415E09E
S3150800D2E07B6893F825309B00DAB27B6883F82420A4
S3150800D2F07B68DB8C5B089AB27B681A847B68DB8C5C
S3150800D3005B089AB27B685A8400E000BF00BF0C37FE
S3150800D310BD465DF8047B704780B586B002AFF860FD
S3150800D3207A603B600B46FB72F868F97A0223009331
S3150800D330BB697A68FEF77AFD084AFB681A60FB68DB
S3150800D34000229A62FB683A685A62FB680022DA7120
S3150800D350FB6818461037BD4680BD00BF6841070800
S3150800D36080B582B000AF7860054A7B681A607B6832
S3150800D3701846FEF79DFD7B6818460837BD4680BDF2
S3150800D3806841070880B582B000AF78607868FFF713
S3150800D390E7FF2C2178685DF0A9FF7B6818460837F7
S3150800D3A0BD4680BD90B583B000AF78600B46FB7074
S3150800D3B07B681846FEF71AFE7A687B6893F8203071
S3150800D3C019461046FEF798FEFB78002B08D0164B38
S3150800D3D01988164B1B789AB2154B16480AF0E1FACB
S3150800D3E0154B1B881C467B680833194611480AF0FA
S3150800D3F0E1FB0346E31ADA0F13445B109AB20A4BB1
S3150800D4001B8813449AB2084B1A80074B1988074B96
S3150800D4101B789AB27B68083306480AF0C2FA00BF3E
S3150800D4200C37BD4690BD00BFDC110020DE11002080
S3150800D430700E0708B48C0120DA11002080B483B07E
S3150800D44000AF7860396000BF0C37BD465DF8047BD5
S3150800D450704780B582B000AF78600B46FB707B687A
S3150800D460FA7811461846FEF739FD7B685B6A184656
S3150800D4700837BD4680BD80B483B000AF78607B684E
S3150800D4809B6A18460C37BD465DF8047B704780B426
S3150800D49083B000AF7860002318460C37BD465DF8A8
S3150800D4A0047B704780B582B000AF78603960396810
S3150800D4B07868FCF77DF8034618460837BD4680BDF0
S3150800D4C080B584B000AFF860B9607A60BB689B68C5
S3150800D4D0F8687A68B968FCF7E3F8F8681037BD4663
S3150800D4E080BD80B485B000AFF860B9607A603B60F3
S3150800D4F0FB6800221A70FB680022DA77FB680022B4
S3150800D5005A63FB6800229A63FB680022DA63FB68A9
S3150800D510BA685A61FB683A689A61FB683A7E1A7774
S3150800D520FB687A685A62FB68FA695A60FB6897F87A
S3150800D53020201A72FB687A6ADA60FB6801221A747C
S3150800D540FB6897F828205A74FB6897F82C2083F80C
S3150800D55020203A7E97F82C30B2FBF3F3DAB2FB6858
S3150800D5609A773B7E97F82C20B3FBF2F102FB01F287
S3150800D5709B1ADBB2002B05D0FB689B7F0133DAB21E
S3150800D580FB689A77FB6818461437BD465DF8047B36
S3150800D590704780B483B000AF78607B6818460C3754
S3150800D5A0BD465DF8047B704780B483B000AF7860F1
S3150800D5B039607B683A685A6100BF0C37BD465DF82A
S3150800D5C0047B704780B586B000AF78607B681B78AF
S3150800D5D0052B00F0A980786800F0BAFF00237B616C
S3150800D5E07B68DB7F1A467B6893F8203003FB02F3DF
S3150800D5F07A6892F8202013443B617B681B7F1A46A1
S3150800D6003B69934202DD7B681B7F3B617B68DB7F5E
S3150800D6101A467B6893F8203003FB02F37B617A692C
S3150800D6203B699A422DDA7B6893F91D301A467B6965
S3150800D630934211D17B689A697B699B0013441868E9
S3150800D6407B689A697B699B0013441B681B681033C7
S3150800D6501B680121984710E07B689A697B699B00E3
S3150800D660134418687B689A697B699B0013441B6896
S3150800D6701B6810331B68002198477B6901337B615F
S3150800D680CDE700237B617B681B7A1A467B69934248
S3150800D6902FDA7B685A687B699B0013441B68184617
S3150800D6A0FFF71DFC03461A467B681B789A4210D181
S3150800D6B07B685A687B699B0013441B681846FFF70A
S3150800D6C0B4FC03461A467B68DB7F9A4201D10123E4
S3150800D6D000E00023002B08D07B685A687B699B0012
S3150800D6E013441B681846FFF707FC7B6901337B6107
S3150800D6F0C9E77B681B78002B7DD1414B1B7801332A
S3150800D700DAB23F4B1A703E4B1B78072B73D97B68EE
S3150800D71001221A703A4B00221A707B6801221A7489
S3150800D720786801F01CF966E0354B1B780133DAB2EC
S3150800D730334B1A70324B1B78072B5CD9304B0022BF
S3150800D7401A707B6801221A74786801F008F97868FB
S3150800D75001F005F97B681B78002B19D17B681B6BD8
S3150800D76001211846FEF7DBFB7B68DB6A002B08D035
S3150800D7707B68DA6B7B68DB6A1946104601F0CFF9DD
S3150800D78039E07B68DB6B0021184601F0C8F932E006
S3150800D7907B681B78042B2ED17B6893F820301A46B9
S3150800D7A07B68DB7F03FB02F3FB607B681B7F1A4603
S3150800D7B0FB6893421FDA7B6893F91D301A46FB68AB
S3150800D7C093420AD17B689A69FB689B0013441B68DD
S3150800D7D000211846FEF7A3FB09E07B689A69FB68F7
S3150800D7E09B0013441B6801211846FEF7E3FBFB6800
S3150800D7F00133FB60D9E700BF1837BD4680BD00BFBF
S3150800D800F811002090B589B000AF78607B681B7866
S3150800D810042B40F00C817B689A697B6893F91D306C
S3150800D8209B00134418687B689A697B6893F91D30D6
S3150800D8309B0013441B681B6814331B687A68526A7A
S3150800D840114698477B685B6A1B782B2B32D17B681D
S3150800D8509A697B6893F91D309B0013441B68184628
S3150800D860FEF783FB0346002B14BF01230023DBB21C
S3150800D870002B1AD0786801F072F87B6803221A70B8
S3150800D8800023FB617B681B7F1A46FB6993420CDA0F
S3150800D8907B689A69FB699B0013441B681846FEF768
S3150800D8A07CFBFB690133FB61ECE77B6801221A7498
S3150800D8B000F00EBE7B685B6A1B780B2B40F0B280CB
S3150800D8C07B689A697B6893F91D309B0013441B6833
S3150800D8D01846FEF74AFB0346002B14BF0123002314
S3150800D8E0DBB2002B00F099807B68DB68002B46D002
S3150800D8F07B689A697B6893F91D309B001344186806
S3150800D9007B689A697B6893F91D309B0013441B68F2
S3150800D9101B6808331B6801219847786801F01FF8CF
S3150800D9207B689A697B6893F91D309B0013441B68D2
S3150800D9301846FEF74EFB0346032B0CBF01230023B4
S3150800D940DBB2002B3FD07B6893F820301A467B6801
S3150800D950DB7F03FB02F3BB617B681B7F1A46BB694F
S3150800D960934230DA7B689A69BB699B0013441B684B
S3150800D9701846FEF712FBBB690133BB61ECE77B680F
S3150800D98003221A707B6893F820301A467B68DB7F7F
S3150800D99003FB02F37B617B681B7F1A467B69934214
S3150800D9A00CDA7B689A697B699B0013441B681846E6
S3150800D9B0FEF7CDFA7B6901337B61ECE77B680122D0
S3150800D9C01A7400F085BD7B681B78032B04D17B682D
S3150800D9D001221A7400F07CBD7B681B78052B5CD18C
S3150800D9E07B689B6A0021184600F09EFF7B689C6A4C
S3150800D9F07B68DB6B184601F02EF901467B68DB6B0A
S3150800DA001A46204600F092FD7B68DA6B7B689B6AB3
S3150800DA101946104601F083F83FE07B6801221A7424
S3150800DA2000F056BD7B6801221A7400F051BD7B6870
S3150800DA301B78052B28D17B68DB6A184600F083FF24
S3150800DA400346052B0CBF01230023DBB2002B17D09E
S3150800DA507B6802221A70786800F081FF7B68DA6BAF
S3150800DA607B68DB6A1946104601F059F87B68DB6B60
S3150800DA70184601F099F87B6801221A7400F028BD4F
S3150800DA80786800F06CFF08E07B681B78032B04D0ED
S3150800DA907B6800221A7400F01BBD7B6801221A7489
S3150800DAA07B689B69002B0ED17B685B6A1B780B2B06
S3150800DAB009D07B685B6A1B782B2B04D07B68002215
S3150800DAC01A7400F005BD7B685B6A1B780B3B212B3B
S3150800DAD000F2EB8401A252F823F000BF65DB0008D0
S3150800DAE0EFE000089DE1000829E0000889E3000846
S3150800DAF0ABE40008ABE40008ABE40008ABE40008BC
S3150800DB00ABE40008ABE40008ABE40008ABE40008AB
S3150800DB10ABE40008ABE40008ABE40008ABE400089B
S3150800DB20ABE40008ABE40008ABE40008ABE400088B
S3150800DB30ABE40008ABE40008ABE40008ABE400087B
S3150800DB40ABE40008ABE40008ABE40008ABE400086B
S3150800DB50ABE40008ABE40008ABE4000869DF0008A2
S3150800DB60FFDF00087B689B69002B2ED17B680422A7
S3150800DB701A70786800F0F3FE7B689B6A002B03D165
S3150800DB807B6802221A7020E07B689B6A002118468F
S3150800DB9000F0CAFE7B689C6A7B68DB6B184601F05E
S3150800DBA05AF801467B68DB6B1A46204600F0BEFC35
S3150800DBB07B68DA6B7B689B6A1946104600F0AFFFF4
S3150800DBC07B6801221A7400F083BC7B681B78022BE1
S3150800DBD052D1786800F0C3FE7B6800221A707B6811
S3150800DBE01B6B01211846FEF79AF97B68DB6A002B46
S3150800DBF009D07B68DB6A184600F0A5FE0346052BAC
S3150800DC0001D0012300E00023002B09D07B68DA6BE2
S3150800DC107B68DB6A1946104600F081FF00F049BCB4
S3150800DC207B68DB6A002B0DD07B68DB6A184600F040
S3150800DC308AFE0346052B05D17B689B6A002B01D11A
S3150800DC40012300E00023002B0ED07B68DA6B7B688B
S3150800DC50DB6A1946104600F062FF7B68DB6B1846E4
S3150800DC6000F0A2FF00F025BC7B68DB6B002118469C
S3150800DC7000F055FF00F01DBC7B689A697B6893F934
S3150800DC801D309B0013441B681846FEF77AF90346B5
S3150800DC90FB737B689A697B6893F91D309B00134474
S3150800DCA01B681846FEF761F90346BB73FB7B012B1D
S3150800DCB000F0FF83BB7B032B00F0FB837B689A692C
S3150800DCC07B6893F91D309B0013441B681846FEF7C2
S3150800DCD080F903467B737B689A697B6893F91D30E4
S3150800DCE09B00134418687B689A697B6893F91D3012
S3150800DCF09B0013441B681B6808331B680021984760
S3150800DD00B860BB68002B02D17B7B002B13D17B68E4
S3150800DD10DB6A184600F017FE0346052B14BF0123DD
S3150800DD200023DBB2002B03D07B6800221A7002E0C6
S3150800DD307B6805221A707B7B002B39D1BB68002BC8
S3150800DD401FD07B68BA689A627B689B6A002118466E
S3150800DD5000F0EAFD7B689C6A7B68DB6B184600F07E
S3150800DD607AFF01467B68DB6B1A46204600F0DEFB2D
S3150800DD707B68DA6B7B689B6A1946104600F0CFFE13
S3150800DD8097E37B68DB6A002B08D07B68DA6B7B68D5
S3150800DD90DB6A1946104600F0C2FE8AE37B68D86B38
S3150800DDA07B68596B7B689B6B1A4600F09BFE80E389
S3150800DDB07B7B012B37D1BB68002B2CD07B68BA68DC
S3150800DDC09A627B689B6A0021184600F0ADFD7B6865
S3150800DDD0986A7B689A697B6893F91D309B0013449F
S3150800DDE01B68194600F0CFFD7B689C6A7B68DB6B75
S3150800DDF0184600F030FF01467B68DB6B1A46204662
S3150800DE0000F094FB7B68DA6B7B689B6A19461046C0
S3150800DE1000F085FE4DE3BB68002B40F04A83786826
S3150800DE2000F09DFD45E37B7B022B30D1BB68002BC0
S3150800DE3000F03F837B68BA689A627B689B6A002118
S3150800DE40184600F071FD7B68986A7B689A697B685A
S3150800DE5093F91D309B0013441B68194600F093FD87
S3150800DE607B689C6A7B68DB6B184600F0F4FE01460B
S3150800DE707B68DB6B1A46204600F058FB7B68DA6B3A
S3150800DE807B689B6A1946104600F049FE11E37B7BC6
S3150800DE90032B5CD17B681B78032B40F00A837B68D5
S3150800DEA09A697B6893F91D309B00134419687B684F
S3150800DEB09A697B6893F91D309B0013441B681B689D
S3150800DEC02C331B68084698470346022B14BF0123C8
S3150800DED00023DBB2002B00F0EE82786800F03FFDED
S3150800DEE07B681B78042B02D07B6804221A707B6837
S3150800DEF093F820301A467B68DB7F03FB02F33B610D
S3150800DF007B681B7F1A463B69934280F2D2827B6804
S3150800DF1093F91D301A463B6993420AD17B689A6980
S3150800DF203B699B0013441B6800211846FDF7F7FF61
S3150800DF3009E07B689A693B699B0013441B680121C9
S3150800DF401846FEF737F83B6901333B61D8E77B7B18
S3150800DF50042B40F0AE827B681B78032B40F0A98225
S3150800DF607B6804221A70A4E27B68DB6A002B46D021
S3150800DF707B689B69002B1ED17B6800221A70786823
S3150800DF8000F0EDFC7B681B6B1846FDF7E0FF7B682D
S3150800DF90DB6A002B08D07B68DA6B7B68DB6A19467C
S3150800DFA0104600F0BCFD0EE07B68DB6B00211846CE
S3150800DFB000F0B5FD07E07B681B6B1846FDF7C7FF49
S3150800DFC07B6800221A707B68DB6A184600F0BBFC87
S3150800DFD00346052B0CBF01230023DBB2002B05D01B
S3150800DFE07B68DB6A0021184600F09EFC7B68DA6BCA
S3150800DFF07B68DB6A1946104600F091FD68E27B688B
S3150800E000DB6A002B40F059827B68D86B7B68596BBA
S3150800E0107B689B6B1A4600F065FD7B6800221A70C8
S3150800E020786800F09CFC48E27B6893F91D30DBB207
S3150800E0300133DBB25AB27B685A777B681B7F1A4674
S3150800E0407B6893F91D309A420BDC7B685B7C002B5E
S3150800E05007D17B681B7F013BDBB25AB27B685A77D4
S3150800E06044E07B681B7F1A467B6893F91D309A4209
S3150800E0700FDC7B685B7C002B0BD07B681B7F013B2E
S3150800E080DBB25AB27B685A777B685B6A01221A70E0
S3150800E0902CE07B6893F91D307A6892F8202093FB70
S3150800E0A0F2F102FB01F29B1A002B40F008827B6812
S3150800E0B0DB7F1A467B689B7F013B9A4280F2FF8191
S3150800E0C07B6893F82030042B06D17B68DB7F01330D
S3150800E0D0DAB27B68DA77F2E17B6893F91D30DBB256
S3150800E0E0013BDBB25AB27B685A77E8E1E7E17B6825
S3150800E0F093F91D30DBB2013BDBB25AB27B685A7723
S3150800E1007B6893F91D30002B07DA7B685B7C002B54
S3150800E11003D17B6800225A773FE07B6893F91D306C
S3150800E120002B10DA7B685B7C002B0CD07B68002206
S3150800E1305A777B68D86B7B68596B7B689B6B1A46EA
S3150800E14000F0D0FC29E07B6893F91D3001337A682A
S3150800E15092F8202093FBF2F102FB01F29B1A002BA6
S3150800E16040F0AF817B68DB7F002B00F0AA817B68DB
S3150800E17093F82030042B06D17B68DB7F013BDAB2AB
S3150800E1807B68DA779DE17B6893F91D30DBB2013352
S3150800E190DBB25AB27B685A7793E192E17B6893F8CF
S3150800E1A02030042B5BD97B6893F91D30042B56D19C
S3150800E1B07B6893F91D30DBB2013BDBB25AB27B6850
S3150800E1C05A777B6893F91D30002B07DA7B685B7CEE
S3150800E1D0002B03D17B6800225A773FE07B6893F9CE
S3150800E1E01D30002B10DA7B685B7C002B0CD07B681B
S3150800E1F000225A777B68D86B7B68596B7B689B6B68
S3150800E2001A4600F06FFC29E07B6893F91D3001334C
S3150800E2107A6892F8202093FBF2F102FB01F29B1A2E
S3150800E220002B40F0AF807B68DB7F002B00F0AA80D4
S3150800E2307B6893F82030042B06D17B68DB7F013B93
S3150800E240DAB27B68DA779DE07B6893F91D30DBB23A
S3150800E2500133DBB25AB27B685A7793E092E07B6867
S3150800E260DB7F002B29D07B6893F82030042B00F045
S3150800E2702A817B68DB7F013BDAB27B68DA777B68C9
S3150800E28093F91D30DAB27B6893F82030D31ADBB2E3
S3150800E2905AB27B685A777B6893F91D30002B80F257
S3150800E2A012817B68DA7F7B6893F8203012FB03F3D0
S3150800E2B0DBB25AB27B685A7705E17B68DB7F002BB5
S3150800E2C040F001817B68DB6A002B46D07B689B693E
S3150800E2D0002B1ED17B6800221A70786800F03FFB7D
S3150800E2E07B681B6B1846FDF732FE7B68DB6A002BE2
S3150800E2F008D07B68DA6B7B68DB6A1946104600F043
S3150800E3000EFC0EE07B68DB6B0021184600F007FC6C
S3150800E31007E07B681B6B1846FDF719FE7B68002231
S3150800E3201A707B68DB6A184600F00DFB0346052B5E
S3150800E3300CBF01230023DBB2002B05D07B68DB6A08
S3150800E3400021184600F0F0FA7B68DA6B7B68DB6A16
S3150800E3501946104600F0E3FBBAE07B68DB6A002B3F
S3150800E36040F0B3807B68D86B7B68596B7B689B6B86
S3150800E3701A4600F0B7FB7B6800221A70786800F02E
S3150800E380EEFAA2E000BF9EE07B6893F82030042BEB
S3150800E39056D97B6893F91D30022B51DD7B6893F9BA
S3150800E3A01D30DBB20133DBB25AB27B685A777B6821
S3150800E3B01B7F1A467B6893F91D309A420BDC7B68F3
S3150800E3C05B7C002B07D17B681B7F013BDBB25AB213
S3150800E3D07B685A7733E07B681B7F1A467B6893F91C
S3150800E3E01D309A420FDC7B685B7C002B0BD07B6868
S3150800E3F01B7F013BDBB25AB27B685A777B685B6A44
S3150800E40001221A701BE07B6893F91D307A6892F82E
S3150800E410202093FBF2F102FB01F29B1A002B42D15A
S3150800E4207B68DB7F1A467B689B7F013B9A423ADA18
S3150800E4307B68DB7F0133DAB27B68DA7733E032E078
S3150800E4407B68DB7F1A467B689B7F013B9A423EDAF4
S3150800E4507B6893F82030042B39D07B68DB7F013347
S3150800E460DAB27B68DA777B6893F91D30DAB27B68B3
S3150800E47093F820301344DBB25AB27B685A777B682C
S3150800E4801B7F1A467B6893F91D309A421FDC7B680E
S3150800E490DA7F7B6893F8203012FB03F3DBB25AB2BB
S3150800E4A07B685A7713E000BF11E07B6800221A7474
S3150800E4B00EE000BF0CE000BF0AE000BF08E000BFA6
S3150800E4C006E000BF04E000BF02E000BF00E000BFB6
S3150800E4D02437BD4690BD00BF80B483B000AF7860D6
S3150800E4E039607B683A685A6300BF0C37BD465DF8E9
S3150800E4F0047B704780B483B000AF786039607B686E
S3150800E5003A689A6300BF0C37BD465DF8047B7047CE
S3150800E51080B483B000AF786039607B683A68DA63A4
S3150800E52000BF0C37BD465DF8047B704780B485B0E4
S3150800E53000AFF860B9607A60FB68BA68DA62FB68AF
S3150800E5407A68DA6300BF1437BD465DF8047B704706
S3150800E55090B59DB000AF7860B949BA4809F04DFB4F
S3150800E560B84809F017FB0321B64809F0BEFD7B68D9
S3150800E57093F82030042B1FD17B68DB7F002B0CD04F
S3150800E580B149B04809F016FB0346C3F1F90399B23D
S3150800E590AD4B0522AB4809F004FA7B68DB7F1A46C7
S3150800E5A07B689B7F013B9A423AD0A84B0522F9210A
S3150800E5B0A44809F0F6F933E0A24B1B8887F86F30B8
S3150800E5C0A349A04809F0F6FA0346DBB297F86F208C
S3150800E5D0D31A87F86F307B68DB7F1A467B689B7F88
S3150800E5E0013B9A4207D097F86F3099B2984B0322AD
S3150800E5F0944809F0D6F99749924809F0DBFA034698
S3150800E600DBB297F86F20D31A87F86F3097F86F3018
S3150800E6109BB2013B99B28F4B03228A4809F0C1F994
S3150800E6208D49884809F0E9FA864809F068FA854864
S3150800E63009F0B0FA0321834809F057FD7B685A6947
S3150800E64007F1180311461846FAF7FBFD07F10C0304
S3150800E65082491846FAF7F5FD07F118038049184666
S3150800E660FEF720FF0346002B14BF01230023DBB26D
S3150800E670002B00F04281002387F86E3007F1240052
S3150800E68007F1180108230022FBF70AF807F124020C
S3150800E69007F10C0311461846FAF714FF07F124038D
S3150800E6A01846FAF709FE07F10C031846FAF7DAFCDA
S3150800E6B0034600220021634809F073F907F10C03A9
S3150800E6C01846FAF7CFFC034619465E4809F072FA6F
S3150800E6D00346DAB297F86E30134487F86E3007F1BE
S3150800E6E0300007F118010C230822FAF7D9FF07F1C1
S3150800E6F0300207F10C0311461846FAF7E3FE07F154
S3150800E70030031846FAF7D8FD7B68DB7F002B04D167
S3150800E71003214C4809F0E9FC03E00121494809F0C6
S3150800E720E4FC97F86E309CB207F10C031846FAF72A
S3150800E73099FC034600222146424809F032F907F1BE
S3150800E7400C031846FAF78EFC034619463D4809F0AD
S3150800E75031FA0346DAB297F86E30134487F86E300A
S3150800E7600321384809F0C1FC7B68DB7F002B15D1F3
S3150800E77007F13C0007F118010F230D22FAF790FF65
S3150800E78007F13C0207F10C0311461846FAF79AFE00
S3150800E79007F13C031846FAF78FFD14E007F1480025
S3150800E7A007F118010E230C22FAF77AFF07F148023F
S3150800E7B007F10C0311461846FAF784FE07F14803D9
S3150800E7C01846FAF779FD97F86E309CB207F10C03F4
S3150800E7D01846FAF747FC034600222146194809F06D
S3150800E7E0E0F807F10C031846FAF73CFC034619460D
S3150800E7F0144809F0DFF90346DAB297F86E30134485
S3150800E80087F86E3007F1540007F1180113230F2219
S3150800E810FAF746FF07F1540207F10C0311461846AA
S3150800E820FAF750FE07F154031846FAF745FD7B68D8
S3150800E830DB7F012B16D10321024809F056FC15E0AF
S3150800E840786F0708B48C0120740E0708780E07083D
S3150800E8507C0E0708800E070810670708840E07084D
S3150800E860880E070801212F4809F03FFC97F86E30FB
S3150800E8709CB207F10C031846FAF7F4FB034600228C
S3150800E8802146284809F08DF807F10C031846FAF7CF
S3150800E890E9FB03461946234809F08CF90346DAB220
S3150800E8A097F86E30134487F86E3003211D4809F037
S3150800E8B01CFC07F1600307F1180113221846FEF73E
S3150800E8C0FFFD07F1600207F10C0311461846FAF737
S3150800E8D0F9FD07F160031846FAF7EEFC97F86E3073
S3150800E8E09CB207F10C031846FAF7BCFB0346002254
S3150800E8F021460C4809F055F806E07B685B6900225A
S3150800E9000021084809F04DF807F10C031846FAF7F4
S3150800E910D3FC07F118031846FAF7CEFC00BF743784
S3150800E920BD4690BDB48C012080B483B000AF78603A
S3150800E9300B46FB707B68FA781A7000BF0C37BD4629
S3150800E9405DF8047B704780B483B000AF78607B685D
S3150800E9501B7818460C37BD465DF8047B704780B5B2
S3150800E96082B000AF78607B68DB68002B07D07B68D5
S3150800E970DB687868984703461A467B681A7000BFB2
S3150800E9800837BD4680BD80B483B000AF7860396073
S3150800E9907B683A681A6300BF0C37BD465DF8047B8E
S3150800E9A0704780B483B000AF78607B6800221A7421
S3150800E9B000BF0C37BD465DF8047B704780B483B052
S3150800E9C000AF78607B6801221A7400BF0C37BD4619
S3150800E9D05DF8047B704780B483B000AF78607B68CD
S3150800E9E01B7C18460C37BD465DF8047B704780B41F
S3150800E9F085B000AFF860B9601346FB71FB68BA686A
S3150800EA009A61FB68FA791A77FB6893F82030FA79E5
S3150800EA10B2FBF3F3DAB2FB689A77FB6893F8202027
S3150800EA20FB79B3FBF2F102FB01F29B1ADBB2002B76
S3150800EA3005D0FB689B7F0133DAB2FB689A7700BF83
S3150800EA401437BD465DF8047B704780B483B000AFC9
S3150800EA5078607B689A697B6893F91D309B0013443C
S3150800EA601B6818460C37BD465DF8047B704780B4B2
S3150800EA7083B000AF78607B681B6B18460C37BD46C1
S3150800EA805DF8047B704780B483B000AF7860396066
S3150800EA907B683A689A6200BF0C37BD465DF8047B0E
S3150800EAA0704780B483B000AF78607B689B6A002BA0
S3150800EAB001D1002300E0012318460C37BD465DF856
S3150800EAC0047B704780B483B000AF78607B6800220F
S3150800EAD01A707B6801221A7400BF0C37BD465DF8B0
S3150800EAE0047B704780B584B000AFF860B9607A607F
S3150800EAF0FB680022DA60FB6801221A74FB681B684F
S3150800EB001B68B968F8689847FB681B6804331B6874
S3150800EB107968F868984700BF1037BD4680BD80B44D
S3150800EB2083B000AF786039603B68002B02D17B6800
S3150800EB3001221A747B683A68DA6000BF0C37BD4652
S3150800EB405DF8047B704780B483B000AF78603960A5
S3150800EB507B683A685A6000BF0C37BD465DF8047B8F
S3150800EB60704780B483B000AF786039607B683A68D4
S3150800EB709A6000BF0C37BD465DF8047B704780B5C8
S3150800EB8082B000AF78607B68DB68002B05D07B68B5
S3150800EB90DB681846FEF716FD02E07B685B68984757
S3150800EBA000BF0837BD4680BD80B582B000AF78602B
S3150800EBB07B68DB68002B05D07B68DB681846FEF7A8
S3150800EBC021FE02E07B689B68984700BF0837BD4670
S3150800EBD080BD80B582B000AF78607B68DB68002BAB
S3150800EBE00BD07B68DB681846FFF7F5FE03461A4626
S3150800EBF07B681A747B681B7C01E07B681B7C184663
S3150800EC000837BD4680BD80B582B000AF78607B68A6
S3150800EC10DB68002B04D07B68DB681846FFF7C1FE6B
S3150800EC207B6800221A7400BF0837BD4680BD80B5D0
S3150800EC3082B000AF78607B68DB68002B04D07B6805
S3150800EC40DB681846FFF7BAFE7B6801221A7400BF14
S3150800EC500837BD4680BD80B483B000AF78607B6856
S3150800EC60DB6818460C37BD465DF8047B704780B4F0
S3150800EC7083B000AF78607B6800221A727B68012235
S3150800EC8083F848207B68062283F8812000BF0C376A
S3150800EC90BD465DF8047B704780B582B000AF7860EA
S3150800ECA07B689B68002B04D07B689B681846FFF737
S3150800ECB0DEFF00BF0837BD4680BD80B582B000AF15
S3150800ECC078607B685B68002B02D07B685B68984736
S3150800ECD07B681B681C331B687868984700BF083731
S3150800ECE0BD4680BD80B485B000AFF8600B467A603B
S3150800ECF0FB7200BF1437BD465DF8047B7047000001
S3150800ED0080B582B000AF7860054A7B681A6078687B
S3150800ED1005F002FD7B6818460837BD4680BD00BF72
S3150800ED208C42070880B483B000AF78600B46FB704E
S3150800ED301346BB70BA78FB78796898001346DB00EF
S3150800ED40134403440B442033DA791B7A03F00F0388
S3150800ED501B0213439BB218460C37BD465DF8047B6D
S3150800ED60704780B483B000AF78600B46FB701346DB
S3150800ED70BB70BA78FB78796898001346DB001344B1
S3150800ED8003440B4420331A7A1209D2B25B7A1B0168
S3150800ED9013439BB218460C37BD465DF8047B704793
S3150800EDA080B483B000AF78600B46FB701346BB7027
S3150800EDB0BA78FB78796898001346DB001344034455
S3150800EDC00B4420339B79C3F3C013DBB283F00103F2
S3150800EDD0DBB218460C37BD465DF8047B704780B435
S3150800EDE083B000AF78600B46FB701346BB70BA78E9
S3150800EDF0FB78796898001346DB00134403440B44F8
S3150800EE0020339B79C3F30603DBB218460C37BD469D
S3150800EE105DF8047B7047000080B582B000AF78606B
S3150800EE200B46FB70FB78012B1ED17B68B3F91A30B1
S3150800EE3007EE903AF8EEE77A7B68B3F9183007EEF2
S3150800EE40103AB8EEC77AF0EE470AB0EE670A5CF0F9
S3150800EE5047FBF0EE407A9FED167A77EE877A9FEDBC
S3150800EE60157A67EE877A1DE07B68B3F9163007EEE8
S3150800EE70903AF8EEE77A7B68B3F9183007EE103A5D
S3150800EE80B8EEC77AF0EE470AB0EE670A5CF028FBE0
S3150800EE90F0EE407A9FED067A77EE877A9FED057A4F
S3150800EEA067EE877AB0EE670A0837BD4680BD00BFB1
S3150800EEB0DB0F4940E12E654280B483B000AF78602D
S3150800EEC07B6893F82130C3F30303DBB218460C378B
S3150800EED0BD465DF8047B704780B582B000AF7860A8
S3150800EEE000220021786800F01CF800BF0837BD46EC
S3150800EEF080BD80B582B000AF78600B46FB70FB78AA
S3150800EF00202B05D1FF220021786800F00AF804E0DA
S3150800EF100022FF21786800F004F800BF0837BD46D4
S3150800EF2080BD80B483B000AF78600B46FB70134693
S3150800EF30BB707B68FA7883F846207B68BA7883F8D2
S3150800EF4047207B68012283F84D2000BF0C37BD4659
S3150800EF505DF8047B704780B483B000AF78600846DC
S3150800EF6011461A460346FB700B46BB7013467B7068
S3150800EF707B68FA7883F848207B68BA7883F8492052
S3150800EF807B687A7883F84A207B68012283F84D20CB
S3150800EF9000BF0C37BD465DF8047B704780B582B06C
S3150800EFA000AF786039603B681B14D9B23B681B1206
S3150800EFB0DAB23B68DBB27868FFF7CDFF00BF0837E7
S3150800EFC0BD4680BD80B483B000AF78600B46FB7049
S3150800EFD01346BB707B68FA7883F84B207B68BA784F
S3150800EFE083F84C207B68012283F84D2000BF0C373C
S3150800EFF0BD465DF8047B704780B584B000AFF86005
S3150800F000B9603B601346FB71F868FA793B68B968E2
S3150800F01004F068F8FB6878331846FFF771FE084A6B
S3150800F020FB681A60074AFB689A67FB6878331846D4
S3150800F03005F072FBFB6818461037BD4680BD00BF59
S3150800F040504207088042070880B483B000AF786052
S3150800F0507B685B7D18460C37BD465DF8047B7047B8
S3150800F06080B584B000AFF8600B467A60FB72FB6827
S3150800F0707833F97A7A68184605F089FA00BF1037A6
S3150800F080BD4680BD80B582B000AF78607B687833B6
S3150800F090184605F041FB786800F055F87B685B6810
S3150800F0A0002B05D17B687833FF211846FFF776FFDA
S3150800F0B000BF0837BD4680BD80B582B000AF786016
S3150800F0C07B687833184605F027FB00BF0837BD462E
S3150800F0D080BD80B596B000AF7860396007F1080347
S3150800F0E04F22002118465DF019FB52233B7211236B
S3150800F0F07B728023BB72FF233B733B685B78FB7391
S3150800F1003B681B783B743B689B787B743B68DB7871
S3150800F110BB743B681B79FB743B685B793B753B6842
S3150800F1209B797B753B680022DA7107F108034F2249
S3150800F1301946786800F01AF800BF5837BD4680BDF2
S3150800F140A0F17800C5E780B584B000AF78604323A6
S3150800F1503B7302237B7307F10C0302221946786876
S3150800F16000F004F800BF1037BD4680BD90B587B0E3
S3150800F17002AFF860B9601346FB71FB689868FB68D4
S3150800F1809989FB689B7DFA68D27DFC790192009388
S3150800F1902346BA6803F042F800BF1437BD4690BD4F
S3150800F1A080B483B000AF7860044A7B681A607B68D5
S3150800F1B018460C37BD465DF8047B704700420708C1
S3150800F1C080B582B000AF786039607B681846FFF773
S3150800F1D0E7FF074A7B681A607B68181D054B002203
S3150800F1E03968FFF709FF7B6818460837BD4680BDB2
S3150800F1F0B0410708A00E070880B582B000AF786056
S3150800F200084611461A460346FB700B46BB70134662
S3150800F2107B707B6803F17C007B78BA78F978FFF716
S3150800F2209AFE00BF0837BD4680BD80B582B000AFE4
S3150800F23078600B46FB701346BB707B687C33BA78E4
S3150800F240F9781846FFF76EFD034618460837BD4697
S3150800F25080BD80B582B000AF78600B46FB70134660
S3150800F260BB707B687C33BA78F9781846FFF779FD66
S3150800F270034618460837BD4680BD80B582B000AF44
S3150800F28078600B46FB707B687C33FA781146184623
S3150800F29005F06DF9034618460837BD4680BD80B5AA
S3150800F2A082B000AF78600B46FB707B687C33FA78D7
S3150800F2B01146184605F022F9034618460837BD4692
S3150800F2C080BD80B582B000AF78600B46FB707B6866
S3150800F2D07C33FA781146184605F090F80346184626
S3150800F2E00837BD4680BD80B582B000AF78600B4652
S3150800F2F0FB707B687C33FA781146184605F0B4F83B
S3150800F300034618460837BD4680BD80B582B000AFB3
S3150800F31078600B46FB707B687C33FA781146184692
S3150800F320FFF77AFDF0EE407AB0EE670A0837BD4679
S3150800F33080BD80B582B000AF78600B46FB7013467F
S3150800F340BB707B687C33BA78F9781846FFF747FDB7
S3150800F350034618460837BD4680BD80B582B000AF63
S3150800F36078600B46FB701346BB707B687C33BA78B3
S3150800F370F9781846FFF714FD034618460837BD46C0
S3150800F38080BD80B582B000AF78607B687C33184654
S3150800F390FFF792FD034618460837BD4680BD80B57F
S3150800F3A082B000AF78607B687C331846FFF794FD1F
S3150800F3B000BF0837BD4680BD80B582B000AF786013
S3150800F3C00B46FB707B687C33FA7811461846FFF7C4
S3150800F3D090FD00BF0837BD4680BD80B582B000AF3E
S3150800F3E078600B46FB701346BB707B687C33BA7833
S3150800F3F0F9781846FFF795FD00BF0837BD4680BD6A
S3150800F40080B582B000AF78600B46FB701346BB70C0
S3150800F4107B687C33BA78F9781846FFF7D3FD00BFC6
S3150800F4200837BD4680BD80B582B000AF78607B687E
S3150800F43004331846FFF708FE034618460837BD4644
S3150800F44080BD80B582B000AF78607B68043318460B
S3150800F45003F0B9FE00BF0837BD4680BD80B582B04F
S3150800F46000AF78607B6804331846FFF715FC00BFC9
S3150800F4700837BD4680BD80B483B000AF78607B682E
S3150800F4800022DA717B6818460C37BD465DF8047BA6
S3150800F4907047000080B582B000AF7860114A7B687B
S3150800F4A01A607B68043300221A605A607B6804334A
S3150800F4B01846FFF7E0FF7B680C3300221A605A6093
S3150800F4C07B680C331846FFF7D6FF7B680022A3F843
S3150800F4D04C20786805F001FC7B6818460837BD465D
S3150800F4E080BD00BF2447070880B483B000AF7860AA
S3150800F4F00B46FB70FB787A680C339B0013445B68F9
S3150800F500C3F30B239BB218460C37BD465DF8047B44
S3150800F510704780B483B000AF78600B46FB70FB7809
S3150800F5207A680C339B001344DB88C3F30B139BB236
S3150800F53018460C37BD465DF8047B704780B483B027
S3150800F54000AF78600B46FB70FB787A680C339B003B
S3150800F55013441B79C3F3C013DBB283F00103DBB298
S3150800F56018460C37BD465DF8047B704780B483B0F7
S3150800F57000AF78600B46FB70FB787A680C339B000B
S3150800F58013441B79C3F30603DBB218460C37BD4692
S3150800F5905DF8047B7047000080B582B000AF7860E4
S3150800F5A00B46FB70FB78012B22D17B68B3F92D3013
S3150800F5B01BB25B4207EE903AF8EEE77A7B68B3F93E
S3150800F5C02B301BB25B4207EE103AB8EEC77AF0EE64
S3150800F5D0470AB0EE670A5BF083FFF0EE407A9FEDCC
S3150800F5E0177A77EE877A9FED167A67EE877A20E0A4
S3150800F5F07B68B3F929301BB207EE903AF8EEE77A42
S3150800F6007B68B3F92B301BB25B4207EE103AB8EEB3
S3150800F610C77AF0EE470AB0EE670A5BF061FFF0EED4
S3150800F620407A9FED067A77EE877A9FED057A67EE40
S3150800F630877AB0EE670A0837BD4680BDDB0F4940BA
S3150800F640E12E654280B582B000AF786000220021C5
S3150800F650786800F01CF800BF0837BD4680BD80B545
S3150800F66082B000AF78600B46FB70FB78202B05D183
S3150800F670FF220021786800F00AF804E00022FF2142
S3150800F680786800F004F800BF0837BD4680BD80B42E
S3150800F69083B000AF78600B46FB701346BB707B687F
S3150800F6A0FA7883F842207B68BA7883F843207B6827
S3150800F6B0012283F84A2000BF0C37BD465DF8047B5B
S3150800F6C0704780B483B000AF7860084611461A4682
S3150800F6D00346FB700B46BB7013467B707B68FA7853
S3150800F6E083F847207B68BA7883F848207B687A785D
S3150800F6F083F849207B68012283F84A2000BF0C372B
S3150800F700BD465DF8047B704780B582B000AF78606F
S3150800F71039603B681B14D9B23B681B12DAB23B68E6
S3150800F720DBB27868FFF7CDFF00BF0837BD4680BD5E
S3150800F73080B487B000AFF860B9607A60BB687B6157
S3150800F7407B685A1E7A60002B14BF01230023DBB2A4
S3150800F750002B10D07B695A1C7A611B781A46FB6805
S3150800F760DBB253409B00074A13441A68FB681B0A1E
S3150800F7705340FB60E4E7FB6818461C37BD465DF856
S3150800F780047B70479042070880B584B000AFF860E4
S3150800F790B9603B601346FB71F868FA793B68B9684B
S3150800F7A003F0A0FCFB6878331846FFF773FE0A4A95
S3150800F7B0FB681A60094AFB689A67FB68002283F8A7
S3150800F7C0C620FB687833184605F087FAFB681846A2
S3150800F7D01037BD4680BD00BFE8460708184707082A
S3150800F7E080B483B000AF78607B685B7D18460C37C1
S3150800F7F0BD465DF8047B704780B584B000AFF860FD
S3150800F8000B467A60FB72FB687833F97A7A68184691
S3150800F81005F087F900BF1037BD4680BD80B582B0B8
S3150800F82000AF78607B687833184605F056FA786832
S3150800F83000F0BFF87B685B68002B06D17B687833DD
S3150800F8404FF47F011846FFF75FFF00BF0837BD4634
S3150800F85080BD80B582B000AF78607B687833184683
S3150800F86005F03BFA00BF0837BD4680BD90B59BB092
S3150800F87002AF7860396007F10C034F220021184661
S3150800F8805CF04CFFA2233B7331237B737B6893F8B0
S3150800F890C6301B01DBB2BB737B6893F8C6300133F5
S3150800F8A0DAB27B6883F8C6207B6893F8C6300F2BDC
S3150800F8B00CBF01230023DBB2002B03D07B68002298
S3150800F8C083F8C6201023FB73FF233B74F7237B744E
S3150800F8D03B685B78BB743B681B78FB743B689B781A
S3150800F8E03B767B6803F1840207F10C030E33194655
S3150800F8F0104605F07FFA7B6803F17C0207F10C03DA
S3150800F90019331946104605F075FA032387F8363079
S3150800F9103B68DB78002B01D0012300E0022387F83F
S3150800F92039303B681B7987F83B303B685B7987F849
S3150800F9303C303B689B7987F83D303B68DB7987F834
S3150800F9403E3007F10C034B2219464FF0FF30FFF704
S3150800F950EFFE0346DB43FB65FB6DDBB287F85730EA
S3150800F960FB6D1B0ADBB287F85830FB6D1B0CDBB24C
S3150800F97087F85930FB6D1B0EDBB287F85A303B68A7
S3150800F98000221A727B6898687B6899897B681B7E57
S3150800F9907A68527E07F10C04019200934F2322469F
S3150800F9A002F03CFC00BF6437BD4690BDA0F178006C
S3150800F9B05CE790B587B002AF786043233B730923B1
S3150800F9C07B737B6898687B6899897B689B7D7A6876
S3150800F9D0D27D07F10C04019200930223224602F01D
S3150800F9E01DFC00BF1437BD4690BD000080B582B02F
S3150800F9F000AF786039607B681846FFF7D1FB074A85
S3150800FA007B681A607B68181D054B00223968FFF76A
S3150800FA10BBFE7B6818460837BD4680BD9846070872
S3150800FA20A80E070880B582B000AF78600846114670
S3150800FA301A460346FB700B46BB7013467B707B6801
S3150800FA4003F17C007B78BA78F978FFF73AFE00BFB5
S3150800FA500837BD4680BD80B582B000AF78600B46DA
S3150800FA60FB701346BB707B687C33FA7811461846E0
S3150800FA70FFF73AFD034618460837BD4680BD80B5F0
S3150800FA8082B000AF78600B46FB701346BB707B688C
S3150800FA907C33FA7811461846FFF73BFD03461846AD
S3150800FAA00837BD4680BD80B582B000AF78600B468A
S3150800FAB0FB707B687C33FA781146184605F021F806
S3150800FAC0034618460837BD4680BD80B582B000AFEC
S3150800FAD078600B46FB707B687C33FA7811461846CB
S3150800FAE004F0D6FF034618460837BD4680BD80B5E4
S3150800FAF082B000AF78600B46FB707B687C33FA787F
S3150800FB001146184604F042FF034618460837BD4614
S3150800FB1080BD80B582B000AF78600B46FB707B680D
S3150800FB207C33FA781146184604F068FF03461846EF
S3150800FB300837BD4680BD80B582B000AF78600B46F9
S3150800FB40FB707B687C33FA7811461846FFF724FD6C
S3150800FB50F0EE407AB0EE670A0837BD4680BD80B53C
S3150800FB6082B000AF78600B46FB701346BB707B68AB
S3150800FB707C33FA7811461846FFF7F8FC0346184610
S3150800FB800837BD4680BD80B582B000AF78600B46A9
S3150800FB90FB701346BB707B687C33FA7811461846AF
S3150800FBA0FFF7CCFC034618460837BD4680BD80B42F
S3150800FBB083B000AF78600F2318460C37BD465DF852
S3150800FBC0047B704780B582B000AF78607B687C3371
S3150800FBD01846FFF737FD00BF0837BD4680BD80B51C
S3150800FBE082B000AF78600B46FB707B687C33FA788E
S3150800FBF011461846FFF733FD00BF0837BD4680BDDE
S3150800FC0080B582B000AF78600B46FB701346BB70B8
S3150800FC107B687C33BA78F9781846FFF738FD00BF59
S3150800FC200837BD4680BD80B483B000AF78600B4608
S3150800FC30FB701346BB7000BF0C37BD465DF8047BEE
S3150800FC40704780B582B000AF78607B680433184689
S3150800FC50FFF7C6FD034618460837BD4680BD80B582
S3150800FC6082B000AF78607B680433184603F0ABFABD
S3150800FC7000BF0837BD4680BD80B582B000AF78604A
S3150800FC807B6804331846FFF707F800BF0837BD46F8
S3150800FC9080BD80B483B000AF786039607B683A680D
S3150800FCA05A6000BF0C37BD465DF8047B70470000FC
S3150800FCB098B500AF0F4B1B78002B0AD10E4B18686E
S3150800FCC00D4B1B681B681C68FF2300220021A047F8
S3150800FCD00DE0084B1B78012B09D1084B1868074B18
S3150800FCE01B681B681C680023FF220021A04700BF71
S3150800FCF098BD00BFF9110020001200200412002050
S3150800FD0090B583B000AF0346FB711E4AFB791370AA
S3150800FD10FB79002B16D1CC205BF0EAFA03461C4689
S3150800FD20194B1B6819462046FFF74AFA174B1C6001
S3150800FD30164B1B68043316491846FFF7AAFF134BE0
S3150800FD401B681AE0FB79012B16D1CC205BF0D0FAA0
S3150800FD5003461C460C4B1B6819462046FFF746FE11
S3150800FD600C4B1C600B4B1B68043309491846FFF7FC
S3150800FD7090FF084B1B6800E0002318460C37BD4669
S3150800FD8090BD00BFF9110020FC11002000120020D0
S3150800FD90B1FC00080412002080B483B000AF78607C
S3150800FDA03960064B00221A70054A3B6813607B6867
S3150800FDB018460C37BD465DF8047B7047F9110020DC
S3150800FDC0FC11002080B483B000AF78607B681846C9
S3150800FDD00C37BD465DF8047B704780B483B000AF2E
S3150800FDE07860084611461A460346FB700B46BB70F8
S3150800FDF013467B70002318460C37BD465DF8047B16
S3150800FE00704780B483B000AF7860084611461A463A
S3150800FE100346FB700B46BB7013467B7000231846DF
S3150800FE200C37BD465DF8047B704780B483B000AFDD
S3150800FE307860002318460C37BD465DF8047B70478A
S3150800FE4080B483B000AF7860002318460C37BD46EF
S3150800FE505DF8047B704780B483B000AF78600023F8
S3150800FE6018460C37BD465DF8047B704780B483B0EE
S3150800FE7000AF78600B46FB7000BF0C37BD465DF8D7
S3150800FE80047B704780B483B000AF78600B467B80F4
S3150800FE9013463B80002318460C37BD465DF8047BA5
S3150800FEA0704780B483B000AF78600B46FB700023C0
S3150800FEB018460C37BD465DF8047B704780B483B09E
S3150800FEC000AF78600B46FB70012318460C37BD4619
S3150800FED05DF8047B704780B483B000AF78607B68B8
S3150800FEE018460C37BD465DF8047B704780B485B06C
S3150800FEF000AF786039600023FB73FB7B0F2B12D8A9
S3150800FF00FA7B7B681E3253F82230002B07D1FA7B26
S3150800FF107B681E32396843F82210002304E0FB7B15
S3150800FF200133FB73E9E7D32318461437BD465DF85A
S3150800FF30047B704780B483B000AF7860044A7B685E
S3150800FF401A607B6818460C37BD465DF8047B704717
S3150800FF503047070880B483B000AF78607B6800221A
S3150800FF601A707B6800225A7000229A700022DA7092
S3150800FF7000221A717B6818460C37BD465DF8047B6B
S3150800FF80704780B483B000AF78607B6800221A603F
S3150800FF907B6800221A717B6800225A717B681846B2
S3150800FFA00C37BD465DF8047B704780B483B000AF5C
S3150800FFB0786039603B68D3F801207B681A603B6833
S3150800FFC01A787B685A717B685A797B681A7100BF00
S3150800FFD00C37BD465DF8047B704780B483B000AF2C
S3150800FFE078607B6800221A607B6800221A717B6839
S3150800FFF00022DA807B6818460C37BD465DF8047B1C
S31508010000704780B483B000AF786039603B68D3F835
S3150801001001207B681A607B680022DA8000BF0C37F2
S31508010020BD465DF8047B704780B485B000AFF860C3
S31508010030B9607A607B80FB681B79002B02D0012BA3
S3150801004009D029E0FB687A88DA80FB681B790133D5
S31508010050DAB2FB681A71FB68DB88002B15D07B685E
S315080100601B88002B11D0FB68DB88013B9AB2FB6821
S31508010070DA80BB681B685A1CBB681A607B681B88D8
S31508010080013B9AB27B681A80E5E7FB68DB88002B9F
S3150801009002D1FB6800221A71FB68DB88002B0CBFB2
S315080100A001230023DBB218461437BD465DF8047BED
S315080100B0704780B483B000AF7860084611461A4687
S315080100C00346FB700B46BB7013467B7000BF0C37AB
S315080100D0BD465DF8047B704780B483B000AF786095
S315080100E0044A7B681A607B6818460C37BD465DF87A
S315080100F0047B7047B447070880B483B000AF7860C3
S315080101007B6893F8503018460C37BD465DF8047B7A
S31508010110704780B483B000AF78607B6893F87A3013
S3150801012018460C37BD465DF8047B704780B483B02A
S3150801013000AF78600B46FB70FB78E02B0CBF012300
S315080101400023DBB218460C37BD465DF8047B7047C1
S3150801015080B483B000AF78600B467B8013463B8042
S315080101607B8840F65C22934204D13B8842F2E8122E
S31508010170934209D07B8840F20D52934206D13B88BF
S3150801018040F25A62934201D101232DE07B681B7D1F
S31508010190002B13D17B685B7D002B0FD17B689B7D80
S315080101A0002B0BD17B68DB7D002B07D17B681B7E7F
S315080101B0002B03D17B685B7E002B14D07B8840F231
S315080101C04C5293420FD13B88B3F51A7F09D03B882D
S315080101D040F22F42934204D03B8840F2D5329342F3
S315080101E001D1012300E0002318460C37BD465DF80E
S315080101F0047B704780B584B000AF786039607B684E
S315080102001846FFF797FE7B6804331846FFF764FF25
S315080102102B4A7B681A602B4A7B685A607B680022E6
S3150801022083F841207B68002283F843207B680022FB
S3150801023083F846207B68002283F848207B680022E1
S3150801024083F849207B683A68DA647B68002283F878
S3150801025050207B68012283F85E207B6800221A669B
S315080102607B68002283F878207B68002283F879204E
S315080102707B68002283F87A200023FB73FB7B032B20
S315080102800AD8FB7B7A6818339B00134400225A600C
S31508010290FB7B0133FB73F1E7786800F07DFA7B6835
S315080102A0DB6C002B06D07B68DB6C7A681146184636
S315080102B0FFF71CFE7B6818461037BD4680BD00BF98
S315080102C074470708A847070890B58FB002AF78604A
S315080102D0084611461A460346FB700B46BB70134681
S315080102E07B70122387F82E3007F10803BB620023BF
S315080102F07B6200233B62786800F04EFA7B68DB6C10
S315080103001846FFF7E8FDF8617B6893F85030002B33
S3150801031001D0D92387E0FB691B681B680021F869AE
S31508010320984778627B6A002B01D1D6237BE07B6AEA
S315080103301B68002B01D1D72375E07B6A1B683B62DA
S315080103407B6803F151027B6A1A607B6A7A789A7133
S315080103507B68D86C07F10803009312230022002159
S3150801036005F02FFF034687F82F307B6A3A6A1A6031
S3150801037097F82F30002B46D1FB691B6804331C689C
S31508010380BB78F9780022F869A04703461A467B68C4
S3150801039083F850207B6893F85030002B01D1D42381
S315080103A041E0BB6A1B79092B17D0BB6ADA797B68EE
S315080103B083F85220BB6A5A7C7B6883F85420BB6A4F
S315080103C01B899AB27B68A3F87620BB6A5B899AB2C5
S315080103D07B68A3F87420E02325E000BF7B68D86C0E
S315080103E07B6893F850100023002205F087FFD1237C
S315080103F087F82F307B681B6808331B68786898472D
S3150801040097F82F300FE000BF97F82F300D2B02D049
S31508010410E12387F82F307B681B6808331B687868E7
S31508010420984797F82F3018463437BD4690BD80B5A2
S3150801043096B002AF7860084611461A460346FB7025
S315080104400B46BB7013467B707B6893F8543087F86C
S315080104504D307B68002283F854207B68DB6C184694
S31508010460FFF739FDB864BB6C1B681B687A6892F89C
S3150801047050201146B86C984778647B6C002B01D1E3
S31508010480D62385E14FF4967049F0A6F87B68D86CB7
S315080104907B6893F850300022002105F02FFF0346B0
S315080104A087F84F3097F84F30002B03D07B6C00222A
S315080104B09A7165E17B6C00229A71BB6C1B681B689B
S315080104C07A6892F850201146B86C984778647B6C24
S315080104D0002B01D1D6235BE17B6C7A789A717B6814
S315080104E0D86C7B6893F850107B685133012204F06D
S315080104F0EEFD034687F84F3097F84F30002B40F052
S3150801050028817B68B3F8763040F24C52934277D112
S315080105107B68B3F87430B3F51A7F0DD07B68B3F8EE
S31508010520743040F22F42934206D07B68B3F8743098
S3150801053040F2D532934263D1642049F04DF87B6885
S31508010540D86C7B6893F850107B6893F85120012387
S3150801055005F002FF034687F84F3097F84F30002B16
S3150801056040F0F9807B681B7D002B13D17B685B7D8E
S31508010570002B0FD17B689B7D002B0BD17B68DB7D24
S31508010580002B07D17B681B7E002B03D17B685B7E22
S31508010590002B19D07B68B3F87430B3F51A7F06D0EF
S315080105A07B68B3F8743040F22F42934206D17B68D8
S315080105B014331946786802F0B0F805E07B681433FD
S315080105C01946786802F0E9F87B68D86C7B6893F875
S315080105D050107B6893F85120002305F0BDFE7B6817
S315080105E0D86C7B6893F850100023002205F086FE2C
S315080105F07B681B6808331B6878689847D123C7E06E
S31508010600002387F84E3097F84E2097F84D309A42D6
S315080106105ED27B68B3F8763040F65C22934206D107
S315080106207B68B3F8743042F2E81293420DD07B68C6
S31508010630B3F8763040F20D52934220D17B68B3F875
S31508010640743040F25A62934219D17B681A1D07F138
S3150801065008031146184602F0F3F87B68D86C7B68E4
S3150801066093F8501097F84E2007F1080300931346A4
S31508010670002205F0F6FD034687F84F3018E07B683F
S315080106801A1D07F108031146184602F027F97B6877
S31508010690D86C7B6893F8501097F84E2007F1080339
S315080106A000931346002205F0DCFD034687F84F3018
S315080106B097F84F30002B50D17B6893F85E30032BA7
S315080106C005D897F84E30013387F84E309BE700BFBF
S315080106D07B6893F85E30032B45D97B68D86C7B68B9
S315080106E093F850107B6893F85E207B68513304F0C9
S315080106F0EEFC034687F84F3097F84F30002B2ED182
S315080107007B68D86C7B6893F850107B6893F8512006
S315080107107B6893F85D3005F01FFE034687F84F3076
S3150801072097F84F30002B1CD17B686422A3F88420EC
S315080107307B680022A3F882207B68002283F8812047
S315080107407B6800221A727B68012283F87A200023CB
S315080107501EE000BF14E000BF12E000BF10E000BFBA
S315080107600EE000BF0CE000BF7B68D86C7B6893F88D
S3150801077050100023002205F0C1FDD12387F84F3020
S315080107807B681B6808331B687868984797F84F3069
S3150801079018465037BD4680BD80B584B000AF786035
S315080107A00023FB73FB7B032B45D8FA7B7968134639
S315080107B05B0013440B44513300221A70FB7B002B58
S315080107C001D0002000E00820FA7B796813465B0017
S315080107D013440B44523302461A70FA7B796813465E
S315080107E05B0013440B4403F15002D3786FF3000303
S315080107F0D370FA7B796813465B0013440B4403F103
S315080108005002D3786FF34103D370FB7B002B01D0E1
S31508010810012100E00F21FA7B786813465B00134437
S31508010820034403F15002D37861F38703D370FB7B4A
S315080108300133FB73B6E70023FB73FB7B032B1CD841
S31508010840FB7B7A6818339B0013445B68002B10D036
S31508010850FB7B7A6818339B0013445968FB7B7A68DB
S3150801086018339B0013445B681B6808331B680846EA
S315080108709847FB7B0133FB73DFE77B68002283F82C
S3150801088041207B68002283F842207B68002283F896
S3150801089046207B68002283F847207B68002283F87C
S315080108A07D207B68002283F850207B68012283F82B
S315080108B05E207B6800221A667B68002283F878200E
S315080108C07B68002283F87A207B68002283F87920E6
S315080108D000BF1037BD4680BD80B485B000AF7860D3
S315080108E0084611461A460346FB700B46BB7013466B
S315080108F07B707B78002B5DD17B68FA7883F85D2065
S31508010900FB69DB7803F00303032B14D1FB699B789E
S315080109105BB2002B0FDA0123FB73FA7B7968134666
S315080109205B0013440B4403F15002D378012161F3B0
S315080109308703D3700EE0FB69DB7803F00303022B10
S315080109403AD1FB699B785BB2002B01DA022300E0FE
S315080109500323FB73FB699B78FA7B03F00F03D8B279
S31508010960796813465B0013440B44513302461A70E7
S31508010970FB699B889BB2FA7BD8B2796813465B0000
S3150801098013440B44523302461A707B6893F8782055
S31508010990FB699B799A4204D2FB699A797B6883F849
S315080109A078207B6893F85E300133DAB27B6883F886
S315080109B05E2002E000BF00E000BF1437BD465DF8C7
S315080109C0047B7047A0F10400FFF786BF80B582B0AB
S315080109D000AF78607868FFF7DFFE7B68DB6C184646
S315080109E0FFF779FA03461A6808321268796891F8A6
S315080109F0501018469047002318460837BD4680BD53
S31508010A0080B582B000AF78607B6893F87A3083F05E
S31508010A100103DBB2002B01D000231DE048F0D0FD15
S31508010A2002467B681B6ED31ADB43DB0FDBB2002B56
S31508010A3011D048F0C5FD02467B6893F878301A4410
S31508010A407B681A66786800F00BF8786800F022FB74
S31508010A50786800F04BFE002318460837BD4680BD6E
S31508010A60B0B588B002AF78604023BB817B68D86C8B
S31508010A707B6893F850107B6893F854407B688933F8
S31508010A807A6892F8782007F10C05019200932B46B3
S31508010A90224604F084FC0346FB73FB7B002B03D040
S31508010AA0FB7B042B40F0F1827B6893F88930013B8C
S31508010AB0352B00F2EA8201A252F823F09D0C0108B7
S31508010AC0FD0C0108550E01083F0F0108B10E01087A
S31508010AD0FD0F0108E30E01087510010875100108DC
S31508010AE08B1001088B100108751001087510010893
S31508010AF0950B0108751001088B1001088B10010868
S31508010B0075100108751001088B1001088B10010872
S31508010B10CB0F0108F50F01087510010875100108BA
S31508010B2075100108751001088B1001088B10010852
S31508010B308B1001088B100108751001088B1001082C
S31508010B408B1001088B1001088B1001088B10010806
S31508010B508B1001088B1001088B1001088B100108F6
S31508010B608B1001088B1001088B1001088B100108E6
S31508010B708B1001088B1001088B10010865100108FC
S31508010B80751001086D1001088B1001088B100108FA
S31508010B90751001087B6893F88E30002B40F06C8243
S31508010BA07B68B3F8863043F001039AB27B68A3F8F1
S31508010BB086207B6893F88C30012B14D17B6893F8D7
S31508010BC08D30102B0FD17B6893F88F207B6883F8C3
S31508010BD040207B68B3F8863043F040039AB27B68BD
S31508010BE0A3F8862059E07B6893F88C30042B2AD128
S31508010BF07B6893F88D30102B25D17B68B3F8863046
S31508010C0003F40073002B14D17B6893F88F30002B03
S31508010C100FD17B6893F8973003F00803002B04D0B3
S31508010C207B68012283F8792003E07B68002283F838
S31508010C3079207B68B3F8863043F400739AB27B68EF
S31508010C40A3F8862029E07B6893F88C30092B40F0BD
S31508010C5013827B6893F88D30102B40F00D820023A8
S31508010C60FB75FB7D052B0ED8FB7D9A1DFB7D7968EF
S31508010C700A4492F889107A6813440A461A75FB7D64
S31508010C800133FB75EDE77B68B3F8863043F0200343
S31508010C909AB27B68A3F88620EEE1EDE17B6893F8CA
S31508010CA08830042B21D97B6893F84330002B04D173
S31508010CB07B6893F84830002B17D07B68002283F8AD
S31508010CC088207B68002283F841207B68002283F80C
S31508010CD043207B68002283F846207B68002283F83C
S31508010CE048207B680A2283F881207B6893F888303C
S31508010CF00133DAB27B6883F88820C6E17B6893F80A
S31508010D008B30002B00F0BA810023BB757B6893F802
S31508010D108B30BA7D9A4280F0B1817B6893F88B302B
S31508010D20DB00DAB2BB7D194649000B44DBB213443A
S31508010D30BB7300237B757B7D022B11D87B7D1A1D26
S31508010D40BB7B1A447B7D79680A4492F889107A68D4
S31508010D5013440A4683F87E207B7D01337B75EAE7D7
S31508010D607B6893F84330002B38D07B6893F8803042
S31508010D70002B33D17B6893F87F30052B2ED17B6806
S31508010D8093F87E3003F00C03002B27D07B680122F1
S31508010D9083F87C2000233B753B7D052B14D83B7DCE
S31508010DA0D91CBA7D13465B0013445B00CA183B7D08
S31508010DB079680A4492F889107A6813440A461A77B8
S31508010DC03B7D01333B75E7E77B68B3F8863043F033
S31508010DD080039AB27B68A3F886203AE07B6893F889
S31508010DE04830002B31D07B6893F87F3003F00F032E
S31508010DF0052B2AD17B6893F87E3003F0C803002BB4
S31508010E0023D00023FB74FB7C052B14D8FB7CD91C4F
S31508010E10BA7D13465B0013445B00CA18FB7C7968EC
S31508010E200A4492F889107A6813440A461A77FB7CB1
S31508010E300133FB74E7E77B68B3F8863043F0800338
S31508010E409AB27B68A3F8862003E0BB7D0133BB75A4
S31508010E505CE713E17B68B3F8863043F480739AB292
S31508010E607B68A3F886207B6893F88B30002B1AD110
S31508010E707B6893F88C301AB27B6893F88D301B0225
S31508010E801BB203F470631BB213431BB29AB27B689D
S31508010E905A837B68B3F8863043F002039AB27B68BB
S31508010EA0A3F88620F1E07B68062283F88120ECE02E
S31508010EB07B6893F88B30002B40F0E2807B68B3F8AF
S31508010EC0863043F004039AB27B68A3F886207B68D0
S31508010ED0B3F8863023F002039AB27B68A3F886201A
S31508010EE0CEE07B6893F88B30002B40F0CB80002353
S31508010EF0BB74BB7C1D2B18D8BB7C03F10902BB7CD8
S31508010F0079680A4492F889107A6813440A4683F87C
S31508010F102220BB7C7A68134493F82230002B03D035
S31508010F20BB7C0133BB74E4E700BF7B68B3F886304A
S31508010F3043F008039AB27B68A3F88620A2E000234F
S31508010F407B747B7C052B0ED87B7C9A1C7B7C796811
S31508010F500A4492F889107A6813440A461A777B7C00
S31508010F6001337B74EDE700233B743B7C022B10D8DD
S31508010F703B7C03F108023B7C79680A4492F88910A4
S31508010F807A6813440A4683F87E203B7C01333B7416
S31508010F90EBE77B6893F87F3003F00F03052B0AD143
S31508010FA07B6893F87E3003F0C803002B03D07B6877
S31508010FB0012283F847207B68B3F8863043F0100393
S31508010FC09AB27B68A3F886205FE07B6893F8433082
S31508010FD0002B03D0786800F0ECFE56E07B681B69AD
S31508010FE0002B03D0786800F0E4FE4EE0786800F044
S31508010FF093FF4AE0786800F0CAFF46E07B6893F8F9
S315080110008B30002B23D17B6893F84330002B0CD00F
S315080110107B6893F8413083F00103DBB2002B04D0DF
S315080110207B68012283F841202EE07B6893F84830DB
S31508011030002B29D07B6893F8463083F00103DBB295
S31508011040002B21D07B68012283F846201CE07B68AF
S315080110505B8B1946786801F082F87B68102283F861
S31508011060812011E0786800F0CDFF0EE0786801F084
S3150801107010F80AE000BF08E000BF06E000BF04E080
S3150801108000BF02E000BF00E000BF00BF1837BD4641
S31508011090B0BD00BF80B582B000AF78607B6893F8B9
S315080110A08130132B00F2EF8201A252F823F000BF20
S315080110B0011101083B110108C1110108E1110108DB
S315080110C00112010855120108FB120108291301082A
S315080110D0631301088B130108C11301081F140108C2
S315080110E05D1401088315010887160108C915010849
S315080110F0F71501088B120108C1120108E11201084E
S315080111007B68B3F8823001339AB27B68A3F88220F0
S315080111107B68B3F882207B68B3F884309A4240F240
S31508011120B482786800F07DFB7B68012283F8812010
S315080111307B680022A3F88220A7E27B68B3F8823095
S3150801114001339AB27B68A3F882207B68B3F88630AC
S3150801115003F00103002B0BD07B680022A3F8822041
S315080111607B68022283F88120786801F030F88EE2E4
S315080111707B68B3F882207B68B3F884309A4240F2E0
S3150801118086827B68B3F884301A46920013445B0062
S315080111909AB27B68A3F884207B68B3F88430B3F5E8
S315080111A0FA6F04D97B684FF4FA62A3F884207B6846
S315080111B0002283F881207B680022A3F8822066E258
S315080111C07B68B3F8863003F00103002B00F06182D7
S315080111D07B68032283F88120786800F072FB58E265
S315080111E07B68B3F8863003F02003002B00F05382A6
S315080111F0786800F08AFB7B68042283F881204AE23A
S315080112007B68B3F8863003F04003002B00F0458273
S315080112107B68DB68002B0AD07B68DB68194678682F
S3150801122000F05DFC7B68052283F8812035E27B6846
S3150801123093F84930002B08D00021786800F089FB23
S315080112407B68112283F8812027E27B68062283F8CE
S31508011250812022E27B68B3F8863003F00103002B74
S3150801126000F01D827B6893F84930002B08D00021D5
S31508011270786800F06EFB7B68112283F881200EE204
S315080112807B68062283F8812009E27B68B3F88630F9
S3150801129003F40073002B00F004827B6893F879301D
S315080112A0002B08D00121786800F09DFC7B6812228A
S315080112B083F88120F5E17B68062283F88120F0E135
S315080112C07B68B3F8863003F00103002B00F0EB814D
S315080112D0786800F04DFC7B68132283F88120E2E1EF
S315080112E07B68B3F8863003F00103002B00F0DD813B
S315080112F07B68062283F88120D7E17B6893F848301A
S31508011300002B04D17B6893F84330002B07D078680B
S3150801131000F08FFC7B68072283F88120D8E17B687F
S315080113200A2283F88120D3E17B68B3F8863003F07B
S315080113308003002B00F0BB81786800F0B2FC7B6863
S3150801134093F87C30002B07D0786800F074FB7B6833
S315080113500C2283F88120AAE17B68082283F8812080
S31508011360A5E17B68B3F8863003F00103002B00F092
S31508011370A0817B68002283F87C20786800F0ACFCA9
S315080113807B68092283F8812093E17B68B3F886306C
S3150801139003F48073002B00F08E817B68B3F88630E6
S315080113A003F00203002B07D0786800F0ADFE7B68D6
S315080113B00A2283F881207EE1786800F08DFC7AE1C3
S315080113C07B6893F8413083F00103DBB2002B00F010
S315080113D074817B6893F8433083F00103DBB2002BF9
S315080113E000F06B817B6893F8463083F00103DBB22A
S315080113F0002B00F062817B6893F8483083F0010383
S31508011400DBB2002B00F05981786800F029FA7B6875
S3150801141001221A727B680B2283F881204DE17B68D1
S31508011420B3F8863003F01003002B0AD07B6800223C
S315080114301A72786800F0FFFA7B680C2283F881201B
S315080114403DE17B68B3F8863003F00403002B00F016
S3150801145036817B68102283F8812030E17B68B3F8F6
S31508011460863003F00803002B00F02B817B682233BA
S315080114700822994918465BF059FF0346002B47D1C4
S315080114807B68012283F842207B68002283F8442086
S315080114907B68002283F845207B68002283F87B203D
S315080114A07B68223316228D4918465BF03FFF0346B7
S315080114B0002B04D17B68012283F8442028E07B684D
S315080114C022331622864918465BF030FF0346002B65
S315080114D010D17B68012283F87B207B6893F87B20F7
S315080114E07B6883F844207B6893F844207B6883F8FB
S315080114F045200DE07B68223313227A4918465BF0B2
S3150801150015FF0346002B03D17B68012283F87B2054
S315080115107B6893F88030002B17D17B6893F87F306E
S31508011520252B12D17B6893F87E30082B0DD17B6869
S31508011530223313226C4918465BF0F8FE0346002B4A
S3150801154003D17B68012283F87D207B6893F84330B9
S31508011550002B04D17B6893F84830002B09D07B68AF
S3150801156093F87C30002B04D07B68082283F881200D
S31508011570A7E0786800F017FA7B680D2283F88120C6
S315080115809FE07B68B3F8863003F00203002B00F076
S315080115909A807B6893F87D30002B03D07B68012203
S315080115A083F846207B6800225A727B6800229A7269
S315080115B07B680022DA727B680022A3F886207B68A2
S315080115C00F2283F881207EE07B68B3F882300133ED
S315080115D09AB27B68A3F882207B68B3F88230B3F5A8
S315080115E07A7F72D97B680022A3F882207B680A2257
S315080115F083F8812069E07B68B3F8863003F0040339
S31508011600002B64D07B680022A3F886207B68893387
S315080116104022002118465BF081F87B68C9334022D5
S31508011620002118465BF07AF87B68002283F843208C
S315080116307B6893F843207B6883F842207B6893F89C
S3150801164042207B6883F841207B68002283F87C204E
S315080116507B6893F87C207B6883F848207B6893F83D
S3150801166048207B6883F847207B6893F847207B6886
S3150801167083F846207B68002283F87D207B680A224E
S3150801168083F8812023E000BF22E000BF20E000BFED
S315080116901EE000BF1CE000BF1AE000BF18E000BF53
S315080116A016E000BF14E000BF12E000BF10E000BF63
S315080116B00EE000BF0CE000BF0AE000BF08E000BF73
S315080116C006E000BF04E000BF02E000BF00E000BF83
S315080116D000BF0837BD4680BDB00E0708BC0E070817
S315080116E0D40E0708EC0E0708000F0708B0B586B038
S315080116F002AF786040237B817B68D86C7B6893F85E
S3150801170050107B6893F857407B68C9337A6892F81A
S31508011710782007F10A05019200932B46224603F029
S315080117203EFE03467B737B7B002B25D17B89002BF1
S3150801173022D00023FB73FB7B032B1DD8FB7B7A6826
S3150801174018339B0013445B68002B11D0FB7B7A6826
S3150801175018339B0013445868FB7B7A6818339B003F
S3150801176013445B681B681B687A68C9321146984737
S31508011770FB7B0133FB73DEE70023BB73BB7B032BC8
S315080117801CD8BB7B7A6818339B0013445B68002B13
S3150801179010D0BB7B7A6818339B0013445968BB7B0E
S315080117A07A6818339B0013445B681B6804331B680B
S315080117B008469847BB7B0133BB73DFE700BF103789
S315080117C0BD46B0BD80B58CB008AFF860B9601346A8
S315080117D0FB80FB68B3F8863023F001039AB2FB68F5
S315080117E0A3F88620FB68D86CFB6893F85010FB6851
S315080117F093F8512000230793BB680693FB8805934A
S31508011800FB88049300230393002302930023019387
S3150801181000230093202303F0EAFC00BF1037BD46DE
S3150801182080BD80B582B000AF78607B680022A3F8DE
S3150801183086207B68032283F889207B680C2283F83B
S315080118408A207B68002283F88B207B6889330322F0
S3150801185019467868FFF7B6FF00BF0837BD4680BD51
S3150801186080B582B000AF78607B68B3F8863023F024
S3150801187010039AB27B68A3F886207B681A2283F83C
S3150801188089207B680C2283F88A207B68012283F8E9
S315080118908B207B68DB68002B04D07B68032283F8E6
S315080118A08C2003E07B68022283F88C207B688933CD
S315080118B0042219467868FFF785FF00BF0837BD4639
S315080118C080BD80B582B000AF78607B68B3F886309A
S315080118D023F020039AB27B68A3F886207B68092245
S315080118E083F889207B68102283F88A207B68002286
S315080118F083F88B207B688933032219467868FFF7BA
S3150801190061FF00BF0837BD4680BD80B582B000AF14
S3150801191078607B68B3F8863023F040039AB27B6817
S31508011920A3F886207B68012283F889207B68102228
S3150801193083F88A207B68002283F88B207B688933A9
S31508011940032219467868FFF73DFF00BF0837BD46F1
S3150801195080BD80B582B000AF78600B46FB707B68AE
S31508011960B3F8863023F400739AB27B68A3F886200D
S315080119707B68042283F889207B68102283F88A20F1
S315080119807B68012283F88B207B68FA7883F88C20A0
S315080119907B688933042219467868FFF713FF00BF6D
S315080119A00837BD4680BD80B582B000AF78607B68D8
S315080119B0B3F8863023F002039AB27B68A3F886202F
S315080119C07B68092283F889207B68042283F88A20A8
S315080119D07B68072283F88B207B681A7F7B6883F8EC
S315080119E08C207B685A7F7B6883F88D207B689A7F79
S315080119F07B6883F88E207B68DA7F7B6883F88F2083
S31508011A007B6893F820207B6883F890207B6893F89D
S31508011A1021207B6883F891207B68002283F8922035
S31508011A207B6889330A2219467868FFF7CBFE00BF1F
S31508011A300837BD4680BD80B582B000AF78607B6847
S31508011A40B3F8863023F008039AB27B68A3F8862098
S31508011A507B68192283F889207B68042283F88A2007
S31508011A607B680A2283F88B207B681A7F7B6883F858
S31508011A708C207B685A7F7B6883F88D207B689A7FE8
S31508011A807B6883F88E207B68DA7F7B6883F88F20F2
S31508011A907B6893F820207B6883F890207B6893F80D
S31508011AA021207B6883F891207B68012283F89220A4
S31508011AB07B68002283F893207B68002283F89420B0
S31508011AC07B68002283F895207B6889330D221946A5
S31508011AD07868FFF777FE00BF0837BD4680BD90B529
S31508011AE085B000AF786039607B68132283F8892056
S31508011AF07B680C2283F88A203868F6F793FB03463D
S31508011B00DBB20133DAB27B6883F88B200023FB73DF
S31508011B10FC7B3868F6F786FB03469C420ED2FB7BB4
S31508011B203A681A44FB7B033311787A6813440A46E8
S31508011B3083F88920FB7B0133FB73E9E7FB7B0333DE
S31508011B407A681344002283F889207B6803F18904A3
S31508011B503868F6F767FB03469BB204339BB21A460D
S31508011B6021467868FFF72EFE00BF1437BD4690BDA3
S31508011B7080B582B000AF78607B68012283F889203E
S31508011B807B680C2283F88A207B68082283F88B20DD
S31508011B907B68FF2283F88C207B68FF2283F88D20DF
S31508011BA07B68FF2283F88E207B68FF2283F88F20CB
S31508011BB07B68FF2283F890207B681F2283F8912097
S31508011BC07B68FF2283F892207B68002283F89320A2
S31508011BD07B6889330B2219467868FFF7F3FD00BF46
S31508011BE00837BD4680BD80B582B000AF78600B4628
S31508011BF0FB707B68562283F889207B680C2283F860
S31508011C008A207B68012283F88B20FB78002B01D080
S31508011C10012200E000227B6883F88C207B688933E7
S31508011C20042219467868FFF7CDFD00BF0837BD467F
S31508011C3080BD80B582B000AF78607B68B3F8863026
S31508011C4023F080039AB27B68A3F886207B68012279
S31508011C5083F889207B68042283F88A207B68052219
S31508011C6083F88B207B68332283F88C207B688B2250
S31508011C7083F88D207B689E2283F88E207B6830222C
S31508011C8083F88F207B680A2283F890207B68893342
S31508011C90082219467868FFF795FD00BF0837BD4643
S31508011CA080BD80B582B000AF78607B68022283F878
S31508011CB089207B68042283F88A207B68002283F8BE
S31508011CC08B207B688933032219467868FFF77AFDEA
S31508011CD000BF0837BD4680BD80B582B000AF7860C9
S31508011CE07B681C331946786800F004F800BF08378A
S31508011CF0BD4680BD80B582B000AF786039607B682B
S31508011D00B3F8863023F481739AB27B68A3F88620E8
S31508011D107B68052283F889207B68042283F88A2058
S31508011D207B680D2283F88B203B681A787B6883F8D9
S31508011D308C203B685A787B6883F88D203B689A78B3
S31508011D407B6883F88E203B68DA787B6883F88F2076
S31508011D503B681A797B6883F890203B685A797B68D7
S31508011D6083F891207B68182283F892207B68CC221D
S31508011D7083F893207B68012283F894207B680022EC
S31508011D8083F895207B68002283F896207B680022D9
S31508011D9083F897207B68002283F898207B6889332B
S31508011DA0102219467868FFF70DFD00BF0837BD46B2
S31508011DB080BD90B585B000AF78607B680D2283F849
S31508011DC089207B68042283F88A207B68172283F896
S31508011DD08B207B681A7F7B6883F88C207B685A7F07
S31508011DE07B6883F88D207B689A7F7B6883F88E20D1
S31508011DF07B68DA7F7B6883F88F207B6893F82020DD
S31508011E007B6883F890207B6893F821207B6883F8A8
S31508011E1091207B6893F84330002B3FD07B680622DC
S31508011E2083F892207B6893F87B30002B13D000232C
S31508011E30FB73FB7B052B22D8FA7BFB7B0A3379687C
S31508011E400A44117D7A6813440A4683F88920FB7B84
S31508011E500133FB73EDE70023BB73BB7B052B0ED860
S31508011E60BA7BBB7B0A3379680A44117F7A681344C3
S31508011E700A4683F88920BB7B0133BB73EDE7102340
S31508011E807B737B7B192B3CD87B7B7A6813440022B6
S31508011E9083F889207B7B01337B73F2E77B681B69B7
S31508011EA01846F6F7BFF90346DAB27B6883F892203B
S31508011EB000233B733C7B7B681B691846F6F7B2F92E
S31508011EC003469C420FD27B681A693B7B1A443B7BCB
S31508011ED00A3311787A6813440A4683F889203B7BCA
S31508011EE001333B73E6E73B7B0F2B0AD83B7B0A336F
S31508011EF07A681344002283F889203B7B01333B73BC
S31508011F00F1E77B6889331A2219467868FFF75AFC84
S31508011F1000BF1437BD4690BD80B582B000AF78606A
S31508011F207B680E2283F889207B68042283F88A203D
S31508011F307B68062283F88B207B681A7F7B6883F887
S31508011F408C207B685A7F7B6883F88D207B689A7F13
S31508011F507B6883F88E207B68DA7F7B6883F88F201D
S31508011F607B6893F820207B6883F890207B6893F838
S31508011F7021207B6883F891207B68893309221946D9
S31508011F807868FFF71FFC00BF0837BD4680BD80B5DE
S31508011F9082B000AF78607B680C2283F889207B6861
S31508011FA0042283F88A207B68062283F88B207B68C3
S31508011FB01A7F7B6883F88C207B685A7F7B6883F855
S31508011FC08D207B689A7F7B6883F88E207B68DA7F11
S31508011FD07B6883F88F207B6893F820207B6883F8D9
S31508011FE090207B6893F821207B6883F891207B6891
S31508011FF08933092219467868FFF7E4FB00BF0837D9
S31508012000BD4680BD80B582B000AF78607B682B2263
S3150801201083F889207B68042283F88A207B68092251
S3150801202083F88B207B681A7F7B6883F88C207B6812
S315080120305A7F7B6883F88D207B689A7F7B6883F853
S315080120408E207B68DA7F7B6883F88F207B6893F81C
S3150801205020207B6883F890207B6893F821207B6891
S3150801206083F891207B68032283F892207B680022FB
S3150801207083F893207B68002283F894207B68893350
S315080120800C2219467868FFF79DFB00BF0837BD4645
S3150801209080BD80B582B000AF78607B682C2283F85A
S315080120A089207B68042283F88A207B68062283F8C4
S315080120B08B207B681A7F7B6883F88C207B685A7F24
S315080120C07B6883F88D207B689A7F7B6883F88E20EE
S315080120D07B68DA7F7B6883F88F207B6893F82020FA
S315080120E07B6883F890207B6893F821207B6883F8C6
S315080120F091207B688933092219467868FFF762FBC4
S3150801210000BF0837BD4680BD80B582B000AF786094
S315080121107B68112283F889207B68042283F88A2048
S315080121207B68022283F88B207B685B8BDAB27B683B
S3150801213083F88C207B685B8B1B12DBB203F00F03E1
S31508012140DAB27B6883F88D207B68893305221946C4
S315080121507868FFF737FB00BF0837BD4680BD80B5F5
S3150801216082B000AF78600B467B807B68B3F8863017
S3150801217023F004039AB27B68A3F886207B680622BB
S3150801218083F889207B68042283F88A207B680322E6
S3150801219083F88B207B88DAB27B6883F88C207B886E
S315080121A01B12DBB203F00F03DAB27B6883F88D20CA
S315080121B07B68132283F88E207B68893306221946A9
S315080121C07868FFF7FFFA00BF0837BD4680BD80B5BE
S315080121D082B000AF78607B68242283F889207B6807
S315080121E00C2283F88A207B68032283F88B207B687C
S315080121F0042283F88C207B68082283F88D207B686B
S31508012200002283F88E207B6889330622194678686E
S31508012210FFF7D8FA00BF0837BD4680BDB0B58AB00A
S3150801222002AFF8607A601A460B467B8113467B72C9
S315080122306B461D467B7ADC1DBC6123460133184675
S315080122404FF000014FF000024FF00003CB0043EAC4
S315080122505073C2002346013318464FF000014FF070
S3150801226000024FF00003CB0043EA5073C200234635
S3150801227001330733DB08DB00ADEB030D02AB00339B
S315080122807B617B89DAB27B691A707B891B125BB227
S3150801229003F00F035BB243F020035BB2DAB27B694A
S315080122A05A707B7A0433DAB27B699A707B7A043383
S315080122B01B12DAB27B69DA707B697A7A1A717B7AD0
S315080122C01B12DAB27B695A717B6997F830209A71C9
S315080122D07B6997F83420DA710023FB837B7A9BB2FA
S315080122E0FA8B9A420BD2FB8B7A681A44FB8B08331A
S315080122F011787A69D154FB8B0133FB83EEE7FB68CE
S31508012300D86CFB6893F85010FB6893F85A207B7ACF
S315080123109BB208339CB27B690093234603F046F9C6
S315080123200346FB74FB7C002B02D0642047F054F96A
S31508012330AD4600BF2037BD46B0BD80B586B002AFF9
S31508012340F8607B600B467B8113467B72FB68022231
S3150801235083F80921FB687A7A83F80A21FB68042243
S3150801236083F80B21FB68002283F80C213B8BDAB238
S31508012370FB6883F80D213B8B1B12DAB2FB6883F8E5
S315080123800E217B681A78FB6883F80F217B685A78D7
S31508012390FB6883F81021FB6803F209127989002387
S315080123A00193012300930823F868FFF737FF00BF5D
S315080123B01037BD4680BD80B586B002AFF8607B6038
S315080123C00B467B8113467B72FB68032283F809213E
S315080123D0FB687A7A83F80A21FB68082283F80B21BD
S315080123E0FB68002283F80C217B681A78FB6883F85E
S315080123F00D217B685A78FB6883F80E21BB691A7828
S31508012400FB6883F80F21BB695A78FB6883F81021AA
S31508012410FB683A7F83F81121FB68002283F81221B1
S31508012420FB68002283F81321FB68002283F8142134
S31508012430FB6803F2091279890023019301230093AA
S315080124400C23F868FFF7EAFE00BF1037BD4680BDCA
S3150801245080B586B002AFF8607B600B467B81134678
S315080124607B72FB68042283F80921FB687A7A83F870
S315080124700A21FB68082283F80B21FB68002283F8EE
S315080124800C217B681A78FB6883F80D217B685A78DA
S31508012490FB6883F80E21FB68002283F80F21FB688D
S315080124A0002283F81021FB68012283F81121FB68B9
S315080124B0022283F81221FB68FF2283F81321FB68A5
S315080124C0FF2283F81421FB6803F209127989002394
S315080124D00193012300930C23F868FFF79FFE00BFC1
S315080124E01037BD4680BD80B586B002AFF8607B6007
S315080124F00B467B8113467B72FB68052283F809210B
S31508012500FB687A7A83F80A21FB680A2283F80B2189
S31508012510FB68002283F80C217B681A78FB6883F82C
S315080125200D217B685A78FB6883F80E21FB68002227
S3150801253083F80F21FB68002283F81021FB6800222B
S3150801254083F81121FB68002283F81221FB68012216
S3150801255083F81321FB68022283F81421FB68A02261
S3150801256083F81521FB68022283F81621FB6803F21A
S315080125700912798900230193012300930E23F86830
S31508012580FFF74CFE00BF1037BD4680BD80B586B04B
S3150801259002AFF8607B600B467B8113467B72FB6852
S315080125A0062283F80921FB687A7A83F80A21FB68EF
S315080125B0042283F80B21FB68002283F80C217B682F
S315080125C01A78FB6883F80D217B685A78FB6883F8CB
S315080125D00E21BB691A78FB6883F80F21BB695A7803
S315080125E0FB6883F81021FB6803F209127989002335
S315080125F00193012300930823F868FFF70FFE00BF34
S315080126001037BD4680BD80B586B002AFF8607B60E5
S315080126100B467B8113467B72FB68072283F80921E7
S31508012620FB687A7A83F80A21FB68042283F80B216E
S31508012630FB68002283F80C217B681A78FB6883F80B
S315080126400D217B685A78FB6883F80E21BB691A78D5
S31508012650FB6883F80F21BB695A78FB6883F8102158
S31508012660FB6803F209127989002301930123009378
S315080126700823F868FFF7D2FD00BF1037BD4680BDB5
S3150801268080B584B002AF7860084611461A460346FB
S315080126907B800B467B7013463B707B680B2283F865
S315080126A009217B687A7883F80A217B68082283F8EE
S315080126B00B217B68002283F80C217B683A7883F822
S315080126C00D217B683A7C83F80E217B68002283F80A
S315080126D00F217B68002283F810217B68002283F88A
S315080126E011217B68002283F812217B68002283F876
S315080126F013217B68002283F814217B6803F20912EF
S31508012700798800230193012300930C237868FFF746
S3150801271085FD00BF0837BD4680BD80B58EB008AFC0
S315080127207860396001233B7300237B730023FB75B3
S31508012730FB7D052B11D8FB7DC3F105031A463B68C2
S315080127401A44FB7D0233127807F118010B4403F88A
S315080127500C2CFB7D0133FB75EAE77B68D86C7B683B
S3150801276093F850107B6893F851200023079307F1DB
S315080127700C03069308230593082304930023039364
S3150801278003230293F523019309230093212302F0DE
S315080127902EFD00BF1837BD4680BD80B58EB008AF87
S315080127A07860396005233B731023FB7401233B755D
S315080127B002237B751223BB750023FB75FB7D052B55
S315080127C00ED8FB7D3A681A44FB7D0133127807F16E
S315080127D018010B4403F80C2CFB7D0133FB75EDE75F
S315080127E07B68D86C7B6893F850107B6893F8512006
S315080127F00023079307F10C0306930B2305930B2379
S3150801280004930023039303230293052301930923C6
S315080128100093212302F0EBFC00BF1837BD4680BDAB
S3150801282080B483B000AF7860044A7B681A607B681D
S3150801283018460C37BD465DF8047B7047C047070844
S3150801284080B582B000AF786039607B681846FFF7BB
S31508012850E7FF214A7B681A607B683A685A607B6899
S3150801286008331846FDF776FB7B6810331846FDF7E3
S3150801287088FB7B6818331846FDF7AFFB7B68002297
S3150801288083F830207B68002283F831207B68002298
S3150801289083F832207B68002283F838207B6803F1AD
S315080128A020027B68C3F809207B6803F110027B6864
S315080128B0083319461046FDF778FB7B6803F11802C1
S315080128C07B68083319461046FDF79BFB7B6818465B
S315080128D00837BD4680BD00BF6847070880B582B086
S315080128E000AF786039607B681846FFF799FF214A7F
S315080128F07B681A607B683A685A607B6808331846B1
S31508012900FDF728FB7B6810331846FDF73AFB7B6811
S3150801291018331846FDF761FB7B68002283F83020DF
S315080129207B68002283F831207B68002283F83220F5
S315080129307B68002283F838207B6803F120027B68D4
S31508012940C3F809207B6803F110027B68083319462E
S315080129501046FDF72AFB7B6803F118027B680833EA
S3150801296019461046FDF74DFB7B6818460837BD46E4
S3150801297080BD00BF5C47070880B586B000AFF86028
S315080129807A603B600B467B817B89FB827B683B6176
S31508012990FB8A002B0FD007F1160207F1100319461F
S315080129A0F86800F02DF8034683F00103DBB2002B2B
S315080129B000D1EDE700BF1837BD4680BD80B586B0AA
S315080129C000AFF8607A603B600B467B817B89FB82AE
S315080129D07B683B61FB8A002B0FD007F1160207F1D2
S315080129E010031946F86800F081F9034683F00103DC
S315080129F0DBB2002B00D1EDE700BF1837BD4680BD1D
S31508012A00F0B589B002AFF860B9607A60FB68203327
S31508012A107B61FB6820333B61FB6893F83030042BFC
S31508012A2000F25E8101A252F823F000BF412A010893
S31508012A30612A0108A32A0108B72A01087B2B010884
S31508012A40FB6802221A72FB6803F11002FB6808335D
S31508012A5019461046FDF7A9FAFB68012283F83020CA
S31508012A60FB6810337A68B968184603F0D5FF034640
S31508012A7083F00103DBB2002B01D0002331E1FB68AF
S31508012A80D3F809301A78FB6883F83120FB68D3F844
S31508012A9009305A78FB6883F83220FB68022283F8EA
S31508012AA03020FB6820339A1CFB68C3F80920FB68B1
S31508012AB0032283F83020FB6893F83230023B1F2B40
S31508012AC047D801A252F823F0532B0108532B0108CA
S31508012AD0492B0108532B0108532B0108532B0108D5
S31508012AE0532B0108532B0108532B0108532B0108BB
S31508012AF0532B0108532B0108532B0108532B0108AB
S31508012B00532B0108532B0108532B0108532B01089A
S31508012B10532B0108532B0108532B0108532B01088A
S31508012B20532B0108532B0108532B0108532B01087A
S31508012B30532B0108532B0108532B0108532B01086A
S31508012B40532B0108532B0108FB68002283F8332015
S31508012B5000BFFB6893F83130023BDAB2FB681A72A0
S31508012B60FB6803F11002FB68083319461046FDF7A6
S31508012B701CFAFB68042283F83020FB6893F832308C
S31508012B80052B55D0052B00F38580022B02D0042B8B
S31508012B9015D07FE0FB6810337A68B968184603F0E8
S31508012BA03BFF034683F00103DBB2002B01D0002370
S31508012BB097E07B695A79FB6883F8342086E0FB68DD
S31508012BC010337A68B968184603F026FF034683F07E
S31508012BD00103DBB2002B01D0002382E03B695B795C
S31508012BE0E02B6CD13B699B79012B6AD1FB6893F881
S31508012BF03830002B04D03B69DB79002B04D165E022
S31508012C003B69DB79012B5ED1FB68012283F833200E
S31508012C103B699A78FB6883F836203B69DA78FB6862
S31508012C2083F837203B69DA79FB6883F835204DE06C
S31508012C30FB6810337A68B968184603F0EDFE034657
S31508012C4083F00103DBB2002B01D0002349E0FB68C6
S31508012C5093F83330002B38D0FB685B68002B34D0EF
S31508012C60FB685868FB685B681B681C68FB6893F817
S31508012C703410FB6893F83650FB6893F83760FB68A5
S31508012C8093F83530FA6820320192009333462A4682
S31508012C90A0471AE0FB6803F11800FB6893F8313086
S31508012CA09BB2023B9BB27A68B968FDF7BDF9034648
S31508012CB083F00103DBB2002B08D0002311E000BF2B
S31508012CC004E000BF02E000BF00E000BFFB6803F1BB
S31508012CD02002FB68C3F80920FB68002283F830202C
S31508012CE0012318461C37BD46F0BD00BFF0B589B0B3
S31508012CF002AFF860B9607A60FB6820337B61FB68D4
S31508012D0020333B61FB6893F83030042B00F25E8177
S31508012D1001A252F823F000BF2D2D01084D2D0108FF
S31508012D208F2D0108A32D0108672E0108FB680222D1
S31508012D301A72FB6803F11002FB680833194610463C
S31508012D40FDF733F9FB68012283F83020FB6810335D
S31508012D507A68B968184603F05FFE034683F00103F3
S31508012D60DBB2002B01D0002331E1FB68D3F809302F
S31508012D701A78FB6883F83120FB68D3F809305A784A
S31508012D80FB6883F83220FB68022283F83020FB684F
S31508012D9020339A1CFB68C3F80920FB68032283F8D1
S31508012DA03020FB6893F83230023B1F2B47D801A22B
S31508012DB052F823F03F2E01083F2E0108352E01084F
S31508012DC03F2E01083F2E01083F2E01083F2E01081C
S31508012DD03F2E01083F2E01083F2E01083F2E01080C
S31508012DE03F2E01083F2E01083F2E01083F2E0108FC
S31508012DF03F2E01083F2E01083F2E01083F2E0108EC
S31508012E003F2E01083F2E01083F2E01083F2E0108DB
S31508012E103F2E01083F2E01083F2E01083F2E0108CB
S31508012E203F2E01083F2E01083F2E01083F2E0108BB
S31508012E303F2E0108FB68002283F8332000BFFB6898
S31508012E4093F83130023BDAB2FB681A72FB6803F178
S31508012E501002FB68083319461046FDF7A6F8FB6809
S31508012E60042283F83020FB6893F83230052B55D0BD
S31508012E70052B00F38580022B02D0042B15D07FE0A9
S31508012E80FB6810337A68B968184603F0C5FD03462E
S31508012E9083F00103DBB2002B01D0002397E07B69A5
S31508012EA05A79FB6883F8342086E0FB6810337A6820
S31508012EB0B968184603F0B0FD034683F00103DBB297
S31508012EC0002B01D0002382E03B695B79FF2B6CD193
S31508012ED03B699B79012B6AD1FB6893F83830002B43
S31508012EE004D03B69DB79002B04D165E03B69DB79CA
S31508012EF0012B5ED1FB68012283F833203B699A785E
S31508012F00FB6883F836203B69DA78FB6883F8372053
S31508012F103B69DA79FB6883F835204DE0FB681033A5
S31508012F207A68B968184603F077FD034683F001030A
S31508012F30DBB2002B01D0002349E0FB6893F833305C
S31508012F40002B38D0FB685B68002B34D0FB685868C7
S31508012F50FB685B681B681C68FB6893F83410FB68A0
S31508012F6093F83650FB6893F83760FB6893F8353069
S31508012F70FA6820320192009333462A46A0471AE09E
S31508012F80FB6803F11800FB6893F831309BB2023BEA
S31508012F909BB27A68B968FDF747F8034683F00103DF
S31508012FA0DBB2002B08D0002311E000BF04E000BF0C
S31508012FB002E000BF00E000BFFB6803F12002FB68E6
S31508012FC0C3F80920FB68002283F83020012318463C
S31508012FD01C37BD46F0BD00BF80B485B000AF786030
S31508012FE039600023FB73FB7B032B15D8FB7B7A68BF
S31508012FF018339B0013445B68002B09D1FB7B7A6865
S3150801300018339B0013443A685A6097F90F3005E064
S31508013010FB7B0133FB73E6E74FF0FF3318461437A2
S31508013020BD465DF8047B704780B582B000AF786015
S3150801303039600A4A7B681A607B683A689A607B68D5
S315080130409B68002B05D07B689B6879681846FFF753
S31508013050C3FF7B6818460837BD4680BDF847070891
S3150801306080B485B000AFF860B9601346FB80BB68D1
S315080130701B781A46FB88DBB29A420BD1BB6801332F
S315080130801B781A46FB881B1243F020039A4201D18A
S31508013090012300E0002318461437BD465DF8047B7A
S315080130A0704780B485B000AFF8600B467A60FB7252
S315080130B000BF1437BD465DF8047B704780B483B002
S315080130C000AF786000BF0C37BD465DF8047B7047DA
S315080130D080B483B000AF786000BF0C37BD465DF899
S315080130E0047B704780B586B000AFF860B9603B6075
S315080130F01346FB71FB68B9681846FFF795FF1F4A27
S31508013100FB681A60FB68002283F868200023FB75B8
S31508013110FB7D012B09D8FA7DFB680832002143F8AB
S315080131202210FB7D0133FB75F2E7FB689B68FA7990
S3150801313083F84820FB689B683A681A61FB68502245
S3150801314083F86F20FB68002283F87020FB687022E1
S3150801315083F86B20FB68002283F86C20FB687122D8
S3150801316083F86D20FB68002283F86E20F86800F06A
S3150801317007F8FB6818461837BD4680BDCC470708CF
S3150801318080B582B000AF78607B6800225A757B688B
S31508013190002283F869207B68002283F86A207B680D
S315080131A000221A617B680A229A767B68002283F8D4
S315080131B071207B681B6820331B687868984700BFB5
S315080131C00837BD4680BD90B585B002AF78607B688B
S315080131D093F86A30002B14D07B6898687B689989C4
S315080131E07B681B7D0133DAB27B681A757B681A7DA9
S315080131F07B6803F11B047B686F3300932346FFF753
S31508013200C5F97B6898687B6899897B681B7D01335A
S31508013210DAB27B681A757B681A7D7B6803F1180434
S315080132207B686D3300932346FFF7B0F97B681B680B
S3150801323008331B68786898477B680E229A767B68FC
S31508013240092283F8712000BF0C37BD4690BD90B5A1
S3150801325087B002AF786039607B685B7D83F00103D4
S31508013260DBB2002B23D03B6808331B78022B1ED117
S315080132703B680C331B781A463B680D331B781B02D7
S315080132801343012B13D17B689B689B7A83F0010357
S31508013290DBB2002B0BD07B689B6801229A727B6894
S315080132A09B685A8B7B689A817B680A229A767B6827
S315080132B09B685B7A83F00103DBB2002B3AD07B680B
S315080132C09B6893F84730002B34D07B685B7D83F08D
S315080132D00103DBB2002B2DD07B6893F8693083F0AC
S315080132E00103DBB2002B25D03B6808331B78022B80
S315080132F020D13B680C331B781A463B680D331B7883
S315080133001B021343112B15D17B689B68002283F896
S3150801331047207B689B6801225A727B68012283F8E1
S3150801332069207B689B685A8B7B689A817B68002237
S3150801333083F8712078687B689B891A463968FFF794
S315080133408FFE0346002B00F0D9833B6806331B78B2
S315080133501A463B6807331B781B021343012B40F0BF
S315080133609B823B6808331B78012B00F0C1833B68BD
S3150801337008331B78032B40F08D803B6810331B788C
S315080133801A463B6811331B781B021343002B40F086
S31508013390AF833B6812331B781A463B6813331B7895
S315080133A01B021343002B40F0A3833B680E331A78A4
S315080133B07B6893F86F309A4224D13B680F331A78A9
S315080133C07B6893F870309A421CD13B685A7A7B68BD
S315080133D01A753B681A7B7B68DA763B685A7B7B6889
S315080133E01A777B681B7D0133DAB27B681A757B68AD
S315080133F098687B6899897B681A7D7B681B33FFF718
S3150801340027F875E33B680E331A787B6893F86B30B7
S315080134109A421AD13B680F331A787B6893F86C3055
S315080134209A4212D13B685A7A7B681A753B681A7BAD
S315080134307B689A753B685A7B7B68DA757B681B697A
S3150801344043F004027B681A6152E33B680E331A782B
S315080134507B6893F86D309A4240F04A833B680F3394
S315080134601A787B6893F86E309A4240F041833B683C
S315080134705A7A7B681A753B681A7B7B681A763B68A9
S315080134805A7B7B685A767B681B6943F040027B68E6
S315080134901A612DE33B6808331B78022B5AD13B6826
S315080134A00C331B781A463B680D331B781B021343F2
S315080134B0012B12D13B685A7A7B681A753B689A7B4D
S315080134C07B68DA763B68DA7B7B681A777B681B69E7
S315080134D043F480727B681A610AE33B680C331B78F4
S315080134E01A463B680D331B781B021343112B12D165
S315080134F03B685A7A7B681A753B689A7B7B689A752A
S315080135003B68DA7B7B68DA757B681B6943F00102E5
S315080135107B681A61ECE23B680C331B781A463B68F8
S315080135200D331B781B021343132B40F0E1823B68D2
S315080135305A7A7B681A753B689A7B7B681A763B6868
S31508013540DA7B7B685A767B681B6943F010027B68D5
S315080135501A61CDE23B6808331B78052B5ED13B68BF
S3150801356010331B781A463B6811331B781B02134329
S31508013570002B40F0BD823B680C331A787B6893F8C0
S315080135806F309A4212D13B680D331A787B6893F8EB
S3150801359070309A420AD13B685A7A7B681A757B68F9
S315080135A01B6943F400727B681A61A1E23B680C331C
S315080135B01A787B6893F86B309A4212D13B680D33BF
S315080135C01A787B6893F86C309A420AD13B685A7A22
S315080135D07B681A757B681B6943F002027B681A616E
S315080135E086E23B680C331A787B6893F86D309A4209
S315080135F040F07E823B680D331A787B6893F86E300B
S315080136009A4240F075823B685A7A7B681A757B68DC
S315080136101B6943F020027B681A6169E23B6808333B
S315080136201B78042B55D13B680C331A787B6893F8C1
S315080136306F309A4213D13B680D331A787B6893F839
S3150801364070309A420BD17B6898687B6899893B6888
S3150801365009331A787B681B33FEF745FF48E23B6856
S315080136600C331A787B6893F86B309A4213D13B680E
S315080136700D331A787B6893F86C309A420BD17B68C4
S3150801368098687B6899893B6809331A787B68163389
S31508013690FEF729FF2CE23B680C331A787B6893F80E
S315080136A06D309A4240F024823B680D331A787B6864
S315080136B093F86E309A4240F01B827B6898687B6863
S315080136C099893B6809331A787B681833FEF70BFF2B
S315080136D00EE23B6808331B78062B70D13B680C3326
S315080136E01A787B6893F86F309A4212D13B680D338A
S315080136F01A787B6893F870309A420AD13B685A7AED
S315080137007B681A757B681B6943F480627B681A615A
S31508013710EEE13B680C331A787B6893F86B309A4272
S3150801372021D13B680D331A787B6893F86C309A423D
S3150801373019D13B685A7A7B681A757B6898687B68E1
S3150801374099897B681A7D7B6803F16B047B6816335C
S3150801375000932346FEF757FF7B681B6808331B68EF
S3150801376078689847C4E13B680C331A787B6893F804
S315080137706D309A4240F0BC813B680D331A787B68FC
S3150801378093F86E309A4240F0B3813B685A7A7B6867
S315080137901A757B6898687B6899897B681A7D7B6846
S315080137A003F16D047B68183300932346FEF72BFF5C
S315080137B07B681B6808331B687868984798E13B68FB
S315080137C008331B78072B4CD13B680C331A787B6876
S315080137D0DB7E9A4211D13B680D331A787B681B7FD1
S315080137E09A420AD13B685A7A7B681A757B681B69C3
S315080137F043F480427B681A617AE13B680C331A7894
S315080138007B689B7D9A4211D13B680D331A787B6898
S31508013810DB7D9A420AD13B685A7A7B681A757B68BE
S315080138201B6943F008027B681A6161E13B680C3346
S315080138301A787B681B7E9A4240F05A813B680D33A1
S315080138401A787B685B7E9A4240F052813B685A7AC5
S315080138507B681A757B681B6943F080027B681A616D
S3150801386046E13B6808331B780A2B40F041813B68E7
S315080138705A7A7B681A757B6898687B6899897B6828
S315080138801A7D3B680C331C783B680D331B78009313
S315080138902346FEF7F5FE2BE13B6806331A787B686B
S315080138A093F86F309A4240F087803B6807331A785D
S315080138B07B6893F870309A427ED13B6808331B784F
S315080138C0022B31D17B68032283F828203B685A7A78
S315080138D07B6883F829203B689A7A7B6883F82A20D3
S315080138E07B68002283F82B207B68052283F82C202D
S315080138F07B68002283F82D207B68002283F82E201E
S315080139007B68002283F82F207B68002283F8302009
S315080139107B68002283F831207B6828330A221946FE
S31508013920786800F06DFBE0E03B6808331B78042BF0
S3150801393031D17B68052283F828203B685A7A7B684F
S3150801394083F829203B689A7A7B6883F82A207B6862
S31508013950002283F82B207B68052283F82C207B68BC
S31508013960002283F82D207B68022283F82E207B68AB
S31508013970352283F82F207B68002283F830207B6864
S31508013980002283F831207B6828330A221946786891
S3150801399000F036FBA9E03B6808331B78062B40F09C
S315080139A0A4803B68093319783B680A331B781A46A1
S315080139B0786800F03FFB98E03B6806331A787B6825
S315080139C093F86D309A4262D13B6807331A787B685F
S315080139D093F86E309A425AD13B6808331B78A12B6B
S315080139E040F0858045F0ECFD02467B685A673B68E6
S315080139F005331B781B021AB23B6804331B781BB2CA
S31508013A0013431BB2FB817B681B6814331B68FA8955
S31508013A10D2B2013AD1B23A680932786898473B6816
S31508013A2009331B78012B02D0022B16D05FE07B6885
S31508013A301B6A002B27D07B68186A7B681B6A1B6880
S31508013A401C68FB89DBB2023BDAB23B680A33009396
S31508013A50134600227968A04715E07B685B6A002B4C
S31508013A6013D07B68586A7B685B6A1B681C68FB898C
S31508013A70DBB2023BDAB23B680A33009313460022F3
S31508013A807968A04701E000BF31E000BF2FE03B683D
S31508013A9006331A787B6893F86B309A4228D13B68CB
S31508013AA007331A787B6893F86C309A4220D13B68C1
S31508013AB008331B78A32B1BD13B6805331B781B02E4
S31508013AC01AB23B6804331B781BB213431BB2BB8182
S31508013AD07B681B6818331B68BA89D2B2013AD1B21E
S31508013AE03A6809327868984702E000BF00E000BFEB
S31508013AF0786800F007F8786800F0B4F800BF143762
S31508013B00BD4690BDB0B584B002AF78607B689B7E38
S31508013B100E2B00F084800E2B00F39F800A2B02D017
S31508013B200B2B68D099E07B681B6903F48073002B23
S31508013B3041D07B681B6923F480727B681A617B68B4
S31508013B4098687B6899897B681A7D7B6803F16F049D
S31508013B507B681B330125019500932346FEF72BFC51
S31508013B60012045F039FD7B6898687B6899897B68EF
S31508013B701A7D7B6803F16F047B681B330025019569
S31508013B8000932346FEF717FC7B681B7D0133DAB2E7
S31508013B907B681A75012045F01FFD7B6898687B686C
S31508013BA099897B681A7D7B681B33FEF751FC7B6814
S31508013BB00B229A764CE07B681B6903F48063002B21
S31508013BC046D07B681B6923F480627B681A617B682F
S31508013BD0002283F86A207B6898687B6899897B68E4
S31508013BE01A7D7B6803F16F047B681B3300932346B8
S31508013BF0FEF709FD2CE07B681B6903F40073002BB3
S31508013C0028D07B681B6923F400727B681A617B687C
S31508013C10012283F86A207B680A229A761AE07B6871
S31508013C201B6903F48043002B16D07B689A687B686E
S31508013C309B8919461046FEF792FA7B684FF6FF7282
S31508013C409A817B681B6808331B687868984703E084
S31508013C5000BF02E000BF00E000BF00BF0837BD4655
S31508013C60B0BD0000B0B584B002AF78607B6893F848
S31508013C707130013B082B00F22C8101A252F823F086
S31508013C80B13E01084B3D0108833D0108A53C0108E9
S31508013C907D3E0108C33C0108CB3D0108013E0108F0
S31508013CA03D3E01087B681B6903F00203002B00F007
S31508013CB00181786800F0F9F97B68062283F871209A
S31508013CC0F8E07B681B6903F01003002B00F0F48011
S31508013CD07B6898687B6899897B681A7D7B6803F19C
S31508013CE06D047B6818330125019500932346FEF779
S31508013CF062FB012045F070FC7B6898687B689989AE
S31508013D007B681A7D7B6803F16D047B68183300258F
S31508013D10019500932346FEF74EFB7B681B7D013315
S31508013D20DAB27B681A75012045F056FC7B689868FB
S31508013D307B6899897B681A7D7B681833FEF788FB4F
S31508013D407B68082283F87120B6E07B681B6903F05B
S31508013D500403002B00F0B2807B681B7D0133DAB2C5
S31508013D607B681A757B6898687B6899897B681A7D70
S31508013D707B681633FEF76CFB7B68032283F8712098
S31508013D809CE07B681B6903F00203002B00F0988016
S31508013D90786800F08AF9012045F01EFC7B681B7DD6
S31508013DA00133DAB27B681A757B6898687B689989EA
S31508013DB07B681A7D7B686D3313240094FEF7BDFA80
S31508013DC07B68072283F871207AE07B681B6903F018
S31508013DD04003002B76D07B681B7D0133DAB27B6802
S31508013DE01A757B6898687B6899897B681A7D7B68F0
S31508013DF01833FEF72DFB7B68082283F8712061E0F2
S31508013E007B681B6903F02003002B5DD07B689B68E8
S31508013E10002283F846207B689B68002283F84820A5
S31508013E207B6801225A757B681B6810331B687868A2
S31508013E3098477B68012283F8712045E07B681B69F6
S31508013E4003F08003002B41D07B681B7D0133DAB276
S31508013E507B681A757B6898687B6899897B681A7D7F
S31508013E607B6803F116047B686B3300932346FEF7E0
S31508013E708DFB7B68052283F8712027E07B681B6927
S31508013E8003F00803002B23D07B689A687B689B891B
S31508013E9019461046FEF763F97B684FF6FF729A8159
S31508013EA07B6800221A617B68002283F871200FE083
S31508013EB000BF0EE000BF0CE000BF0AE000BF08E04B
S31508013EC000BF06E000BF04E000BF02E000BF00E05B
S31508013ED000BF00BF0837BD46B0BD00BFB0B584B04E
S31508013EE002AF78607B6893F87130002B40F08480CC
S31508013EF07B689B6893F84630002B3AD07B689B68B1
S31508013F005B7A83F00103DBB2002B32D07B685B7DE1
S31508013F1083F00103DBB2002B2BD07B6893F8693061
S31508013F2083F00103DBB2002B23D07B689B68012257
S31508013F305A727B68012283F869207B689B685A8BD1
S31508013F407B689A817B6800221A617B6800221A7550
S31508013F507B6898687B6899897B681A7D7B686B336F
S31508013F6011240094FEF7E9F97B68022283F871208F
S31508013F7041E07B681B6903F00103002B3BD07B689A
S31508013F8098687B6899897B681A7D7B6803F16B045D
S31508013F907B6816330125019500932346FEF70BFA34
S31508013FA0012045F019FB7B6898687B6899897B68CD
S31508013FB01A7D7B6803F16B047B681633002501952E
S31508013FC000932346FEF7F7F97B681B7D0133DAB2C6
S31508013FD07B681A75012045F0FFFA7B6898687B684B
S31508013FE099897B681A7D7B681633FEF731FA7B68F7
S31508013FF0042283F8712000BF00BF0837BD46B0BD53
S3150801400090B587B002AFF860B9601346FB71FB68DB
S315080140109868FB689989FB68DB7EFA68127FFC79E8
S31508014020019200932346BA68FEF7F8F800BF1437E1
S31508014030BD4690BD80B582B000AF78600B46FB7077
S315080140401346BB707B68072283F828207B68FA78B9
S3150801405083F829207B68BA7883F82A207B680022AE
S3150801406083F82B207B68052283F82C207B680022A5
S3150801407083F82D207B68022283F82E207B6835225F
S3150801408083F82F207B68002283F830207B68002282
S3150801409083F831207B6828330A2219467868FFF7A6
S315080140A0AFFF00BF0837BD4680BD90B587B002AFE8
S315080140B078607B6893F86830002B08D07B6893F8A2
S315080140C06830012B03D07B68002283F868207B685F
S315080140D093F8683043F07003DBB2FB737B6898682A
S315080140E07B6899897B689B7D7A68D27D07F10F0485
S315080140F00192009301232246FEF790F800BF143778
S31508014100BD4690BD80B483B000AF0346FB71FB7911
S31508014110002B00F0D480FB79132B00F0D080FB79BB
S31508014120012B00F0CA80FB79142B00F0C680FB79BD
S31508014130022B00F0C080FB79152B00F0BC80FB79BF
S31508014140032B00F0B680FB79162B00F0B280FB79C1
S31508014150082B00F0AC80FB79182B00F0A880FB79BE
S31508014160212B00F0A480FB79262B00F0A080FB7997
S31508014170172B00F09C80FB791B2B00F09880FB79AC
S31508014180332B00F09480FB79092B00F08E80FB79A4
S31508014190192B00F08A80FB79272B00F08680FB79A2
S315080141A0282B00F08280FB790A2B7CD0FB79292BFE
S315080141B079D0FB790B2B74D0FB792A2B71D0FB793B
S315080141C00E2B6CD0FB792B2B69D0FB79242B66D06F
S315080141D0FB790F2B61D0FB792C2B5ED0FB79252B34
S315080141E05BD0FB790C2B56D0FB792D2B53D0FB7961
S315080141F00D2B4ED0FB792E2B4BD0FB79042B46D0B9
S31508014200FB791E2B43D0FB79052B3ED0FB791D2B61
S315080142103BD0FB79062B36D0FB791F2B33D0FB79A4
S31508014220072B2ED0FB79202B2BD0FB792F2B26D0D1
S31508014230FB79102B23D0FB79222B20D0FB79302B4D
S315080142401BD0FB79112B18D0FB791A2B15D0FB79CA
S31508014250232B12D0FB79312B0DD0FB79122B0AD0E7
S31508014260FB791C2B07D0FB79322B01D1132327E0CD
S315080142704FF0FF3324E0122322E0112320E010231C
S315080142801EE00F231CE00E231AE00D2318E00C2371
S3150801429016E00B2314E00A2312E0092310E0082391
S315080142A00EE007230CE006230AE0052308E00423B1
S315080142B006E0032304E0022302E0012300E00023D1
S315080142C018460C37BD465DF8047B704780B584B047
S315080142D000AF0346FB71FB791846FFF713FF034648
S315080142E0FB73FB7B112B02D94FF0FF3301E097F9E2
S315080142F00F3018461037BD4680BD000080B483B024
S3150801430000AF78600B46FB70FB78032B6ED801A2D1
S3150801431052F823F025430108574301088943010848
S31508014320BB4301087B681B7A03F00F03DBB2072B3B
S315080143300DD07B681B7A03F00F03DBB2002B06D086
S315080143407B681B7A03F00F03DBB2012B01D1012332
S315080143504DE000234BE07B681B7A03F00F03DBB2C9
S31508014360012B0DD07B681B7A03F00F03DBB2022BFE
S3150801437006D07B681B7A03F00F03DBB2032B01D14E
S31508014380012334E0002332E07B681B7A03F00F0334
S31508014390DBB2032B0DD07B681B7A03F00F03DBB26C
S315080143A0042B06D07B681B7A03F00F03DBB2052BBF
S315080143B001D101231BE0002319E07B681B7A03F076
S315080143C00F03DBB2052B0DD07B681B7A03F00F03B5
S315080143D0DBB2062B06D07B681B7A03F00F03DBB230
S315080143E0072B01D1012302E0002300E00023184630
S315080143F00C37BD465DF8047B704700BF80B584B0B5
S3150801440000AF78600B46FB70FB781846FFF75EFF36
S315080144100346FB7397F90F30002B01DA00231DE0E1
S3150801442097F90F30032B06DCFB7819467868FFF7F6
S3150801443065FF034612E07B689B68C3F317031946B9
S3150801444097F90F30074A13441B7821FA03F303F04F
S315080144500103002B14BF01230023DBB218461037D2
S31508014460BD4680BD0C48070880B586B000AF7860A8
S315080144700B46FB70FB781846FFF728FF0346FB75CA
S3150801448097F91730002B01DA002331E097F9173035
S31508014490194A13441B781A46012393403B617B68EA
S315080144A093F84320B3F844301B0213431A463B6979
S315080144B01340002B14BF01230023FB737B6893F879
S315080144C04320B3F844301B0213431A463B69DB43C6
S315080144D0134023F07F427B68D1B20020014383F861
S315080144E04310120A92B200210A43A3F84420FB7B27
S315080144F018461837BD4680BD0C48070880B584B0F4
S3150801450000AF78600B46FB70FB781846FFF7DEFEB6
S315080145100346FB7397F90F30002B01DA002322E0DB
S315080145200E20FFF7EFFD03461A4697F90F3093421F
S315080145300CBF01230023DBB2002B02D07B68DB7A98
S3150801454011E00F20FFF7DEFD03461A4697F90F30F3
S3150801455093420CBF01230023DBB2002B02D07B68F8
S315080145601B7B00E0002318461037BD4680BD80B48A
S3150801457083B000AF78600B46FB70FB787A6813440A
S315080145801B7918460C37BD465DF8047B704780B524
S3150801459086B000AFF8600B467A60FB72FB7A012B96
S315080145A040F2A6807B68002B00F0A2807B681B780E
S315080145B0012B0ED1FB68181D7B68591CFB7A013B40
S315080145C0DBB23C2B28BF3C23DBB21A4658F07EF8F7
S315080145D016E07B681B78112B40F09880FB7A032B39
S315080145E040F29680FB68181D7B68D91CFB7A033B51
S315080145F0DBB23C2B28BF3C23DBB21A4658F066F8DF
S31508014600FB689B68C3F31702FB681B6CC3F31703AC
S315080146109A426DD0FB689B68C3F317031A46FB6879
S315080146201B6CC3F31703DB43134023F07F42FB687C
S31508014630D1B20020014383F84310120A92B2002135
S315080146400A43A3F84420FB689B68C3F31701FA6879
S31508014650136C61F3170313640023FB750021F868D3
S31508014660FFF74CFE0346002B03D0FB7D43F0010305
S31508014670FB750121F868FFF741FE0346002B03D0BD
S31508014680FB7D43F00203FB750221F868FFF736FE4E
S315080146900346002B03D0FB7D43F00403FB7503217E
S315080146A0F868FFF72BFE0346002B03D0FB7D43F08A
S315080146B00803FB75FB6893F84E30FA7D9A4217D0CA
S315080146C0FB6893F84E305BB2DB435AB297F9173061
S315080146D013405BB203F00F03D9B2FA6892F843307C
S315080146E061F3030382F84330FB68FA7D83F84E20B1
S315080146F0FB6893F84D30002B0BD0FB681B681B68D1
S31508014700FA6846321146F868984702E000BF00E0A9
S3150801471000BF1837BD4680BD80B485B000AF78604C
S315080147200023FB73FB7B032B08D8FB7B7A681344B6
S315080147307F221A71FB7B0133FB73F3E77A6893686F
S315080147406FF3170393607A68136C6FF31703136497
S315080147500023FB73FB7B012B08D8FB7B7A68134488
S315080147600022DA72FB7B0133FB73F3E70023FB7349
S31508014770FB7B022B1BD80023BB73BB7B012B12D8F7
S31508014780FA7BBB7B796898001346DB001344034424
S315080147900B4403F12002937943F080039371BB7BA9
S315080147A00133BB73E9E7FB7B0133FB73E0E77A6807
S315080147B0137A082161F3030313727A6892F8403079
S315080147C0082161F3030382F840307A6892F843308E
S315080147D06FF3030382F843307B68002283F84E2087
S315080147E07B68002283F847207B6893F847207B681B
S315080147F083F846207B68002283F84A207B6893F871
S315080148004A207B6883F849207B6893F849207B68AE
S3150801481083F848207B68002283F84C207B6893F84C
S315080148204C207B6883F84B207B68002283F84D2057
S3150801483000BF1437BD465DF8047B704780B483B06A
S3150801484000AF78607B6800221A707B680022DA71F3
S3150801485000BF0C37BD465DF8047B704780B584B050
S3150801486000AF0346FB71FB791846FFF74BFC03467D
S31508014870FB73FB7B122B02D94FF0FF3301E097F94B
S315080148800F3018461037BD4680BD000080B483B08E
S3150801489000AF78600B46FB70FB78032B6ED801A23C
S315080148A052F823F0B5480108E748010819490108F3
S315080148B04B4901087B68DB7E03F00F03DBB2072B4C
S315080148C00DD07B68DB7E03F00F03DBB2002B06D02D
S315080148D07B68DB7E03F00F03DBB2012B01D10123D9
S315080148E04DE000234BE07B68DB7E03F00F03DBB270
S315080148F0012B0DD07B68DB7E03F00F03DBB2022BA5
S3150801490006D07B68DB7E03F00F03DBB2032B01D1F4
S31508014910012334E0002332E07B68DB7E03F00F03DA
S31508014920DBB2032B0DD07B68DB7E03F00F03DBB212
S31508014930042B06D07B68DB7E03F00F03DBB2052B65
S3150801494001D101231BE0002319E07B68DB7E03F01C
S315080149500F03DBB2052B0DD07B68DB7E03F00F035B
S31508014960DBB2062B06D07B68DB7E03F00F03DBB2D6
S31508014970072B01D1012302E0002300E0002318469A
S315080149800C37BD465DF8047B704700BF80B584B01F
S3150801499000AF78600B46FB70FB781846FFF75EFFA1
S315080149A00346FB7397F90F30002B01DA00231EE04B
S315080149B097F90F30032B06DCFB7819467868FFF761
S315080149C065FF034613E07B68DA7E9B8B1B02134364
S315080149D0194697F90F30084A13441B7821FA03F34D
S315080149E003F00103002B14BF01230023DBB2184691
S315080149F01037BD4680BD00BF2048070880B586B080
S31508014A0000AF78600B46FB70FB781846FFF726FF68
S31508014A100346FB7597F91730002B01DA002331E0BD
S31508014A2097F91730194A13441B781A4601239340FC
S31508014A303B617B6893F83F20B3F840301B02134370
S31508014A401A463B691340002B14BF01230023FB734D
S31508014A507B6893F83F20B3F840301B0213431A468C
S31508014A603B69DB43134023F07F427B68D1B20020C8
S31508014A70014383F83F10120A92B200210A43A3F8B0
S31508014A804020FB7B18461837BD4680BD20480708DD
S31508014A9080B584B000AF78600B46FB70FB7818468A
S31508014AA0FFF7DCFE0346FB7397F90F30002B01DA9B
S31508014AB0002322E00E20FFF725FB03461A4697F945
S31508014AC00F3093420CBF01230023DBB2002B02D027
S31508014AD07B681B7E11E00F20FFF714FB03461A467D
S31508014AE097F90F3093420CBF01230023DBB2002B49
S31508014AF002D07B685B7E00E0002318461037BD466E
S31508014B0080BD80B483B000AF78600B46FB70FB783C
S31508014B107A6813441B7D18460C37BD465DF8047B3D
S31508014B20704780B586B000AFF8600B467A60FB72B5
S31508014B30FB7A012B40F2B5807B68002B00F0B1802F
S31508014B407B681B78012B0FD1FB6803F114007B6886
S31508014B50591CFB7A013BDBB2282B28BF2823DBB281
S31508014B601A4657F0B3FD17E07B681B78312B40F0E6
S31508014B70AE80FB7A022B40F2AC80FB6803F114008D
S31508014B807B68991CFB7A023BDBB2282B28BF2823BA
S31508014B90DBB21A4657F09AFDFB68DA7E9B8B1B023D
S31508014BA013431A46FB68DB6BC3F317039A4270D0AB
S31508014BB0FB68DA7E9B8B1B0213431A46FB68DB6B89
S31508014BC0C3F31703DB43134023F07F42FB68D1B2DB
S31508014BD00020014383F83F10120A92B200210A43CA
S31508014BE0A3F84020FB68DA7E9B8B1B021343194608
S31508014BF0FA68D36B61F31703D3630023FB750021AE
S31508014C00F868FFF743FE0346002B03D0FB7D43F00C
S31508014C100103FB750121F868FFF738FE0346002BEF
S31508014C2003D0FB7D43F00203FB750221F868FFF709
S31508014C302DFE0346002B03D0FB7D43F00403FB75D1
S31508014C400321F868FFF722FE0346002B03D0FB7DFC
S31508014C5043F00803FB75FB6893F84B30FA7D9A42DB
S31508014C6017D0FB6893F84B305BB2DB435AB297F91E
S31508014C70173013405BB203F00F03D9B2FA6892F802
S31508014C803F3061F3030382F83F30FB68FA7D83F80E
S31508014C904B20FB68B3F84C3001339AB2FB68A3F892
S31508014CA04C20FB6893F84A30002B07D1FB68DB7A66
S31508014CB0002B03D1FB68DB7C002B0BD0FB681B6840
S31508014CC01B68FA6842321146F868984702E000BF45
S31508014CD000E000BF1837BD4680BD80B584B000AF7F
S31508014CE078600023FB73FB7B032B08D8FB7B7A6870
S31508014CF013447F221A75FB7B0133FB73F3E77B6849
S31508014D000022DA7600229A837A68D36B6FF3170347
S31508014D10D3630023FB73FB7B012B08D8FB7B7A68E3
S31508014D20134400221A76FB7B0133FB73F3E7002356
S31508014D30FB73FB7B012B0CD8FB7B7A680C339B003E
S31508014D4013441A7942F080021A71FB7B0133FB7313
S31508014D50EFE77A68D37E082161F30303D3767A688D
S31508014D6092F83C30082161F3030382F83C307A68F3
S31508014D7092F83F306FF3030382F83F307B680022D5
S31508014D8083F84B207B6804331846FFF757FD7B6889
S31508014D900C331846FFF752FD7B68002283F843203F
S31508014DA07B6893F843207B6883F842207B6800225E
S31508014DB083F844207B68002283F845207B6800221B
S31508014DC083F846207B68002283F849207B6893F89C
S31508014DD049207B6883F848207B6893F848207B68DC
S31508014DE083F847207B68002283F84A2000BF1037E2
S31508014DF0BD4680BD80B483B000AF786039607B68FA
S31508014E001B78FC2B58D0FC2B5ADC262B22D0262BC0
S31508014E1056DC012B02D0022B0ED051E03B68012251
S31508014E201A703B6801337A6852781A703B68023304
S31508014E307A6892781A7050E03B6802221A703B68C9
S31508014E4001337A6852781A703B6802337A68927825
S31508014E501A7042E03B6826221A707B685A783B68CA
S31508014E600133D243D2B21A707B689B78002B03D0E8
S31508014E703B68023302221A703B6804337A68D27897
S31508014E801A703B6805337A6812791A703B680633DB
S31508014E907A6852791A707B689A793B68093352089D
S31508014EA0D2B21A703B6809331B78002B14D13B68C0
S31508014EB0093301221A700FE03B68FC221A700CE0D4
S31508014EC03B6800221A703B68013300221A703B685E
S31508014ED0023300221A7000E000BF7B680022DA71F3
S31508014EE000BF0C37BD465DF8047B704780B483B0BC
S31508014EF000AF7860064A7B681A607B6800225A60B0
S31508014F007B6818460C37BD465DF8047B704700BFC1
S31508014F102040070880B582B000AF78607B681846E4
S31508014F20FFF7E4FF054A7B681A607B684FF47A72DB
S31508014F309A607B6818460837BD4680BD3C48070815
S31508014F4080B500AF01221021024846F02DF900BFB5
S31508014F5080BD00BF0010024080B500AF00221021BD
S31508014F60024846F021F900BF80BD00BF001002408B
S31508014F7080B584B000AF78600B46FB70FFF7ECFF95
S31508014F80F91C4FF0FF33012209484AF0C5FF0023F7
S31508014F90FB7307F10F014FF0FF33012204484BF071
S31508014FA0F7F8FFF7CDFFFB7B18461037BD4680BDE6
S31508014FB0148F012080B584B000AF78600B46FB7072
S31508014FC01346BB70FFF7C8FFFB7843F00203DBB259
S31508014FD03B73BB787B7307F10C014FF0FF33022259
S31508014FE004484AF099FFFFF7ABFF00BF1037BD46EB
S31508014FF080BD00BF148F012080B500AF4FF400516A
S31508015000024846F0B9F80346184680BD0008024032
S3150801501080B582B000AF7860786801F0C5F97B6821
S31508015020184601F0DDF97B68002283F8B820054BA4
S3150801503011221A70786800F007F87B681846083755
S31508015040BD4680BD0912002080B483B000AF7860E8
S315080150507B68002283F8B82000BF0C37BD465DF88F
S31508015060047B704780B586B000AF78600B46FB704D
S315080150701346BB707B68FA781146184601F0EAF9BF
S31508015080F860FB68002B03D0FB681B68002B01D175
S31508015090002318E0FB681B687B610023FB74FB682F
S315080150A05B79FA7C9A420DD27B691B78BA789A4267
S315080150B001D17B6907E07B6903337B61FB7C0133A3
S315080150C0FB74ECE7002318461837BD4680BD80B54A
S315080150D086B000AFF8607B600B46FB721346BB7265
S315080150E07B68002B01D1D82315E0FB68FA7A1146B3
S315080150F0184601F0AFF978617B69002B01D1D623F7
S3150801510009E07B69FA7A1A717B697A681A607B69A0
S31508015110BA7A5A71002318461837BD4680BD80B53C
S3150801512086B000AFF8607B600B46FB721346BB7214
S31508015130FB68FA7A1146184601F08CF978617B69A1
S31508015140002B01D1D6234EE07B691B68002B01D1C8
S31508015150D72348E0BA7AFB7A1946F868FFF782FF3F
S3150801516002467B681A607B681B68002B01D1DB232A
S3150801517039E07B681B689B78C3F38503DBB20F2B89
S3150801518028BF0F23DBB21A46012393409AB23B6A22
S315080151901A803B6A1B88013B9AB23B6A1A80FB7AE2
S315080151A01A46E021F868FFF705FFD821F868FFF7E6
S315080151B0DFFE0346FB747B699B79002B09D0FB68EC
S315080151C093F8B820FB7C1343DBB243F00203DBB24E
S315080151D003E0FB7C23F00603DBB21A46D821F86804
S315080151E0FFF7E8FE002318461837BD4680BD90B57F
S315080151F08BB002AF7860084611461A460346FB7023
S315080152000B46BB7013467B700023FB760023FB60BD
S3150801521000237B8107F10C00BA78F97807F10A03B4
S31508015220009303467868FFF77AFF0346FB77FB7F0F
S31508015230002B01D0FB7FAEE07B7803F08003002BC7
S31508015240CCBF01230023FB767B783B7497F830307B
S315080152507B7497F83430BB7497F83830FB74BB8F7E
S31508015260BB82B7F84030FB8207F1100308222021E0
S31508015270786801F015F97B89BA781021786800F009
S31508015280FBFA0346FB77FB7F002B01D0FB7F82E00D
S31508015290BB6C002B72D0FB7E002B57D0B7F8403081
S315080152A0BB83FA68937843F002039370BB8B002B98
S315080152B05FD0B7F844303B81F9687A8907F108006D
S315080152C000230193BB6C00930346786800F0A6F8A7
S315080152D00346FB77FB7F062B14D1F8217868FFF785
S315080152E047FE034603F02003002B0CBF01230023CE
S315080152F0DBB2FA6803F00103D9B2937861F341038B
S315080153009370D3E7FB7F002B01D0FB7F43E0FB7F44
S31508015310002B11D1FB6C002B0ED0FB6C1B681C6893
S315080153203989B7F84020BB8BD31A9BB23B8307F167
S315080153301803BA6CF86CA0473B89BA8BD31ABB839E
S315080153403B89B7F844209A4212D8AFE7FA689378AE
S3150801535043F001039370F9687A89B7F84400BB6C86
S3150801536000930346786800F053F90346FB7700E09B
S3150801537000BFFB7F002B01D0FB7F0CE0FB7E002BDF
S3150801538001D0A02100E080217B89BA78786800F0F5
S3150801539073FA034600BF18462437BD4690BD80B54B
S315080153A08AB002AFF8607B600B46FB721346BB728C
S315080153B00023BB610023FB8207F11800BA7AF97A48
S315080153C007F1160300930346F868FFF7A8FE03469C
S315080153D0FB77FB7F002B10D0FB7F8121184601F05C
S315080153E08DF8FB7A8121184601F088F8BB7A81216C
S315080153F0184601F083F8FB7F0CE0B969FA8A97F839
S315080154002C300193BB6A00937B68F86800F006F8B4
S31508015410034600BF18462037BD4680BD80B586B015
S3150801542000AFF860B9603B601346FB800023FB754B
S315080154303B681B887B82BB685B787B743B68002270
S315080154401A80BB689B7803F00203DBB2002B01D0FC
S31508015450202300E010231A46E821F868FFF7AAFD81
S31508015460BB681A78FB880021F86800F005FA03463C
S31508015470FB75FB7D062B23D1F821F868FFF778FD2C
S31508015480034603F01003002B0CBF01230023DBB2F4
S3150801549003F00103D9B2BA68937861F341039370B3
S315080154A0BB689B7803F00203DBB2002B01D02023F3
S315080154B000E010231A46E821F868FFF77BFD6EE045
S315080154C0FB7D002B6CD1C821F868FFF751FD034617
S315080154D003F00403002B0CBF01230023DBB2002BCE
S315080154E002D0F023FB755CE03021F868FFF740FD38
S315080154F00346BB75BA7D7B8A9A4201DD7B8ABB75F9
S315080155003B68B3F900309BB27A8AD31A9BB2BB8245
S31508015510B7F91430002B01DA0023BB82BA7DB7F93B
S3150801552014309342A8BF1346DAB23B6A0821F868D9
S3150801553000F0F0FF38620422C821F868FFF73AFD47
S315080155403B681A88BB7D9BB213449AB23B681A80A2
S31508015550BA7D7B7C9A4204D33B681B887A8A9A4235
S3150801556013D8F821F868FFF703FD034603F0100383
S31508015570002B01D0012100E00021BA68937861F37C
S31508015580410393700023FB750BE097F82430002B39
S315080155903FF466AF97F82430184644F01DF85FE7E4
S315080155A000BFFB7D18461837BD4680BD80B588B05B
S315080155B002AF7860084611461A460346FB700B4649
S315080155C0BB7013463B8000233B610023FB8107F137
S315080155D01000BA78F97807F10E0300930346786844
S315080155E0FFF79DFD0346FB75FB7D002B01D0FB7D77
S315080155F00AE03969FA8938883B6A0093034678686C
S3150801560000F006F8034600BF18461837BD4680BDA8
S3150801561080B58AB000AFF860B96011461A460B46E4
S31508015620FB801346BB80002387F827303B6B3B6220
S31508015630BB88BB83BB685B78FB76FB7E002B02D0FD
S31508015640FB7E402B01D9DA2312E143F0B9FF034669
S3150801565003F59C5308337B61BB689B7803F0010310
S31508015660DBB2002B01D0802300E040231A46E82153
S31508015670F868FFF79FFCBB8B002B00F0DA8000234C
S3150801568087F826300023FB83FB7E9BB2BA8B9342B5
S3150801569028BF13467B827B8ADAB23B6A1021F868F7
S315080156A000F0FEFE7B8ADBB21A463821F868FFF75E
S315080156B081FCBB681B7843F02003DBB21A46F02154
S315080156C0F868FFF777FCC821F868FFF751FC03462D
S315080156D05BB2DB43DBB2DB09DBB2002B00D0F2E7BE
S315080156E08022C821F868FFF765FCF821F868FFF7FA
S315080156F03FFC034603F00F0387F8273097F8273056
S31508015700002B08D043F05CFF02467B69D31A002BB5
S3150801571001DA012300E00023002B00F0818097F8CD
S3150801572027300E2B12D00E2B00F38580042B02D0C6
S31508015730062B15D07FE0FB8B0133FB83FB88002BFF
S3150801574032D0FA8BFB889A422ED175E097F826302B
S31508015750013387F8263097F82630032B26D16BE0DC
S31508015760F821F868FFF704FC034603F02003002B31
S315080157700CBF01230023DBB203F00103D9B2BA68D7
S31508015780937861F300039370BB689B7803F0010378
S31508015790DBB2002B01D0802300E040231A46E82122
S315080157A0F868FFF707FC02E000BF00E000BF00222F
S315080157B03821F868FFF7FEFB3B6A1B781A46102169
S315080157C0F868FFF7F7FB7B8ADBB21A463821F868D7
S315080157D0FFF7F0FBBB681B7843F02003DBB21A46E0
S315080157E0F021F868FFF7E6FBC821F868FFF7C0FB68
S315080157F003465BB2DB43DBB2DB09DBB2002B00D02D
S31508015800F2E78022C821F868FFF7D4FBF821F86887
S31508015810FFF7AEFB034603F00F0387F827306DE762
S31508015820BA8B7B8AD31ABB837B8A3A6A13443B6257
S3150801583021E700BF00E000BF97F82730002B04D00E
S3150801584000223821F868FFF7B5FBF821F868FFF759
S315080158508FFB034603F02003002B01D0012100E052
S315080158600021BA68937861F30003937097F827309B
S3150801587018462837BD4680BD80B586B000AF78602A
S31508015880084611461A460346FB700B46BB7013467B
S315080158903B8043F095FE034603F59C5308333B6171
S315080158A00023FB750023BB750023BB8243F088FEEA
S315080158B002463B69D31ADB0FDBB2002B4CD0FA78D0
S315080158C0BB781343DBB21A46F0217868FFF772FBFF
S315080158D0FF23FB7543F074FE02463B69D31ADB0FBF
S315080158E0DBB2002B10D0C8217868FFF741FB0346CD
S315080158F0FB7397F90F30002BECDA8022C821786800
S31508015900FFF758FB0023FB75F8217868FFF730FB92
S31508015910034603F00F03FB75FB7D042B02D00E2B08
S315080159200CD013E0BB8A0133BB823B88002B0FD016
S31508015930BA8A3B889A420BD1FB7D0EE0BB7D0133C7
S31508015940BB75BB7D032B05D1FB7D06E0FB7D04E022
S3150801595000BFABE700BFA9E7FB7D18461837BD4670
S3150801596080BD000080B584B000AF78600023FB736A
S31508015970786800F0FDFD786800F012FE03463B7377
S315080159803B7B032B2ED801A252F823F0A959010813
S315080159909D590108C5590108C1590108BF4B132270
S315080159A01A700023FB731DE0BC4B1B7803F0F00350
S315080159B0102B02D0B94B11221A700023FB7311E088
S315080159C00123FB73B54B1B7803F0F003102B08D1A9
S315080159D043F0F6FD0346C833B14A1360AF4B2022A4
S315080159E01A7000BF0023BB73BB7B0F2B1BD8BA7B76
S315080159F07B681E3253F82230002B10D0BA7B7B68A5
S31508015A001E3253F82210BA7B7B681E3253F82230B5
S31508015A101B680C331B68084698470346FB72BB7B19
S31508015A200133BB73E0E79D4B1B78A02B00F0238164
S31508015A30A02B00F32F81902B00F01F81902B00F3F0
S31508015A402981802B00F0FE80802B00F32381512BC6
S31508015A5000F0EA80512B00F31D81402B6ADC112BE3
S31508015A60C0F21881113B2F2B00F2148101A252F8C2
S31508015A7023F000BF3B5B01087F5C01087F5C0108DE
S31508015A80955C0108955C0108955C0108955C01081F
S31508015A90955C0108955C0108955C0108955C01080F
S31508015AA0955C0108955C0108955C0108955C0108FF
S31508015AB08B5B0108955C0108955C0108955C0108FA
S31508015AC0955C0108955C0108955C0108955C0108DF
S31508015AD0955C0108955C0108955C0108955C0108CF
S31508015AE0955C0108955C0108955C0108955C0108BF
S31508015AF0A75B0108955C0108955C0108955C01089E
S31508015B00955C0108955C0108955C0108955C01089E
S31508015B10955C0108955C0108955C0108955C01088E
S31508015B20955C0108955C0108955C0108955C01087E
S31508015B30B95B0108502B5FD0ACE07868FFF784FAAF
S31508015B4000237B737B7B0F2B1BD87A7B7B681E32EA
S31508015B5053F82230002B10D07A7B7B681E3253F81B
S31508015B6022107A7B7B681E3253F822301B68083371
S31508015B701B68084698470346FB727B7B01337B7398
S31508015B80E0E7464B12221A7084E043F019FD0246FB
S31508015B90434B1B68D31ADB43DB0FDBB2002B70D0F8
S31508015BA03E4B30221A700122E8217868FFF702FA83
S31508015BB03A4B40221A706DE0E8217868FFF7D8F968
S31508015BC0034603F00103002B0CBF01230023DBB2BC
S31508015BD0002B58D0D8217868FFF7CAF9034643F055
S31508015BE008033B733B7B1A46D8217868FFF7E2F92D
S31508015BF02A4B50221A7046E0C8217868FFF7B8F98F
S31508015C00034603F04003002B14BF01230023DBB234
S31508015C10002B3AD0214B51221A7043F0D1FC03468E
S31508015C2014331F4A136030E043F0CAFC02461C4B8A
S31508015C301B68D31ADB43DB0FDBB2002B27D0174BCC
S31508015C4080221A70FB7B00220021786800F020F977
S31508015C500346FB72FB7A002B09D0FB7AD22B18D0AC
S31508015C60104AFB7A13700D4BA0221A7011E00B4BE8
S31508015C7090221A700DE000BF0CE000BF0AE000BFD9
S31508015C8008E000BF06E000BF04E000BF02E000BF75
S31508015C9000E000BF00BF1037BD4680BD09120020D5
S31508015CA00C1200200812002080B586B000AF78607B
S31508015CB0084611461A460346FB700B46BB70134647
S31508015CC07B7000237B6100233B617B6800211846BA
S31508015CD000F0C0FB78617B69002B01D1D6233AE03D
S31508015CE07B691B68002B01D1D72334E07B697A785D
S31508015CF09A717868BB78F978002200F05FFC034650
S31508015D00FB73FB7B002B01D1D42324E07B68FA7B50
S31508015D101146184600F09EFB38613B69002B01D1FC
S31508015D20D62318E03B697A789A71FB7B0022002119
S31508015D30786800F0E3FA0346BB73BB7B002B09D0F6
S31508015D407B68FA7B1146184600F0D0FC0023FB73EA
S31508015D50BB7B00E0002318461837BD4680BD90B5C9
S31508015D6085B000AF7860084611461A460346FB70AF
S31508015D700B46BB7013467B700023FB73FA787B686E
S31508015D801E3253F82200FA787B681E3253F8223005
S31508015D901B6804331C6897F820307A78B978A047CD
S31508015DA00346BB73BB7BE02B1CD1BB78002B08D108
S31508015DB00122E8217868FFF7FDF8662043F00CFC1C
S31508015DC022E0BA787B681E3253F82200BA787B68DB
S31508015DD01E3253F822301B6814331B687A78114631
S31508015DE0984711E0BB7B0D2B09D1FB7B022B06D80B
S31508015DF0642043F0F1FBFB7B0133FB73BEE7BB7BFE
S31508015E00002B01D0BB7B3FE0FA787B681E3253F842
S31508015E102200FA787B681E3253F822301B681C6808
S31508015E2097F820307A78B978A0470346BB73BB7BCD
S31508015E300D2B09D1FB7B022B06D8642043F0CCFB42
S31508015E40FB7B0133FB7399E7BB7B002B1BD0BB782C
S31508015E50002B08D10122E8217868FFF7ABF8662004
S31508015E6043F0BAFB0FE0BA787B681E3253F822007A
S31508015E70BA787B681E3253F822301B6814331B68C4
S31508015E807A7811469847BB7B18461437BD4690BDAC
S31508015E9080B590B002AF7860084611461A460346A7
S31508015EA0FB700B46BB7013467B70002387F83630B0
S31508015EB007F10C033B630023FB620023BB6200234B
S31508015EC03B7208237B72BB7A6FF30003BB72BB7A02
S31508015ED06FF34103BB72BB7A0F2262F38703BB726E
S31508015EE07868F9F7F8FF78627B6A1B681B680021F6
S31508015EF0786A9847F862FB6A002B01D1D6235CE1E0
S31508015F00FB6A1B68BB62FB6A07F108021A60FB6A37
S31508015F107A789A7107F10C03009312230022002163
S31508015F20786800F04EF9034687F83630FB6ABA6A94
S31508015F301A6097F83630002B02D097F836303CE1D4
S31508015F403B6B1A7A5B7A1B0213437B843B6B9A7A07
S31508015F50DB7A1B0213433B843B6B1B79FB773B6B59
S31508015F605B79BB77002387F8373097F837300F2BE3
S31508015F7000F2818097F837207B681E3253F8223069
S31508015F80002B6ED097F837207B681E3253F8221003
S31508015F9097F837207B681E3253F822301B68103376
S31508015FA01B68084698470346002B14BF01230023A4
S31508015FB0DBB2002B57D197F837207B681E3253F88E
S31508015FC0220097F837207B681E3253F822301B6867
S31508015FD020331B68BA7F114698470346002B2BD0FE
S31508015FE097F837207B681E3253F8220097F8372036
S31508015FF07B681E3253F822301B6818331B683A8CAB
S31508016000798C98470346002B14D197F837207B687B
S315080160101E3253F8220097F837207B681E3253F850
S3150801602022301B681C331B68FA7F114698470346C2
S31508016030002B01D0012300E00023002B14D0B878EF
S31508016040FA7897F837107B78009303467868FFF754
S3150801605086FE034687F8363097F83630D12B09D1B4
S3150801606002E000BF00E000BF97F83730013387F838
S3150801607037307AE700BF97F837300F2B02D897F8F1
S3150801608036309AE0002387F8373097F837300F2BE8
S3150801609000F2888097F837207B681E3253F8223041
S315080160A0002B74D097F837207B681E3253F82210DC
S315080160B097F837207B681E3253F822301B68103355
S315080160C01B68084698470346002B14BF0123002383
S315080160D0DBB2002B5DD197F837207B681E3253F867
S315080160E0220097F837207B681E3253F822301B6846
S315080160F020331B68BA7F114698470346002B2BD0DD
S3150801610097F837207B681E3253F8220097F8372014
S315080161107B681E3253F822301B6818331B683A8C89
S31508016120798C98470346002B14D197F837207B685A
S315080161301E3253F8220097F837207B681E3253F82F
S3150801614022301B681C331B68FA7F114698470346A1
S31508016150002B01D0012300E00023002B1BD1B878C6
S31508016160FA7897F837107B78009303467868FFF733
S31508016170F6FD034687F8363097F83630D12B0BD023
S3150801618097F83630D92B07D097F8363015E000BF87
S3150801619002E000BF00E000BF97F83730013387F807
S315080161A0373072E77B78BA78F9787868FFF77CFD3B
S315080161B0034687F8363097F8363018463837BD46DD
S315080161C080BD80B58AB008AF7860084611461A4680
S315080161D00346FB700B46BB7013463B80BA78F978C9
S315080161E0002307933B6906933B8805933B880493F1
S315080161F000230393012302930023019306230093AB
S3150801620080237868FEF7F3FF034618460837BD462C
S3150801621080BD80B58AB008AF7860084611461A462F
S315080162200346FB700B46BB7013463B80BA78F97878
S31508016230002307937B6906933B8805933B88049360
S3150801624000230393022302933B7C019306230093C5
S3150801625080237868FEF7CBFF034618460837BD4604
S3150801626080BD80B59EB008AF7860084611461A46CB
S315080162700346FB700B46BB7013467B70402387F8B9
S31508016280573007F10C033B65BA78F97807F10C0327
S3150801629001937B78009309237868FFF7BAFF0346D1
S315080162A087F84F3097F84F30002B02D097F84F30C8
S315080162B020E03B6D9A78DB781B021343A7F84C3034
S315080162C0BA78F9783B6E079307F10C0306934023D6
S315080162D00593B7F84C3004930023039302230293E2
S315080162E07B7801930623009380237868FEF77FFF66
S315080162F0034600BF18465837BD4680BD80B58CB0E9
S3150801630008AF7860084611461A460346FB700B46E5
S31508016310BB7013467B70BA78F9780023079300237C
S315080163200693002305930023049300230393002374
S3150801633002937B7801930523009300237868FEF77F
S3150801634056FF0346FB734FF4967043F045F9FB7B02
S3150801635018461037BD4680BD80B58AB008AF78604B
S31508016360084611461A460346FB700B46BB70134690
S315080163707B70BA78F97800230793002306930023E4
S3150801638005930023049300230393002302937B7848
S3150801639001930923009300237868FEF728FF034633
S315080163A018460837BD4680BD80B483B000AF786013
S315080163B07B6818460C37BD465DF8047B70470000BC
S315080163C080B483B000AF7860044A7B681A607B6842
S315080163D018460C37BD465DF8047B704770480708B8
S315080163E080B582B000AF78607B681846FFF7E8FF92
S315080163F0174A7B681A607B680022DA71002178687F
S3150801640000F090F97B6800221A737B681A1D7B6875
S315080164109A607B6800221A717B6808225A717A6829
S3150801642093796FF3000393717A6893796FF3410354
S3150801643093717A6893790F2161F387039371786869
S3150801644000F0A1F97B6818460837BD4680BD00BF34
S315080164505C48070880B584B000AF78600B46FB70CE
S31508016460FB78002B02D17B68083314E0FB781946C8
S31508016470786800F0A1F90346FB73FB7B002B08D073
S315080164807B6803F10801FA7B1346DB009B1A0B4470
S3150801649000E0002300BF18461037BD4680BD000046
S315080164A080B586B000AFF8607B600B46FB72134679
S315080164B0BB72FEF751FDFB7A43F00203DBB2FB75B3
S315080164C007F117014FF0FF3301220B4849F024FD6C
S315080164D0BB7A9AB24FF0FF337968074849F01CFD39
S315080164E0BB7A7A6813447B60FEF72AFD7B681846F7
S315080164F01837BD4680BD00BF148F012080B483B014
S3150801650000AF03463960FB7100BF0C37BD465DF825
S31508016510047B704780B584B000AFF8607B600B469A
S31508016520FB721346BB72FEF717FD07F10B014FF01D
S31508016530FF3301220D4849F0EFFCBB7A1A460021C8
S31508016540786856F0EBF8BB7A9AB24FF0FF33796860
S31508016550064849F01DFEBB7A7A6813447B60FEF74C
S31508016560EFFC7B6818461037BD4680BD148F0120A5
S3150801657080B584B000AF78600023FB73FEF73CFD5D
S315080165800346BB73BB7B002B04D1786800F037F94F
S315080165900346FB73FB7B18461037BD4680BD0000DA
S315080165A080B483B000AF7860034B1B7818460C376C
S315080165B0BD465DF8047B70471012002080B584B093
S315080165C000AF7860084611461A460346FB700B462B
S315080165D0BB7013467B70FB783B733B7B23F07F03D1
S315080165E0DBB2002B02D17B78072B01D9002379E096
S315080165F0BB78002B05D07B68DB79072B01D10023FB
S3150801660070E00021786800F0D7F80346FB73FB7B3E
S31508016610002B01D1002365E03B7B002B24D1BB78FD
S31508016620002B0FD0FA7B79681346DB009B1A0B44C3
S315080166300C3341221A707B68DB790133DAB27B6845
S31508016640DA7108E0FA7B79681346DB009B1A0B447A
S315080166500C3301221A70FA7B79681346DB009B1A00
S315080166600B440C331B783DE000233B723B7BC3F3A1
S315080166700203DAB23B7A62F3C5033B72BB78002B9D
S3150801668013D03B7A43F040033B727B68DB790133D5
S31508016690DAB27B68DA717B68DB7903F00703DAB271
S315080166A03B7A62F302033B720BE03B7A6FF3861384
S315080166B03B727B7803F00703DAB23B7A62F3020393
S315080166C03B72FA7B79681346DB009B1A0B440C3341
S315080166D03A7A1A70FA7B79681346DB009B1A0B44DF
S315080166E00C331B7818461037BD4680BD80B584B07B
S315080166F000AF78600B46FB70FB78412B03D17868B5
S3150801670000F041F80BE0FB781946786800F054F878
S315080167100346FB73FB7B1946786800F093F810373C
S31508016720BD4680BD80B483B000AF78600B46FB7070
S31508016730FA7879681346DB009B1A0B440C3300225E
S315080167401A70FA7879681346DB009B1A0B440D33E5
S3150801675001221A70FA7879681346DB009B1A0B44F2
S315080167600E3300221A70FA787B68191D7868134669
S31508016770DB009B1A03440833196000BF0C37BD467A
S315080167805DF8047B704780B584B000AF786001235B
S31508016790FB73FB7B0F2B08D8FB7B19467868FFF741
S315080167A0C1FFFB7B0133FB73F3E77B680022DA71D8
S315080167B000BF1037BD4680BD80B485B000AF786094
S315080167C00B46FB700123FB73FB7B0F2B10D8FA7B5F
S315080167D079681346DB009B1A0B440C331B78FA784D
S315080167E09A4201D1FB7B04E0FB7B0133FB73EBE7A8
S315080167F0002318461437BD465DF8047B704780B5FB
S3150801680084B000AF78600023FB73C8217868FEF76F
S31508016810AFFB0346BB73BB7B03F02003002B06D0FB
S31508016820786800F057F8FB7B43F02003FB73FB7B8A
S315080168301A46C8217868FEF7BDFBFB7B1846103758
S31508016840BD4680BD80B584B000AF78600B46FB704D
S31508016850FB78002B3AD0FA7879681346DB009B1A45
S315080168600B440C331B783B733B7B03F04003DBB2D1
S31508016870002B25D00123FB73FB7B1A46397B7868ED
S3150801688000F098F80346FB73FB7B002B14BF01232A
S315080168900023DBB2002B05D0FB7B19467868FFF78E
S315080168A0D1FFE9E77B68DB793A7BC2F30202D2B210
S315080168B0934205D17B68DB79013BDAB27B68DA71F1
S315080168C0FB7819467868FFF72DFF00E000BF1037FF
S315080168D0BD4680BD80B584B000AF7860F821786880
S315080168E0FEF746FB0346FB73FB7B23F03F03FB7373
S315080168F0FB7BC02B4AD0C02B55DC802B06D0802BC6
S3150801690051DC002B46D0402B20D04CE0D8217868AA
S31508016910FEF72EFB034603F00203002B0CBF0123EF
S315080169200023DBB2002B08D0C922D8217868FEF7EC
S3150801693041FB1F4B02221A7035E0CB22D821786819
S31508016940FEF738FB1A4B03221A702CE0D821786817
S31508016950FEF70EFB034603F00203002B0CBF0123CF
S315080169600023DBB2002B08D0CB22D8217868FEF7AA
S3150801697021FB0F4B03221A7015E0C922D82178682A
S31508016980FEF718FB0A4B02221A700CE0084B01228B
S315080169901A7008E0D122D8217868FEF70BFB044B60
S315080169A000221A7000BF00BF1037BD4680BD00BF68
S315080169B01012002080B485B000AF78603970134694
S315080169C0FB70FB78002B04D0FB780F2B01D8FB78E2
S315080169D000E00123FB73FB7B0F2B16D8FA7B796842
S315080169E01346DB009B1A0B4408331B79C3F3C20316
S315080169F0DAB23B78C3F30203DBB29A4201D1FB7BDD
S31508016A0004E0FB7B0133FB73E5E7002318461437E3
S31508016A10BD465DF8047B704780B485B000AFF86069
S31508016A20B9607A60FB681B68002B01D1002331E04D
S31508016A30FB681B79002B22D07B681B88002B1ED094
S31508016A40BB681A68FB681B68F96849790846F968DA
S31508016A500979411A0B4412781A70FB681B79013BB4
S31508016A60DAB2FB681A717B681B88013B9AB27B68AC
S31508016A701A80BB681B685A1CBB681A60D8E7FB6892
S31508016A801B79002B01D0002304E0FB685A79FB68C7
S31508016A901A71012318461437BD465DF8047B704701
S31508016AA080B584B000AF786046F0E8FE03460B4A2D
S31508016AB0A2FB03231B0DBB607B68BA6802FB03F3C9
S31508016AC00A3BFB6000BFFB685A1EFA60002BFAD12D
S31508016AD000BF00BF1037BD4680BD00BF83DE1B4324
S31508016AE080B582B000AF0346FB80FB88184642F0AA
S31508016AF073FD00BF0837BD4680BD80B500AF0A20CB
S31508016B00FFF7CEFF00BF80BD80B584B000AFF86047
S31508016B107B600B46FB7213463B81FB7A082B78D8C0
S31508016B2001A252F823F000BF136C01084D6B01084E
S31508016B30756B0108936B0108B56B0108D76B0108E2
S31508016B40EB6B0108EB6B0108FD6B010800221021B4
S31508016B50324844F029FB0220FFF7C2FF0122102127
S31508016B602E4844F021FB01224FF400412C4844F001
S31508016B701BFB4EE03B89002B05D10022202127482B
S31508016B8044F012FB45E001222021244844F00CFB85
S31508016B903FE03B89002B06D101224FF400412048F2
S31508016BA044F002FB35E000224FF400411C4844F052
S31508016BB0FBFA2EE03B89002B05D10022102117484C
S31508016BC044F0F2FA04E001221021144844F0ECFAE8
S31508016BD0FFF793FF1DE0134B186807F108014FF4FF
S31508016BE07A73012249F098F913E00E4B18683A892D
S31508016BF04FF47A73796849F08FF90AE0094B1B68F3
S31508016C003A897968184649F077FD012042F0E4FC93
S31508016C1000BF012318461037BD4680BD0004024057
S31508016C20000002401412002080B582B000AF7860DF
S31508016C300A4A7B68136001224FF40041084844F070
S31508016C40B3FA0A2042F0C8FC064A0749074801F088
S31508016C5098F900BF0837BD4680BD00BF1412002051
S31508016C6000000240096B010830000020B48C0120A5
S31508016C7080B588B002AFF860084611461A46034641
S31508016C807B810B463B811346FB807B8907337B81DE
S31508016C9011E03B6A1B783A89798900930223F868DF
S31508016CA001F006FA3B6A01333B62FB88083BFB802D
S31508016CB07B8908337B81FB88072BEAD8FB88002B65
S31508016CC01CD03B6A1B78FB757B89073B7B81FB7D67
S31508016CD003F00103002B05D03A897B891946F86828
S31508016CE001F0D3F97B8901337B81FB88013BFB806A
S31508016CF0FB7D5B08FB75FB88002BE8D100BF1837C5
S31508016D00BD4680BD80B588B002AFF8600846114619
S31508016D101A4603467B810B463B811346FB80FB885B
S31508016D20FB82FB8A0733FB82FB8ADB08FB82F88836
S31508016D303A8979893B8C00930346F86800F01FF875
S31508016D400346002B17D012E0F8883A8979897B6ABD
S31508016D5000930346F868FFF78BFFFB8A7A6A1344A8
S31508016D607B623B8901333B813B8C013B3B843B8CFA
S31508016D70002BE9D100E000BF1837BD4680BD90B4AD
S31508016D8088B000AFF860084611461A4603467B816B
S31508016D900B463B811346FB803C893B8D23449CB2C1
S31508016DA02346013B9CB2FB68DA8FFB68B3F8423095
S31508016DB0FA83BB833B897B8323463B83BA8B7B8BD5
S31508016DC09A420DD3FA8B3B8B9A4201D8012314E0E0
S31508016DD07A8B3B8B9A4201D901230EE000230CE002
S31508016DE0FA8B3B8B9A4207D87A8B3B8B9A4201D90D
S31508016DF0012302E0002300E00023002B01D1002338
S31508016E0031E07C89FB8823449CB22346013B9CB232
S31508016E10FB689A8FFB68B3F84030FA82BB827B899C
S31508016E207B8223463B82BA8A7B8A9A420DD3FA8AA7
S31508016E303B8A9A4201D8012314E07A8A3B8A9A420C
S31508016E4001D901230EE000230CE0FA8A3B8A9A4213
S31508016E5007D87A8A3B8A9A4201D9012302E000239C
S31508016E6000E0002300BF18462037BD4690BC704796
S31508016E7090B585B000AFF860B9601346FB71BB6881
S31508016E809C68FB799AB200230121F868A04703465A
S31508016E9018461437BD4690BD90B585B000AFF86069
S31508016EA0B9601346FB71BB689C68FB799AB20023EB
S31508016EB00321F868A04700BF1437BD4690BD90B5B9
S31508016EC083B000AF786039603B689C680023002274
S31508016ED004217868A04700BF0C37BD4690BD90B520
S31508016EE083B000AF786039603B689C680023012253
S31508016EF004217868A04700BF0C37BD4690BD90B500
S31508016F0085B000AFF860B9601346FB71BB689C6831
S31508016F10FB799AB200230221F868A04700BF14370B
S31508016F20BD4690BD90B585B000AFF860B96013460F
S31508016F30FB71BB689C68FB799AB200230521F86846
S31508016F40A047034618461437BD4690BD80B586B09E
S31508016F5000AFF860B9607A600023FB757B681B781F
S31508016F60BB75FB7D002B10D1BB7DFF2B0AD0BB7DEA
S31508016F701A46B968F868FFF7D5FF0346002B60D1B2
S31508016F80002364E00123FB755BE0BB7DFF2B0AD17F
S31508016F90BB7D1A46B968F868FFF7C4FF0346002B9C
S31508016FA04DD1002353E0BB7DFE2B4ED0BB7DEF2B8D
S31508016FB045D8BB7DDF2B09D9BB7D03F00F03DBB2B7
S31508016FC01A46B968F868FFF79AFF38E0BB7DCF2BF8
S31508016FD009D9BB7D03F00F03DBB21A46B968F86815
S31508016FE0FFF75AFF2BE0BB7DBF2B1CD9B968F868A0
S31508016FF0FFF765FFBB7D03F00F03BB75BB7D1B0167
S31508017000BB75BB7D0233BB75BB7D9BB21846FFF7CB
S3150801701067FDB968F868FFF762FFBB7D9BB2184642
S31508017020FFF75EFD0BE0BB7DBD2B08D897F916303F
S31508017030002B04DBBB7D9BB21846FFF751FD0023ED
S31508017040FB757B6801337B6088E700BF012318461F
S315080170501837BD4680BD000090B587B000AFF8600F
S31508017060B9603B601346FB800023FB823B685A1CD0
S315080170703A601B787B757B7D3B753B7D03F00F037F
S315080170803B757B7D1B097B753A7DFB8A591CF98209
S315080170901946104B9A5C104B5A547A7DFB8A591C37
S315080170A0F98219460B4B9A5C0B4B5A54FB88013BE8
S315080170B0FB80FB88002BD9D1BB689C68074B1A88D3
S315080170C0054B0821F868A047012318461C37BD4619
S315080170D090BD00BF00000020181200207C48070858
S315080170E090B587B000AFF860B9603B601346FB7195
S315080170F00023FB753B685A1C3A601B78BB75BB7D40
S315080171007B757B7D03F00F037B75BB7D1B09BB7507
S315080171107A7DFB7D591CF97519460F4B9A5C0F4B05
S315080171205A54BA7DFB7D591CF97519460A4B9A5C66
S315080171300A4B5A54FB79013BFB71FB79002BD9D1D8
S31508017140BB689C68054B80220621F868A047012385
S3150801715018461C37BD4690BD1000002018160020A1
S3150801716080B485B000AFF8607B600B46FB721346AE
S31508017170BB72FB7A062B11D801A252F823F000BF85
S315080171809D7101089D7101089D7101089D71010894
S315080171909D7101089D7101089D7101080123184619
S315080171A01437BD465DF8047B704700BF80B586B0CD
S315080171B000AFF860B9601346FB71BB685B681B7A60
S315080171C0FB75BB685B681B88DBB2FA7D12FB03F3B0
S315080171D0FB75FA7DFB791344FB75134AB968F868A0
S315080171E0FFF7B4FEFB7D1A46B968F868FFF79AFE01
S315080171F0FB7D0133DBB21A46B968F868FFF792FEE0
S315080172000022B968F868FFF77AFE5C22B968F8685F
S31508017210FFF788FE0122B968F868FFF770FE00BF1C
S315080172201837BD4680BD00BF0049070880B586B03E
S3150801723000AFF860B9601346FB71BB685B681B7ADF
S31508017240FB75BB685B681B88DBB2FA7D12FB03F32F
S31508017250FB75FA7DFB791344FB75134AB968F8681F
S31508017260FFF774FEFB7D1A46B968F868FFF75AFE00
S31508017270FB7D0833DBB21A46B968F868FFF752FE98
S315080172800022B968F868FFF73AFE5C22B968F8681F
S31508017290FFF748FE0122B968F868FFF730FE00BF1C
S315080172A01837BD4680BD00BF0049070880B58CB0B8
S315080172B000AFF860B9603B601346FB71FB790A3B86
S315080172C00C2B00F2C08001A252F823F001730108C9
S315080172D0477401084774010847740108477401088F
S315080172E0E57301082B74010839740108477401080C
S315080172F04774010847740108177301087F73010869
S315080173000222B968F868FFF7B3FD544AB968F86804
S31508017310FFF71CFE97E0BB685B687B617B69DB68EE
S31508017320BB627B695B897B827B8A9B087B820023A4
S3150801733087F82F301BE097F82F301A46B968F86896
S31508017340FFF734FF7B8ADAB2BB6AB968F868FFF7D8
S31508017350C7FE0022B968F868FFF79EFD7B8ABA6AFC
S315080173601344BB6297F82F30013387F82F3097F80B
S315080173702F309AB27B691B889A42DCD363E0BB68DB
S315080173805B68FB61FB69DB683B62FB695B897B8345
S315080173907B8B5B007B83002387F827301AE097F8FD
S315080173A027301A46B968F868FFF740FF7A8B3B6AB7
S315080173B0B968F868FFF750FE0022B968F868FFF760
S315080173C06BFD7B8B3A6A13443B6297F82730083387
S315080173D087F8273097F827309AB2FB691B889A42B3
S315080173E0DDD330E00122B968F868FFF755FD0022C0
S315080173F0B968F868FFF783FDC122B968F868FFF72D
S3150801740091FD0122B968F868FFF779FD3B681B7899
S315080174105B08DBB21A46B968F868FFF783FD0022F4
S31508017420B968F868FFF738FD0DE00D4AB968F868DC
S31508017430FFF78CFD01230DE00A4AB968F868FFF7E2
S3150801744085FD012306E0FA793B68B968F86801F019
S31508017450A9F8034618463037BD4680BD8048070857
S31508017460104907081C49070880B483B000AF786043
S315080174700B46FB70FB787A6813447B607B681B7844
S3150801748018460C37BD465DF8047B704780B485B055
S3150801749000AF78600B46FB70FB787A6813447B6013
S315080174A07B681B78FB817B6801337B60FB891B0248
S315080174B0FB817B681B789AB2FB891344FB81FB89A4
S315080174C018461437BD465DF8047B704780B582B00F
S315080174D000AF786000217868FFF7C6FF03461846B3
S315080174E00837BD4680BD80B582B000AF7860786840
S315080174F0FFF7ECFF0346022B0AD0022B0ADC002B0E
S3150801750002D0012B02D005E0062304E0032302E0A2
S31508017510062300E0032318460837BD4680BD80B51B
S3150801752082B000AF786005217868FFF79DFF0346B2
S3150801753018460837BD4680BD80B582B000AF786071
S3150801754006217868FFF7A2FF034618460837BD46A5
S3150801755080BD80B582B000AF786008217868FFF7F2
S3150801756095FF034618460837BD4680BD80B582B0EB
S3150801757000AF78600A217868FFF776FF0346184658
S315080175800837BD4680BD80B582B000AF78600B2153
S315080175907868FFF769FF034618460837BD4680BD78
S315080175A080B582B000AF78600C217868FFF75CFF80
S315080175B003465BB218460837BD4680BD80B582B022
S315080175C000AF78600D217868FFF74EFF03465BB27E
S315080175D018460837BD4680BD80B582B000AF7860D1
S315080175E00E217868FFF740FF03465BB21846083755
S315080175F0BD4680BD80B582B000AF78600F2178683E
S31508017600FFF732FF03465BB218460837BD4680BD11
S3150801761080B582B000AF786010217868FFF724FF43
S3150801762003465BB218460837BD4680BD80B582B0B1
S3150801763000AF786039607868FFF755FF03461A4648
S315080176403B68134418460837BD4680BD80B584B0EB
S3150801765000AF786039607B689B681846FFF736FF8C
S315080176600346002B01D0022B1BD13B681A787B6895
S31508017670DA773B685A787B6883F820203B680333BE
S315080176801B785AB27B681A773B6804331B785AB25F
S315080176907B685A773B6805331B785AB27B689A77B9
S315080176A034E03B681B78FB7397F90F3003F00F033F
S315080176B05AB27B689A777B6893F91E30DBB2023B34
S315080176C0DBB25AB27B689A77FB7B1B09FB7397F986
S315080176D00F207B685A773B685B78FB73FB7B03F06B
S315080176E00F03DAB27B6883F82020FB7B1B09FB7347
S315080176F07B68FA7BDA773B689B78FB73FB7B1B0914
S31508017700FB7397F90F207B681A7700BF00BF103704
S31508017710BD4680BD80B483B000AF78607B68002227
S315080177201A777B680022DA777B68002283F82020A3
S315080177307B6800225A777B6800229A7700BF0C374C
S31508017740BD465DF8047B704780B586B000AF7860AA
S315080177500B46FB707B689B687B617B689B68184658
S31508017760FFF7B4FE03463B747B689B681846FFF730
S31508017770BAFE0346FB73FF237B743B7C012B01D1C5
S315080177800F237B747B689B681846FFF7EFFE034659
S31508017790FB747B689B681846FFF7F5FE0346BB73C7
S315080177A07B689B681846FFF7D4FE0346BB81FB78C6
S315080177B0602B09D9BB89002B06D0BB897A6913448A
S315080177C07B616123FB7416E07B689B681846FFF7AB
S315080177D0B3FE0346BB81FB78402B09D9BB89002B35
S315080177E006D0BB897A6913447B614123FB7402E0A5
S315080177F07B6911337B61FA78BB7B9A4204D9786835
S31508017800FFF788FF002332E0FB7CBB74BA7CBB7BA5
S315080178109A4228D87B691B78FF2B03D17B690133F0
S315080178207B6117E0BA7CFB789A4205D17969786859
S31508017830FFF70CFF7B691AE07B6902331A787B7CB8
S315080178401340DBB21A467B6913447B61FB7B7A6979
S3150801785013447B61BA7CBB7B9A4203D0BB7C013360
S31508017860BB74D7E700BF7868FFF754FF00231846B3
S315080178701837BD4680BD80B58CB002AFF8600846A2
S3150801788011461A4603467B810B463B811346FB711B
S31508017890FB791946F868FFF757FFB861BB69002BF2
S315080178A001D1002379E0FB689B68B9691846FFF79F
S315080178B0BDFE7862FB68DB7FFB75FB6893F82030B9
S315080178C0BB75FB6893F91D309AB27B8913447B819A
S315080178D0FB6893F91E309BB23A89D31A3B813B89DF
S315080178E0013B3B81BB7D9BB23A89D31A9BB20133DB
S315080178F09AB2FB7D98B2BB7D9BB279890093034608
S31508017900F868FFF73CFA0346002B03D1FB6893F9A5
S315080179101C3042E0FB7D0733FB75FB7DDB08FB75FD
S315080179203B89FB83BB7D9BB2FA8BD31AFB83FB8B0B
S315080179300133FB83002387F8223026E07B893B84C9
S31508017940002387F8233013E07B6A1B78FA8B398C7E
S3150801795000930023F86800F0ABFB7B6A01337B6276
S315080179603B8C08333B8497F82330013387F823305F
S3150801797097F82320FB7D9A42E6D3FB8B0133FB83E1
S3150801798097F82230013387F8223097F82220BB7DF9
S315080179909A42D3D3FB6893F91C3018462837BD465B
S315080179A080BD80B586B000AFF8607B600B467B81F1
S315080179B013463B810023FB82FB685B6AF86898479C
S315080179C003461A463B8913443B8117E07B681B78BB
S315080179D03A897989F868FFF74EFF03467B7597F967
S315080179E015309AB27B8913447B8197F915309AB27F
S315080179F0FB8A1344FB827B6801337B607B681B78B7
S31508017A00002BE3D1FB8A18461837BD4680BD80B5E1
S31508017A1084B000AF78607B689B68002B6BD07B686D
S31508017A2093F82830002B14D17B689B681846FFF71A
S31508017A3076FD03465AB27B6883F829207B689B68E2
S31508017A401846FFF7ADFD03461A467B6883F82A20D8
S31508017A502DE07B6893F82830012B14D17B689B684D
S31508017A601846FFF7C7FD03461A467B6883F829209F
S31508017A707B689B681846FFF7CBFD03461A467B6869
S31508017A8083F82A2013E07B689B681846FFF796FD62
S31508017A9003461A467B6883F829207B689B68184643
S31508017AA0FFF79AFD03461A467B6883F82A207B6806
S31508017AB093F929301AB27B6893F92A301BB2D31A83
S31508017AC01BB2FB817B6893F82B30402B0DD0FB89C9
S31508017AD0DBB2FB817B6893F82B309BB2FA8912FBE8
S31508017AE003F3FB81FB899B09FB81FB89DAB27B687E
S31508017AF083F82C2000E000BF1037BD4680BD80B555
S31508017B0082B000AF78607B68002283F82820786805
S31508017B10FFF77DFF00BF0837BD4680BD80B582B03F
S31508017B2000AF78607B68012283F828207868FFF720
S31508017B306EFF00BF0837BD4680BD80B483B000AF75
S31508017B407860002318460C37BD465DF8047B7047FC
S31508017B5080B483B000AF78607B68044A5A6200BF7C
S31508017B600C37BD465DF8047B704700BF3B7B0108B7
S31508017B7080B485B000AF78607B6893F92930FB81C2
S31508017B80FB890133FB81FB8918461437BD465DF82D
S31508017B90047B704780B483B000AF78607B68044A81
S31508017BA05A6200BF0C37BD465DF8047B704700BFBB
S31508017BB0717B010880B584B000AF78603960002315
S31508017BC0FB813B681B787B737B7B002B0FD07B7B10
S31508017BD019467868FFF7B8FD7B6893F91C309AB2A5
S31508017BE0FB891344FB813B6801333B60E9E700BF2E
S31508017BF0FB8918461037BD4680BD80B582B000AFF7
S31508017C00786039607B689B683A689A4208D07B68D5
S31508017C103A689A607868FFF7FAFE7868FFF798FF7E
S31508017C2000BF0837BD4680BD90B585B000AFF86086
S31508017C30B9603B601346FB71BB681C68FA793B68FF
S31508017C40B968F868A047034618461437BD4690BD7B
S31508017C5080B584B000AF786039607B689B6B022081
S31508017C60984700230A2239687868FFF7DDFF03463B
S31508017C70FB737B689B6B032098477B689B6B002093
S31508017C809847FB7B18461037BD4680BD80B582B044
S31508017C9000AF786039607B689B6B022098477B68E8
S31508017CA09B6B012098470023142239687868FFF7EF
S31508017CB0BBFF7B683C33172239687868FFF7B4FF46
S31508017CC07B689B6B0020984700BF0837BD4680BD7F
S31508017CD080B584B000AF786039607B689B6B022001
S31508017CE098477B689B6B01209847002315223968C2
S31508017CF07868FFF799FF0346FB73FB7B002B06D0D9
S31508017D007B683C33172239687868FFF78DFF7B68F3
S31508017D109B6B00209847FB7B18461037BD4680BDF4
S31508017D2080B584B000AF786039607B689B6B0220B0
S31508017D3098477B689B6B0120984700231622396870
S31508017D407868FFF771FF0346FB73FB7B002B06D0B0
S31508017D507B683C33172239687868FFF765FF7B68CB
S31508017D609B6B00209847FB7B18461037BD4680BDA4
S31508017D7080B584B000AFF860B9601346FB71FB1D8E
S31508017D800F22B968F868FFF74FFF03461846103700
S31508017D90BD4680BD80B586B000AFF860B9601146B2
S31508017DA01A460B46FB801346BB80FB682E337B6164
S31508017DB07B69FA881A807B69BA885A807B6932227C
S31508017DC0B968F868FFF730FF00BF1837BD4680BDB0
S31508017DD080B586B000AFF860B96011461A460B4601
S31508017DE0FB801346BB80FB682E337B617B69FA886F
S31508017DF01A807B69BA885A807B6997F820205A715C
S31508017E007B6997F824201A717B693B22B968F8685F
S31508017E10FFF70AFF00BF1837BD4680BD80B584B09D
S31508017E2000AF7860396007F10E0346223968786831
S31508017E30FFF7FAFEFB8918461037BD4680BD80B5A7
S31508017E4084B000AF7860396007F10E0347223968BC
S31508017E507868FFF7E9FEFB8918461037BD4680BDED
S31508017E6080B582B000AF786039600023482239684E
S31508017E707868FFF7D9FE03469BB218460837BD4610
S31508017E8080BD80B582B000AF78607B685B681946B3
S31508017E907868FFF7C3FF03461A467B681A807B6832
S31508017EA05B6819467868FFF7CAFF03461A467B6876
S31508017EB05A807B685B6819467868FFF7D1FF0346E5
S31508017EC0DAB27B68DA747B6859687B683C331722B7
S31508017ED07868FFF7A9FE00BF0837BD4680BD0000D8
S31508017EE080B582B000AF78607B6800229A607B68B3
S31508017EF00022DA607B6800225A747B6801221A74B0
S31508017F007B6822229A747B6800229A61012178682B
S31508017F1000F0EBF87868FFF71BFE7B68012283F80F
S31508017F2028207B68002283F829207B68002283F8B1
S31508017F302A207B68402283F82B207B68002283F85D
S31508017F402C207B68024A9A6300BF0837BD4680BD6C
S31508017F507D8C010880B582B000AF78607B685B686C
S31508017F6019467868FFF774FE0346002B01D10023F2
S31508017F7003E07868FFF785FF012318460837BD46F1
S31508017F8080BD80B584B000AFF860B9607A60F868E2
S31508017F90FFF7A6FFFB68BA685A60FB685B687A68F0
S31508017FA09A60F868FFF7D6FF034618461037BD46AC
S31508017FB080BD80B582B000AF78607B685B68194682
S31508017FC07868FFF763FE00BF0837BD4680BD80B5F8
S31508017FD082B000AF78607B689B69002B03D07B6811
S31508017FE09B69786898477B685B6819467868FFF7E4
S31508017FF06FFE034618460837BD4680BD80B582B078
S3150801800000AF78607B689B69002B03D07B689B690E
S31508018010786898477B685B6819467868FFF780FE39
S31508018020034618460837BD4680BD80B582B000AF05
S3150801803078600B46FB707B685B68FA781946786846
S31508018040FFF796FE034618460837BD4680BD80B53C
S3150801805082B000AF78607B6859680023102278687F
S31508018060FFF7E2FD00BF0837BD4680BD80B582B087
S3150801807000AF78607B685968002311227868FFF79A
S31508018080D3FD00BF0837BD4680BD80B582B000AFBD
S3150801809078600B467B8013463B807B6859683B8832
S315080180A07A887868FFF776FE00BF0837BD4680BD37
S315080180B080B586B002AFF860084611461A460346EF
S315080180C07B810B463B811346FB71FB6859683889EE
S315080180D07A893B7E0193FB7900930346F868FFF79B
S315080180E077FE00BF1037BD4680BD80B483B000AFB0
S315080180F078600B46FB707B68FA7883F8342000BFFA
S315080181000C37BD465DF8047B704780B485B000AF77
S3150801811078607B68DB7CFB73FB7B282B01D1FF2313
S3150801812006E07B68DB7C022B01D1032300E00123F7
S3150801813018461437BD465DF8047B704780B582B092
S3150801814000AF78607B68DB7C302B08D17B68FF2227
S3150801815083F834207B68FF2283F8352007E07868A6
S31508018160FFF7D3FF034619467868FFF7BEFF00BF3E
S315080181700837BD4680BD80B483B000AF78607B68A0
S3150801818000229A807B681A887B68DA807B68DB889C
S31508018190013B9AB27B68DA807B6800221A7200BFBB
S315080181A00C37BD465DF8047B704790B482B000AFCA
S315080181B078607B689A887B681B8813449AB27B68C7
S315080181C09A807B689A887B685B889A4201D30023E8
S315080181D018E07B681B7A0133DAB27B681A727B680E
S315080181E0DC887B681B8823449CB27B685B889C423D
S315080181F004D37B685C882346013B9CB27B68224694
S31508018200DA80012318460837BD4690BC704780B40A
S3150801821085B000AF78600B467B8013463B807B6850
S31508018220DB887A889A4294BF01230023DBB2FB7369
S315080182307B689B883A889A422CBF01230023DBB2CC
S31508018240BB737A883B889A428CBF01230023DBB231
S315080182507B73FB7B3B73FA7BBB7B1340FB73BA7B5C
S315080182607B7B1340BB737A7B3B7B13407B73FA7B27
S31508018270BB7B1343FB73FA7B7B7B1343FB73FB7B50
S3150801828003F00103DBB218461437BD465DF8047BDB
S31508018290704780B483B000AF786039603B680022CC
S315080182A01A807B689A883B685A807B685A893B683A
S315080182B09A803B689B88013B9AB23B689A807B68A7
S315080182C0DA883B68DA8000BF0C37BD465DF8047B67
S315080182D07047000080B584B000AF786039603B68AC
S315080182E05B88FB81FB89BB813B685B79032B13D8D0
S315080182F001A252F823F000BF198301080983010876
S315080183001983010811830108BB890833BB8103E07E
S31508018310FB89083BFB8100BFBA89FB891946786846
S31508018320FFF775FF034618461037BD4680BD00BFE7
S3150801833080B485B000AF78607B68DB68FB60FB685A
S31508018340BB607B685B891A46BB681344BB607B6864
S315080183505B891A46BB681344BB60FB685A1CFA6002
S3150801836000221A70FA68BB689A42F6D100BF00BFAC
S315080183701437BD465DF8047B7047B0B487B000AFCB
S31508018380F860084611461A4603467B810B463B812F
S315080183901346FB71FB68DB687B61FB689B883A893E
S315080183A0D31A3B81FB685C89A3089CB23B89DBB283
S315080183B09BB214FB03F39CB222467B6913447B618F
S315080183C07C89A3089CB222467B6913447B617C891C
S315080183D004F003039CB263009CB297F82830002B83
S315080183E00DD103252A46234602FA03F3DDB2EB43F0
S315080183F0DDB27B691B782B40DAB27B691A70FB798F
S3150801840003F00303FB71FB7922469340FB717B69F9
S315080184101A78FB791343DAB27B691A7000BF1C37E5
S31508018420BD46B0BC704780B586B002AFF860B9608A
S315080184301346FB71BB685A88FB689B889A4218D316
S31508018440BB685A88FB68DB889A4214D8BB681A88C5
S31508018450FB685B899A4210D2BB681988BB685A883F
S31508018460BB689879FB7900930346F868FFF785FF9F
S3150801847004E000BF02E000BF00E000BF1037BD46C0
S3150801848080BD000090B583B000AF786039603B6865
S315080184901C7963B2002B04DA002239687868FFF781
S315080184A0C2FF3B685B79032B26D801A252F823F059
S315080184B0C1840108CF840108DD840108EB84010821
S315080184C03B681B8801339AB23B681A8014E03B6803
S315080184D05B8801339AB23B685A800DE03B681B887A
S315080184E0013B9AB23B681A8006E03B685B88013B10
S315080184F09AB23B685A8000BF6300DCB2002CC8D12F
S3150801850000BF00BF0C37BD4690BD00BF90B583B014
S3150801851000AF786039603B681C7924F03F03DAB212
S315080185203B689A713B689B799B09DAB23B689A71F9
S31508018530012239687868FFF776FF3B685B79032B78
S3150801854026D801A252F823F0598501086785010842
S3150801855075850108838501083B681B8801339AB232
S315080185603B681A8014E03B685B8801339AB23B6822
S315080185705A800DE03B681B88013B9AB23B681A801A
S3150801858006E03B685B88013B9AB23B685A8000BFAC
S31508018590A300DCB2002CC0D100BF00BF0C37BD461A
S315080185A090BD00BF80B586B000AFF860B9603B608A
S315080185B01346FB71BB685B687B61FB790A3B3E2B03
S315080185C000F2D38001A252F823F000BF6B8701089D
S315080185D06B8701086B8701086B8701086B870108A0
S315080185E06B8701086B8701086B8701086B87010890
S315080185F06B87010803870108138701082D8701087E
S31508018600478701086B8701086B8701086B87010893
S315080186106B8701086B8701086B8701086B8701085F
S315080186206B8701086B8701086B8701086B8701084F
S315080186306B8701086B8701086B8701086B8701083F
S315080186406B8701086B8701086B8701086B8701082F
S315080186506B870108F7860108ED8601086B87010813
S315080186606B8701086B8701086B870108E18601089A
S315080186706B8701086B8701086B8701086B870108FF
S315080186806B8701086B8701086B8701086B870108EF
S31508018690C98601086B8701086B8701086B87010882
S315080186A06B8701086B8701086B8701086B870108CF
S315080186B06B8701086B8701086B87010851870108D9
S315080186C05B8701086587010839687869FFF702FE43
S315080186D00346002B48D039687869FFF7D3FE43E093
S315080186E0002239687869FFF79EFE3EE039687869A5
S315080186F0FFF70CFF39E0012239687869FFF793FE25
S3150801870033E07B691846FFF736FD7869FFF710FEF7
S315080187102BE07B691846FFF748FD0346002B01D17C
S31508018720002323E07869FFF703FE1EE07B691846FC
S31508018730FFF73BFD0346002B01D1002316E07869BC
S31508018740FFF7F6FD11E039687869FFF7A2FD0CE03D
S315080187507B695A893B681A8007E07B695A883B68B6
S315080187601A8002E0022301E000BF012318461837E8
S31508018770BD4680BD80B588B002AFF860084611468F
S315080187801A4603467B810B463B811346FB80FF2332
S31508018790FB750DE03A897989FB7D00930023F8681A
S315080187A0FFF786FCFB88083BFB807B8908337B81C6
S315080187B0FB88072BEED8FB88002B15D0FB8883F0A6
S315080187C00703FB80FB880133FB80FA7DFB8803F0F6
S315080187D0070302FA03F3FB753A897989FB7D00934E
S315080187E00023F868FFF764FC00BF1837BD4680BD53
S315080187F080B588B002AFF860084611461A460346A6
S315080188007B810B463B811346FB80FF23FB750DE0FD
S315080188103A897989FB7D00930123F868FFF748FCBB
S31508018820FB88083BFB803B8908333B81FB88072B88
S31508018830EED8FB88002B15D0FB8883F00703FB8055
S31508018840FB880133FB80FA7DFB8803F0070302FAF4
S3150801885003F3FB753A897989FB7D00930123F8684F
S31508018860FFF726FC00BF1837BD4680BD80B588B026
S3150801887002AFF860084611461A4603467B810B4645
S315080188803B811346FB807B89FB82F8883A89798983
S315080188903B8C00930346F868FEF771FA0346002BF2
S315080188A026D0FB883A897989F868FFF763FF3B8CFC
S315080188B03A897989F868FFF79BFF7A89FB88134417
S315080188C07B817B89013B7B813B8C3A897989F86875
S315080188D0FFF78EFF3A893B8C13443B813B89013B69
S315080188E03B81FB883A89F98AF868FFF743FF00E07C
S315080188F000BF1837BD4680BD80B584B000AFF860AB
S31508018900084611461A4603467B810B463B811346A8
S31508018910FB80FB883A897989F868FFF72BFF3B8941
S3150801892001333B813B8B013B3B833B8B002BF0D1D6
S3150801893000BF00BF1037BD4680BD80B586B002AF07
S31508018940F860084611461A4603467B810B463B8169
S315080189501346FB80F8883A8979893B8B009303464D
S31508018960F868FEF70CFA0346002B09D0F8883A890D
S3150801897079893B8B00930346F868FFF7BDFF00E052
S3150801898000BF1037BD4680BD80B485B000AFF86022
S31508018990B9603B601346FB71002318461437BD4680
S315080189A05DF8047B7047000080B582B000AF78603F
S315080189B07B685B68074A934207D1064B5A687B680E
S315080189C05A607868FFF75DFA00E000BF0837BD46D0
S315080189D080BD00BF3C00002080B582B000AF786042
